S02B0000443A2F5265702F626D732D6D696E692D732F626D732D6D696E692D732D6669726D776172652F636DA1
S3150801000000000220452F0608912F0608E9F3050886
S31508010010EFF30508F5F30508FBF3050800000000F2
S315080100200000000000000000000000001DE00608B6
S31508010030912F060800000000ADE00608BDE006089D
S31508010040912F0608912F0608912F0608912F060869
S31508010050912F0608912F0608912F0608912F060859
S31508010060912F0608912F0608912F0608912F060849
S31508010070912F0608912F0608912F0608912F060839
S31508010080912F0608912F0608912F0608DD410608CB
S31508010090CD410608912F0608ED410608912F06085D
S315080100A0912F0608912F0608912F0608912F060809
S315080100B041D10308912F0608912F0608912F0608AA
S315080100C0912F0608912F0608912F0608912F0608E9
S315080100D0912F0608912F0608912F0608912F0608D9
S315080100E0912F0608912F0608912F0608912F0608C9
S315080100F0912F0608912F0608912F0608912F0608B9
S31508010100912F0608F5810508912F0608912F0608F3
S31508010110912F0608912F0608912F0608912F060898
S31508010120912F0608912F0608912F0608D5810508F3
S31508010130912F060829C90708912F06080D420608B6
S31508010140FD410608912F06081D420608912F06084B
S31508010150912F0608E5810508912F0608912F0608B3
S31508010160912F0608912F0608912F0608912F060848
S31508010170912F0608912F0608912F06080000000006
S31508010180912F06080000000010B5054C237833B9F5
S31508010190044B13B10448AFF300800123237010BD4B
S315080101A0601F00200000000064950C0808B5034B89
S315080101B01BB103490348AFF3008008BD00000000E6
S315080101C0641F002064950C08A3F5803A704700BFA8
S315080101D0174B002B08BF134B9D46FFF7F5FF002170
S315080101E08B460F461348144A121A77F0A9FC0E4B90
S315080101F0002B00D098470D4B002B00D098470020C4
S31508010200002104000D000D48002802D00C4851F0C9
S315080102100DFD76F069FE2000290060F0EFFD51F032
S31508010220ABFF00BF00000800000000005D0D0708D5
S3150801023000000220601F0020A06A01202D1C06086C
S315080102400000000010B5044608304EF089FC20462F
S3150801025010BD10B5044600F5C87052F012FB04F53E
S31508010260C47034F0BBFF20685EF030FE204610BD36
S31508010270012800D070474FF6FF739942FAD170B53D
S31508010280134C204635F016F8124E324612492046CE
S3150801029051F0CAFC114C204648F0AAF932461049D9
S315080102A0204651F0C1FC0F4D2C464FF47A7344F8A1
S315080102B0083B20464EF012FD002385F820302046E3
S315080102C04EF059FC32460849284651F0ADFC70BD3E
S315080102D0B01F002088010020530201087C1F00205E
S315080102E0D1850508881F0020450201082DE9F04F30
S315080102F0A1B023F0BBFFB24851F00CF8B14877F032
S31508010300EFFF24F0FBF8002800F0E380012424F035
S31508010310CFF802462146AC484FF00AFD01230622D2
S315080103201946AA484FF004FD24F0CEFAA84877F0FA
S31508010330D7FF23F0CDFF26F0D9FF24F0B3F826F036
S31508010340DBFFA44877F0CCFF1EA824F06FFF1EA898
S3150801035024F0E8FF24F0B2FD42F012FF002840F035
S31508010360BA8024F093F8044624F094F8054624F05C
S3150801037089F8064619F074FE034632462946204690
S3150801038039F08EFE944877F0ABFF23F09BFF0F9070
S3150801039023F09EFF109019F067FE119019F068FE80
S315080103A0044619F069FE129019F06AFE139019F0C5
S315080103B06FFE149019F070FE159019F071FE05463E
S315080103C019F072FE064619F05FFE074619F070FE2F
S315080103D0804619F071FE814619F072FE824619F0BF
S315080103E073FE834619F074FE0C90CDF82CB0CDF847
S315080103F028A0CDF82490CDF8208007970696059574
S3150801040015990491149903911399029112990191DD
S315080104100094119B109A71490F9835F05DFB70484D
S3150801042077F05EFF00220023CDE91C23CDE91E23C8
S315080104301CA9AC2025F06AFF1EA9AD2025F066FF90
S315080104401E9A1F9B1C9991421D99994101DA1C928A
S315080104501D9323F03DFF614DDDE91C23294619F063
S31508010460CFFD604877F03CFF23F024FF044623F0D4
S3150801047025FF064624F094F80246314620463AF00E
S31508010480B1F8594877F02CFF24F074F8044624F0A3
S3150801049081F8064624F084F8074623F019FF0090F0
S315080104A02B463A46314620463AF0AAFC4F4877F0A1
S315080104B017FF24F031F8044623F00AFF02462946BD
S315080104C020463AF0ADFA4A4877F00AFF00252E464B
S315080104D09DE002241BE742F079FE42F07DFE454885
S315080104E077F0FEFE3DE723F0ABFF434B93F8203050
S315080104F0002B3AD1F8B941484EF0B9FB3E4B93F877
S315080105002030002B00F0A1800021344B18685EF0E2
S3150801051089FC044618B10122114634F09BFF002CD0
S3150801052000F093800121204634F0A2FF21462B4892
S3150801053034F0F6FE89E0304C04F1080116A84EF0B5
S3150801054072FB23684FF47A7202FB03F3DA171699E2
S315080105508B42179B72EB0303D0DA04F108004EF0C5
S3150801056086FB012384F82030C8E718B123484EF0EA
S315080105707EFBC3E7204C04F1080116A84EF053FB95
S3150801058023684FF47A7202FB03F3DA1716998B4242
S31508010590179B72EB0303B1DA04F108004EF067FB0F
S315080105A0002384F82030A9E7204634F06BFE0028A2
S315080105B058D02146094B18685EF058FC52E000BF36
S315080105C0154E0308642909087429090888290908A0
S315080105D0A0290908B0290908E0290908B01F00203F
S315080105E0FC290908142A0908282A0908382A0908A1
S315080105F0482A0908C8290908881F0020901F0020D1
S31508010600AD201AA925F09AFE022051F0FBFF3AF017
S3150801061043F83AF03FF90DF16701C52026F096FB3C
S315080106209DF86730002B3FF45EAF234C204647F018
S31508010630E5FF204647F0E8FF003818BF01208DF88E
S3150801064078001EA9CD2026F097FB01211B4834F01E
S315080106507BFE044630B134F023FE204634F012FE08
S315080106600028A1D1002051F075FF1A901B91B142C3
S3150801067008BFA84201D005460E463C22002380F059
S31508010680B5FF1343C0D100220023CDE91C23CDE9D0
S315080106901E231CA9AC2025F039FE1EA9AD2025F084
S315080106A035FE1C9A1E9B9A421D9A1F9B72EB0303E9
S315080106B0A6DAAC20A5E700BF7C1F0020B01F0020EA
S315080106C008B54FF6FF710120FFF7D2FD08BD0000FE
S315080106D000B970470EB400B582B004AA0192054B61
S315080106E01B680399D8684FF096FB02B05DF804EBD6
S315080106F003B07047E014002048F2835303800023B7
S315080107008370704710B50446FFF7F6FF204610BD03
S31508010710807870470388C3F30E03038043EAC13325
S31508010720038070470088C0F342207047038823F48A
S3150801073060639BB2038043EA4123038070470088C4
S31508010740C0F302307047038823F4E0439BB2038069
S3150801075043EA013303807047038823F480739BB20D
S31508010760038043EA012303807047038823F0E003EB
S315080107709BB2038043EA411303807047016002710B
S315080107800022427170474171704700002DE9F0431C
S3150801079085B004460E461746006803681B689847E5
S315080107A0002516E0206803681B699847022051F066
S315080107B02DFF40465EF0A6F8207940006B1C019398
S315080107C090300090334602224B496079FFF780FF4B
S315080107D00135022D00F388805EF05CF880462068BA
S315080107E04DF05DFA022051F011FF2179490090314F
S315080107F020684DF027FA0128D4D1314620684DF0FA
S3150801080021FA0128CED120684DF058FA022051F07C
S31508010810FDFE20684DF043FA022051F0F7FE2179DA
S315080108204900903141F0010120684DF00BFA012889
S3150801083016D0206803681B699847022051F0E6FE26
S3150801084040465EF05FF823795B006A1C019290339B
S3150801085000933346022228496079FFF739FFB7E743
S315080108604FF0000906E009F110036B4403F8040C84
S3150801087009F10109B9F1010F07DC012120684DF0E1
S31508010880F4F90028EFDA012300E00023B3B1206868
S3150801089003681B699847022051F0B8FE40465EF08E
S315080108A031F823795B006A1C019290330093334631
S315080108B0022212496079FFF70BFF89E720684DF09C
S315080108C0FDF9022051F0A2FE40465EF01BF82068B1
S315080108D003685B6898479DF80C209DF80D3043EA3C
S315080108E002233B80012004E0206803685B6898477F
S315080108F0002005B0BDE8F083542A0908AC2A090886
S3150801090010B582B00C460DF106020121FFF73EFF34
S3150801091040B1BDF80630C3F30E032380BDF8063097
S31508010920DB0BA37002B010BD08B50A460021FFF71C
S315080109302DFF08BD2DE9F04184B004460E46130A81
S315080109408DF80C308DF80D20006803681B689847F0
S31508010950002516E0206803681B699847022051F0B4
S3150801096055FE38465DF0CEFF227952006B1C019385
S31508010970903200923346022230496079FFF7A8FE89
S315080109800135022D52DC5DF085FF074620684DF0E2
S3150801099086F9022051F03AFE217949009031206802
S315080109A04DF050F90128D5D1314620684DF04AF964
S315080109B00128CFD14FF00008B8F1010F0CD808F182
S315080109C010036B4413F8041C20684DF03BF9012809
S315080109D01BD108F10108EFE70023C3B120680368BA
S315080109E01B699847022051F011FE38465DF08AFFCF
S315080109F023795B006A1C01929033009333460222E5
S31508010A000F496079FFF764FEBAE70123E5E7206835
S31508010A104DF054F9022051F0F9FD38465DF072FFA8
S31508010A20206803685B689847012004E0206803682A
S31508010A305B689847002004B0BDE8F081FC2A0908E4
S31508010A40542B090808B50A880121FFF773FF08BD69
S31508010A500020704708B503681B69012200219847E1
S31508010A6008BD08B503681B6900221146984708BDE9
S31508010A706FF01500704709B1002070476FF0180034
S31508010A8070470120704784B001A880E80E0004B0C1
S31508010A9070476FF01C0070476FF01C0070476FF0CD
S31508010AA0150070476FF01500704701207047012047
S31508010AB07047002070470020704770B504468EB213
S31508010AC011F0010F05D1002516F0100F08D128469F
S31508010AD070BD4DF04EFE08B90025F5E70125F3E78F
S31508010AE020464DF057FE0028F1D045F01005EEE7F7
S31508010AF0A0F1E800FFF7E1BF7AB138B504460D4623
S31508010B0003681B68984720464DF0DAFE287023686B
S31508010B105B6820469847012038BD00207047A0F140
S31508010B20E800FFF7E9BF0AB9002070472DE9F0414F
S31508010B3006460F46154650F0F9F980F0010010F007
S31508010B40FF0803D033681B6830469847002404E041
S31508010B50395D30464DF0B9FE0134AC42F8D3B8F1EF
S31508010B60000F03D033685B68304698472846BDE8CE
S31508010B70F081A0F1E800FFF7D6BF08B54DF0B2FE47
S31508010B80002008BDA0F1E800FFF7F7BF08B54DF052
S31508010B9003FF002008BDA0F1E800FFF7F7BF00003A
S31508010BA010B50446084B03F1080202604433C0F845
S31508010BB0E830EC3051F065FE044BC4F8E8302046C5
S31508010BC04DF04AFE204610BDA42B0908D4480C084E
S31508010BD010B50446094B03F1080240F8E82C4433E2
S31508010BE044F8E839043051F04CFE054BC4F8E830B6
S31508010BF020464DF031FE204610BD00BFA42B090842
S31508010C00D4480C0810B504460B4B03F108020260E0
S31508010C104433C0F8E830EC3051F033FE074BC4F8E2
S31508010C20E83020464DF018FE4FF48871204651F001
S31508010C3035FB204610BD00BFA42B0908D4480C0873
S31508010C4010B504460B4B03F1080240F8E82C44336F
S31508010C5044F8E839043051F014FE074BC4F8E8307B
S31508010C6020464DF0F9FD4FF48871204651F016FBE8
S31508010C70204610BDA42B0908D4480C0810B5044613
S31508010C804DF0F6FC074BC4F8E830074B03F10802B0
S31508010C9022604433C4F8E83004F1EC0051F072FDE7
S31508010CA0204610BDD4480C08A42B090808B54DF0F8
S31508010CB060FD08BD84B000B583B00DF1140C8CE855
S31508010CC00E009DF824300193089B00939CE80E00C2
S31508010CD04DF071FD03B05DF804EB04B0704708B53B
S31508010CE04DF0EEFD08BD08B54DF01EFF08BD08B56F
S31508010CF04DF02CFD08BD08B5EC3051F051FD08BD8D
S31508010D0008B5EC3051F09CFD08BDF0B583B004463A
S31508010D100D4616461F46FFF7EEFF089B00933B4616
S31508010D203246294620464DF0D3FE05462046FFF7B2
S31508010D30E7FF284603B0F0BD10B50446074B40F857
S31508010D405C3B51F09EFD04F130004DF009FF04F1C2
S31508010D5018004DF005FF204610BD00BF382C0908C4
S31508010D6010B50446FFF7E8FF8021204651F096FAB0
S31508010D70204610BD0160027143717047F8B50446FB
S31508010D8006461A4B46F8183B30464DF0A7FF04F1C4
S31508010D90300738464DF0A2FF0025A4F84850A4F8BC
S31508010DA04A5084F84C5084F84D50002323656365F6
S31508010DB084F8585084F8595084F85A5084F85B508E
S31508010DC004F15C0051F0DEFC25714FF47A63A360EF
S31508010DD04FF47A73E360064B2361257530464DF06F
S31508010DE0CAFE38464DF0C7FE2046F8BD382C09081C
S31508010DF0CDCCC441F8B5067D002E36D004460D4645
S31508010E004B7B8BBB0A6840F221339A4201D00026FC
S31508010E102BE008794B798A79CF7947EA022743EAA1
S31508010E20002080F069F9124980F072FA2065384687
S31508010E3080F062F90E4980F06BFA60652B7A84F8C6
S31508010E405830EB7A84F8593004F15C05284651F09C
S31508010E50A7FC012384F85B30284651F0F1FC04F124
S31508010E6018004DF004FF00E000263046F8BD00BF2B
S31508010E7000002041F0B587B00446037DCBB100F1EF
S31508010E80180528464DF0E9FEA3684FF47A7202FB6D
S31508010E9003F3984220D804F1300528464DF0DDFECB
S31508010EA0E3684FF47A7202FB03F398422AD807B033
S31508010EB0F0BD18304DF0DBFE04F130004DF0D7FEE1
S31508010EC004F15C05284651F06BFC002384F85B307D
S31508010ED0284651F0B5FCEAE7002323656365002639
S31508010EE084F8586084F8596004F15C07384651F073
S31508010EF057FC84F85B60384651F0A2FC28464DF051
S31508010F00B6FEC8E700260096019604F15C07384646
S31508010F1051F046FCB4F848301A0A8DF800208DF8CD
S31508010F200130B4F84A301A0A8DF802208DF80330D8
S31508010F3094F84C308DF8043094F84D308DF805301E
S31508010F40384651F07DFC08238DF814308DF816606B
S31508010F508DF8156040F22313029303AB6A4692E8B3
S31508010F60030083E8030002A920792BF073FE2846C3
S31508010F704DF07DFE9BE7043070470000037D03B901
S31508010F80704770B504460D4600F15C06304651F0CF
S31508010F9007FC1249206980F007F980F007FBA4F8DD
S31508010FA048002B7923B194F85B3013B1012300E093
S31508010FB0002384F84C307BB10849286880F0F4F89E
S31508010FC080F0F4FA80B2A4F84A006B7984F84D30BF
S31508010FD0304651F035FC70BD0020F4E70000204191
S31508010FE0006D7047406D704790F85800704738B5E6
S31508010FF0044600F15C05284651F0D2FB94F85B40A3
S31508011000284651F01DFC204638BD0000014B0360FF
S31508011010704700BF482C090810B50446FFF7F6FFCC
S315080110203821204651F03AF9204610BDC0E900237F
S31508011030009B8360019BC360029B0361039B436121
S31508011040049B8361059BC361069B03629DF81C3063
S3150801105080F824309DF8203080F82530704700004C
S3150801106030B4104A026000220284428480F82420A7
S31508011070C284028542858285C28580F8302080F83F
S31508011080312080F832204FF47A6141603C21816039
S31508011090027300240025C0E90445C0E9064530BCB1
S315080110A0704700BF482C090804307047F8B5044654
S315080110B0037B002B7AD00D4609686A680369406983
S315080110C05B1842EB00022361626129686A68A369B9
S315080110D0E0695B1842EB0002A361E26194F83030E3
S315080110E0002B6CD194F8312095F824309A4206D019
S315080110F0012384F8303000220023C4E90423A868B8
S3150801110003689B6898470646002180F0EBF900289A
S315080111107FD14FF08341304680F046F880F046FA99
S3150801112020844FF08341286980F03EF880F03EFA2A
S315080111306084012384F824304FF08341686980F084
S3150801114033F880F033FAE0844FF08341E86980F0A0
S315080111502BF880F02BFA60854FF08341286A80F0DE
S3150801116023F880F023FAA0850023E38595F8253036
S31508011170002B50D04FF08341A86980F015F880F014
S3150801118015FA80B24A4B83FB00239B0800D103461C
S3150801119094F83220002A40D0012A4CD0002384F842
S315080111A0323095F8243084F83130F8BD80F8303083
S315080111B000220023C0E90423C0E90623F5E794F8D1
S315080111C0312095F824309A4203D000220023C4E93D
S315080111D00423216962696668F00E73019B1B60F13D
S315080111E00000800040EA93709B009B1940F10000C3
S315080111F0C00040EA5370DB00994272EB0003FFF42A
S315080112007EAF002384F8303000220023C4E904238A
S3150801121075E700267DE70020B4E794F83030002B07
S31508011220BFD000220023C4E9062300232385012316
S3150801123084F83230B5E794F8302022B900232385A3
S3150801124084F83230ADE7B4F828C0844529D2A669B6
S31508011250E169A2684FF47A7707FB02F2154FA7FBFB
S315080112600272D708920F4FEA471EBEEB070E62F1CC
S315080112700002920042EA9E724FEA8E0E1EEB070E9C
S3150801128042F10002D20042EA5E724FEACE0E76457C
S3150801129071EB020205D300260027C4E906676344F9
S315080112A02385238D83427FF67CAF208579E700BFAE
S315080112B067666666CDCCCCCC90F830007047008C5A
S315080112C07047408C704790F824007047C08C70476F
S315080112D0008D7047408D7047808D7047C08D70476F
S315080112E010B50446074B40F8643B51F0CAFA04F1BD
S315080112F030004DF035FC04F118004DF031FC204664
S3150801130010BD00BF582C090810B50446FFF7E8FFC1
S315080113108821204650F0C2FF204610BD0180827008
S31508011320C3709DF80030037170470000F8B5044694
S3150801133006461E4B46F8183B30464DF0CFFC04F1E5
S31508011340300738464DF0CAFC0025A4F84A50A4F8DF
S315080113504C50A4F84E50A4F85050A4F8525084F8B2
S31508011360545084F8555084F8565084F85750A4F8C8
S315080113705850E56584F86050A4F8625004F1640099
S3150801138051F000FA25710123637141F28833A36094
S315080113904FF4FA73E360F6232382A57430464DF0C1
S315080113A0EAFB38464DF0E7FB2046F8BD582C0908FC
S315080113B010B5847C002C60D04B7B002B5CD10A686D
S315080113C04379013B1B0103F2053C62450DD003F24B
S315080113D0063C624525D003F2073C62453CD003F53D
S315080113E042739A4244D0002447E00B79A0F84A3068
S315080113F08A794B7943EA0223A0F84C300A7ACB79E9
S3150801140043EA0223A0F84E308A7A4B7A43EA02234A
S31508011410A0F85230CB7A80F8543018304DF027FCBA
S315080114202BE091F9043080F8553091F9053080F8B0
S315080114305630CA798B7943EA0223A0F850304A7AA2
S315080114400B7A43EA0223A0F858308B7A80F8573092
S3150801145018304DF00CFC10E08A794B791B0243EAEF
S3150801146002430A791343C36518304DF000FC04E0C2
S3150801147018304DF0FCFB00E00024204610BD70B585
S3150801148086B00446837CCBB100F1180528464DF099
S31508011490E4FBA3684FF47A7202FB03F3984215D86A
S315080114A004F1300528464DF0D8FBE3684FF47A720B
S315080114B002FB03F3984223D806B070BD18304DF0ED
S315080114C0D6FB04F130004DF0D2FBF5E70023A4F872
S315080114D04A30A4F84C30A4F84E30A4F85030A4F899
S315080114E0523084F8543084F8553084F8563084F8EC
S315080114F05730A4F85830E36528464DF0B8FBCFE7D6
S3150801150000230093019304F16406304651F048F92B
S3150801151094F86030C3B301238DF80030B4F8623013
S315080115208DF801301B0A8DF80230238A8DF80330B5
S315080115301B0A8DF80430B4F848308DF805301B0ABB
S315080115408DF80630304651F07BF96379013B1B0172
S3150801155003F5407307228DF8142000228DF8162012
S315080115608DF8152002936B4693E803000390ADF8B6
S315080115701010090C8DF8121002A920792BF06AFBBC
S3150801158028464DF074FB97E70023C5E704307047FA
S31508011590837C03B9704770B504460D4600F16406AD
S315080115A0304651F0FDF82B88A4F84830AB7843B1A2
S315080115B0EB7833B9B4F84A301BB1012384F86030AB
S315080115C002E0002384F8603094F860303BB14FF4B0
S315080115D07A73A4F86230304651F032F970BD0023AF
S315080115E0A4F86230F7E7B0F84A007047B0F84C0043
S315080115F07047B0F84E007047B0F850007047B0F821
S315080116005200704790F85400704790F9550070479A
S3150801161090F95600704790F857007047B0F858008F
S315080116207047C06D704710B443695B8801F5C064A3
S31508011630426852F833209269146001F5B064426831
S3150801164052F83320926A1460426852F833309B6B21
S31508011650197010BC704743695B88426852F8332099
S3150801166092694FF4C0611160426852F83320926A58
S315080116704FF4B0611160426852F833309B6B002217
S315080116801A707047014B0360704700BF682C090840
S3150801169010B50446FFF7F6FF6021204650F0FEFD1F
S315080116A0204610BDF0B58DB004460D465D4B1B684E
S315080116B053B15C4B1B68013B062B1FD8DFE803F0CF
S315080116C00B20355677889D00FFF7ADFF554A1368FD
S315080116D001331360EDE717238DF8203000230493B7
S315080116E0514A039208AA0292052201920122009206
S315080116F042F21002294620462FF09CF80DB0F0BDA3
S315080117004FF48063ADF8203000230493464A0392D0
S3150801171008AA0292062201920222009242F21102BC
S31508011720294620462FF086F8E8E700260896099606
S315080117300A960B9607AA41F209013C4845F006FFAD
S31508011740036808AF9968384677F0B2FC0496364BB9
S31508011750039302970923019310230093334642F218
S315080117601202294620462FF065F8C7E70026089693
S3150801177009960A960B9607AA41F20A012B4845F0E3
S31508011780E5FE036808AF9968384677F091FC049638
S31508011790254B03930297092301931023009333469C
S315080117A042F21302294620462FF044F8A6E7002301
S315080117B004931D4A03921E4A02920922019210229B
S315080117C0009242F21402294620462FF033F895E793
S315080117D0184B1B88ADF8203000230493124A039254
S315080117E008AA0292062201920222009242F21502E8
S315080117F0294620462FF01EF880E70F4B1B88ADF8C7
S31508011800203000230493084A039208AA029206226A
S3150801181001920222009242F21602294620462FF030
S3150801182009F86BE764210020111901084402002018
S31508011830B42100208221002084210020F8B52B4DF7
S31508011840284650F0ADFF2A4B1E782A4B1F782A4BA3
S315080118501C68284650F0F4FF012C24D01DDD023CFB
S31508011860012C1CD8F6B10024244B1C60244B197892
S315080118702448FFF717FF24484DF0F9F91B4D284670
S3150801188050F08EFF1A4B1C701A4B1C701A4B012212
S315080118901A60284650F0D4FF04E0002CE2D0164B1B
S315080118A000221A60F8BD18484DF006FA17497FF06C
S315080118B037FE08B9002FF5D0124C0222104B1978C1
S315080118C020462EF0C8FE2046FFF7C5FE074C2046E7
S315080118D050F066FF0023064A1370064A1370064B3A
S315080118E003221A60204650F0ABFFDBE7882100206F
S315080118F0AC21002086210020B0210020642100208F
S3150801190080210020440200206821002000C05A4599
S3150801191030B583B004460D4601AA2EF09FFF012873
S3150801192013D00222294620462EF095FE2046FFF7BF
S3150801193092FE154C204650F033FF144B03221A60D1
S31508011940204650F07DFF03B030BD022229462046CD
S315080119502EF081FE0E4B1B68072B07D001330C4A6C
S31508011960136029462046FFF79DFEECE72046FFF760
S3150801197072FE054C204650F013FF044B02221A60F2
S31508011980204650F05DFFDEE788210020B0210020C7
S3150801199064210020012800D0704738B54FF6FF733F
S315080119A0994200D038BD0A4C204650F0EBFE094D4D
S315080119B02A460949204650F037F9084C20464DF089
S315080119C08DF92A460649204650F02EF9EAE700BF66
S315080119D08821002088010020832806086821002024
S315080119E0E519010810B504464DF0BAF8204610BDB0
S315080119F0C0E90023009B8360019BC360029B0361CE
S31508011A00039B4361049B8361059BC3619DF8183061
S31508011A1080F820309DF81C3080F821309DF8203060
S31508011A2080F822309DF8243080F823309DF828303C
S31508011A3080F824309DF82C3080F825309DF8303018
S31508011A4080F826309DF8343080F827309DF83830F4
S31508011A5080F828309DF83C3080F829309DF84030D0
S31508011A6080F82A309DF8443080F82B309DF84830AC
S31508011A7080F82C30139B0363149B43637047000063
S31508011A8030B41C4A0260002280F8302080F83120E8
S31508011A9042638263C26380F840204264826480F8AC
S31508011AA04C2080F84D2080F84E2080F84F2080F891
S31508011AB0502080F8512080F8522000214165816527
S31508011AC080F85C2080F85D203F2101713721417142
S31508011AD0094981600273182181830221C18380F833
S31508011AE0202080F8212000240025C0E90A4530BCC1
S31508011AF0704700BF682C0908CDCCC4410430704733
S31508011B0008B502484DF037F808BD00BF6821002026
S31508011B10F0B587B0044690F82130002B79D00D46F0
S31508011B2009686A68836AC06A5B1842EB0002A362A5
S31508011B30E262E86801467FF02FFA7FF037FD84F804
S31508011B403000286901467FF027FA7FF02FFD84F8D7
S31508011B50310095F82330002B62D0012395F8242013
S31508011B60002A5FD00222134395F82520002A5BD06C
S31508011B700422134395F82620002A57D00822134336
S31508011B8095F82720002A53D01022134395F82820C8
S31508011B90002A4FD02022134395F82920002A4BD03A
S31508011BA04022134395F82A20002A47D0802213435E
S31508011BB06363A86803689B6898478C497FF0F4FAC1
S31508011BC07FF0CEFCA063894968697FF0EDFA7FF062
S31508011BD0EDFCE063A8697FF0C3FC84F84000834903
S31508011BE0E8697FF0E1FA7FF0E1FC60647F49A0686B
S31508011BF07FF0DAFA7FF0DAFCA06495F82170FFB17C
S31508011C000126FFB17A49E8687FF06CFC10BB002316
S31508011C1019E080F85D3000220023C0E90A2394E028
S31508011C2000239BE700229EE70022A2E70022A6E7FF
S31508011C300022AAE70022AEE70022B2E70022B6E7B1
S31508011C400026DEE70023334337B9626B002A44D006
S31508011C50002602E00223F6E700263343626B002AD8
S31508011C603DD00826334395F82020002A39D010267E
S31508011C70334395F82220002A35D02022134384F8CD
S31508011C804C30286B10F4000F01D040F07F407FF0F4
S31508011C9037FA56497FF03CFB6065686B7FF02CFA92
S31508011CA052497FF035FBA065524EE06821696269A9
S31508011CB0A3690FC6A28B504B1A80E28B4F4B1A8031
S31508011CC062794F4B1A7094F85D30042B00F28A80C2
S31508011CD0DFE803F00B123D6481000426BDE7002608
S31508011CE0C0E70026C4E70022C8E795F82B3043B3BE
S31508011CF0012384F85D3024E00023ADF80430802107
S31508011D008DF804108DF8052002268DF814608DF8DB
S31508011D1016308DF815300293BDF80430ADF80C3045
S31508011D2002A994F820002AF095FF84F85D60354EE3
S31508011D30304650F035FD344B01221A70304650F0CA
S31508011D407FFD95F82B3084F85C3007B0F0BD2D4F38
S31508011D50384650F025FD2D4B1E68384650F070FD6B
S31508011D60022E0CD0032E03D095F82B30002BE8D188
S31508011D7095F82B303BB1002384F85D30E1E7032366
S31508011D8084F85D30EEE71F4E304650F009FD204BD2
S31508011D9001221A70304650F053FDECE70023ADF8E6
S31508011DA0043001218DF804108DF8052002228DF8E2
S31508011DB014208DF816308DF815300293BDF80430CD
S31508011DC0ADF80C3002A994F820002AF043FF042349
S31508011DD084F85D30B5E795F82B30002BB1D184F83E
S31508011DE05D30AEE7002384F85D30AAE700007A4447
S31508011DF000002041B42100208221002084210020F6
S31508011E008021002088210020AC210020B02100205B
S31508011E108621002008B5FFF711FD08BD90F85C0082
S31508011E20704790F83000704790F831007047406B62
S31508011E307047806B7047C06B704790F940007047D8
S31508011E40406C7047806C704790F84C007047406D45
S31508011E507047806D704708B54FF6FF710120FFF78F
S31508011E6099FD08BD10B50446074B40F8783B50F07C
S31508011E7008FD04F138004CF073FE04F120004CF023
S31508011E806FFE204610BD00BF782C090810B5044620
S31508011E90FFF7E8FFA021204650F000FA204610BDC2
S31508011EA0016042608360009BC360019B0361029BE2
S31508011EB04361039B8361049BC361059B0362069B84
S31508011EC04362079B8362BDF820308385BDF82430C1
S31508011ED0C3859DF8283080F830309DF82C3080F87D
S31508011EE031309DF8303080F832309DF8343080F842
S31508011EF033309DF8383080F834309DF83C3080F81E
S31508011F0035309DF8403080F836309DF8443080F8F9
S31508011F1037309DF8483080F838307047F8B50446B0
S31508011F2006462C4B46F8203B30464CF0D7FE04F1CA
S31508011F30380738464CF0D2FE0025A4F85050A4F8CC
S31508011F405250A4F85450A4F8565084F8585084F8BE
S31508011F50595084F85A5084F85B50A4F85C50A4F898
S31508011F605E5084F8605084F86150A4F8625084F891
S31508011F706450A4F86650A4F86850A4F86A50A4F806
S31508011F806C50A4F86E5084F87050A4F8725084F816
S31508011F90745084F8755084F8765004F1780050F03E
S31508011FA0F1FB257141F28833A3604FF47A73E3603C
S31508011FB0F6232382A574E574042323756575A5752F
S31508011FC0E575257630464CF0D6FD38464CF0D3FDFE
S31508011FD02046F8BD782C090804307047F8B5067E06
S31508011FE02EB104460D464B7B012B02D00026304606
S31508011FF0F8BD0A68284B9A4201D00026F7E70A7904
S315080120004B7943EA0223A0F852308A79CB7943EA1D
S315080120100223A0F8543000F17807384650F0C0FB87
S31508012020B4F8563023F01F039BB2A4F85630A27CAD
S3150801203012B1E27C012A13D02A7A02F01F02134355
S31508012040A4F85630B4F8563043F02003A4F85630B5
S31508012050384650F0F5FB04F120004CF008FEC6E7BF
S315080120602A7A02F0010213431BB2A4F856302A7ADF
S3150801207002F002021343A4F856302A7A02F0040247
S315080120801343A4F856302A7A521002F01002134369
S31508012090A4F85630D6E700BFE550FF182DE9F04FF2
S315080120A09FB00446037ED3B100F1200528464CF0C3
S315080120B0D4FDA3684FF47A7202FB03F3984216D84B
S315080120C004F1380528464CF0C8FDE3684FF47A72E6
S315080120D002FB03F3984221D81FB0BDE8F08F2030E8
S315080120E04CF0C5FD04F138004CF0C1FDF4E70023BE
S315080120F0A4F85230A4F8543004F17806304650F06A
S315080121004FFBB4F8563023F02003A4F85630304676
S3150801211050F096FB28464CF0AAFDD1E70023009320
S31508012120019304F17806304650F03AFBE37D13B18A
S3150801213094F8582062B1228A110A8DF800108DF898
S315080121400120B4F85020110A8DF802108DF80320E9
S3150801215094F85820002A32D000228DF80420A27C57
S31508012160002A37D0E37C63BB237D8DF8053094F8CC
S3150801217059308DF80630637D8DF80730304650F0BA
S315080121805FFB08238DF8143000238DF816300123E0
S315080121908DF81530CA4B029303AB6A4692E80300E1
S315080121A083E8030002A920792AF054FDA37CF3B938
S315080121B0A37D002B59D128464CF059FD8CE7012205
S315080121C0CBE794F85A308DF8053094F85B308DF8E2
S315080121D00630D3E7002BD1D0B4F85C301A0A8DF853
S315080121E005208DF8063032238DF80730C6E73046CC
S315080121F050F0D6FAB4F85C301A0A8DF800208DF83A
S315080122000130B4F85E301A0A8DF802208DF80330D1
S3150801221094F860308DF8043094F861308DF8053003
S31508012220B4F862301A0A8DF806208DF80730304660
S3150801223050F006FB08238DF8243000238DF826304C
S3150801224001238DF825309F4B069307AB6A4692E822
S31508012250030083E8030002AF06AB0FCB87E80F0044
S31508012260394620792AF0F6FCA2E7304650F098FA6A
S31508012270238A1A0A8DF800208DF80130B4F85030F7
S315080122801A0A8DF802208DF8033094F85830002B7D
S3150801229046D000238DF8043094F864308DF8053063
S315080122A04FF000088DF8068001278DF80770304633
S315080122B050F0C6FA08238DF834308DF836808DF83B
S315080122C03570814B0A930BAB6A4692E8030083E8A3
S315080122D0030002AF0AAB0FCB87E80F003946207916
S315080122E02AF0B8FC304650F05BFAB4F866301A0AA0
S315080122F08DF800208DF80130B4F868301A0A8DF887
S3150801230002208DF80330B4F86A301A0A8DF80420D1
S315080123108DF80530B4F86C30FF2B03D8DBB202E038
S315080123200123B7E700238DF8063002238DF807301D
S31508012330304650F085FA4FF0080B8DF844B04FF04F
S3150801234000088DF846804FF0010A8DF845A05E4BCE
S315080123500E930FABE94699E8030083E803000DEBFA
S315080123600B070EAB0FCB87E80F00394620792AF009
S3150801237071FC304650F014FAB4F85C3023FA0BF2CB
S315080123808DF800208DF80130B4F85E3023FA0BF28F
S315080123908DF802208DF80330B4F86E3023FA0BF26B
S315080123A08DF804208DF8053094F870308DF80630D4
S315080123B003238DF80730304650F042FA8DF854B0B1
S315080123C08DF856808DF855A03F4B129313AB99E8BB
S315080123D0030083E8030012AB0FCB87E80F003946E9
S315080123E020792AF037FC304650F0DAF9B4F8623031
S315080123F023FA0BF28DF800208DF80130B4F972300A
S31508012400C3F307228DF802208DF8033094F874304F
S315080124108DF8043094F875308DF8053094F87630D7
S315080124208DF8063004238DF80730304650F008FA47
S315080124308DF864B08DF866808DF865A0224B1693E9
S3150801244017AB99E8030083E8030016AB0FCB87E8BF
S315080124500F00394620792AF0FDFB304650F0A0F9E5
S31508012460B4F86C3023FA0BF28DF800208DF80130A0
S315080124708DF802808DF803808DF804808DF805802B
S315080124808DF8068005238DF80730304650F0D8F9C7
S315080124908DF874B08DF876808DF875A00A4B1A936D
S315080124A01BAB99E8030083E803001EAB13E90F0091
S315080124B087E80F00394620792AF0CCFB7BE600BF76
S315080124C0F4E50618F4FF0018F4E60618037E03B9C6
S315080124D0704770B504460D4600F17806304650F04F
S315080124E05FF9EB8DA4F85030B4F8563013F0200399
S315080124F009D095F8312032B195F832201AB901225E
S3150801250084F8582002E0002284F8582095F83420EF
S31508012510002A00F0B980012284F85920002284F8A3
S315080125205A2095F8342012B1012284F85A2095F8D8
S3150801253036202AB194F85A2042F0020284F85A2029
S3150801254095F838202AB194F85A2042F0040284F802
S315080125505A2095F835202AB194F85A2042F00802F3
S3150801256084F85A202BB994F85A3043F0200384F89A
S315080125705A3094F85A301BB143F0400384F85A3064
S315080125805A2384F85B30524968687EF00DFE7FF065
S315080125900DF8A4F85C004E49A8687EF005FE7FF0A8
S315080125A005F8A4F85E004B49A8697EF0FDFD7EF0AA
S315080125B0FDFF84F860004849E8687EF0EDFC7EF08E
S315080125C0F5FF84F86100454968697EF0EDFD7EF006
S315080125D0EDFFA4F8620095F8303084F864303F497D
S315080125E0E8697EF0E1FD7EF0E1FFA4F866003B496B
S315080125F0286A7EF0D9FD7EF0D9FFA4F8680034492F
S31508012600A86A7EF0D1FD7EF0D1FFA4F86A00AB8DF1
S31508012610A4F86C302E49686A7EF0C6FD7EF0C6FFC6
S31508012620A4F86E0095F9343095F8332043EA42034D
S3150801263084F870302868002846D003689B68984754
S3150801264026497EF0B1FD7EF08BFFA4F872004FF0AB
S315080126507C51A8697EF0A0FC7EF0A8FF84F874007E
S315080126601F49E8687EF098FC7EF0A0FF84F87500A3
S315080126701B4928697EF090FC7EF098FF84F8760065
S31508012680304650F0DDF870BD95F836201AB10322B0
S3150801269084F8592042E795F837201AB1042284F8BC
S315080126A059203BE795F838201AB1052284F85920B4
S315080126B034E795F832201AB1072284F859202DE714
S315080126C0002284F8592029E70023A4F87230BEE7CE
S315080126D000007A440000204000002042000020410A
S315080126E00000C842B0F852007047B0F8540070476D
S315080126F038B5044600F17805284650F051F8B4F883
S315080127005640284650F09CF8204638BD10B5044678
S315080127100B4B0360D0F8C0005CF060FFA06F5CF063
S315080127205DFF04F1480050F0ACF804F130004CF0BC
S3150801273017FA04F118004CF013FA204610BD00BF31
S31508012740D42C090810B50446FFF7E0FF4FF48C7145
S3150801275020464FF0A3FD204610BD01600271704767
S3150801276010B586B00446384B40F8183B4CF0B6FA1B
S3150801277004F130004CF0B2FA04F1480050F002F8C6
S315080127800023E366002384F8703084F871302F4AF9
S31508012790626700930193029303930493059304F1EB
S315080127A07C0304931023059304F18C0302933423C9
S315080127B003936A46042101205CF056FEA0670028AF
S315080127C035D0002300930193029303930493059351
S315080127D004F1C40304931023059304F1D40302936B
S315080127E0342303936A46042101205CF03DFEC4F8B4
S315080127F0C00010B30023C4F80831C4F80C31C4F87A
S31508012800103123712C226271114AA2604FF4FA62C7
S31508012810E26022612375637504F118004CF0ABF987
S3150801282004F130004CF0A7F9204606B010BD51223C
S31508012830084909484EF0D6FAC3E751220549064820
S315080128404EF0D0FAD6E700BFD42C09080000824220
S31508012850CDCCC441802C0908C82C0908043070471E
S3150801286010B58AB00446437D73B190F87130072BD1
S3150801287000F25B81DFE813F00F005C007800B3001B
S31508012880D000070117012F0180F8703018304CF07D
S31508012890EEF90AB010BD0023C3660B79002BF8D0F8
S315080128A0037D1BB9052380F87130F2E700220192F6
S315080128B0134601A9806F5CF039FE10F1020F23D08F
S315080128C030B110F1030F1CD06FF00303049303E03A
S315080128D010230493019B0593A36F0693002201928B
S315080128E0134601A9D4F8C0005CF020FE10F1020FCE
S315080128F01BD060B110F1030F14D06FF003030793D7
S3150801290009E000230493E7E740230493E4E710234F
S315080129100793019B0893D4F8C0300993012384F8DF
S315080129207130B6E700230793F5E740230793F2E7EB
S315080129300B7913B980F87130ABE70023C366806F52
S315080129405CF034FE0028A4D00123C4F8083104F54C
S315080129508473019300231A4601A9A06F5CF0A0FDB8
S31508012960022384F8713094E70B7913B980F8713032
S315080129708FE70023C3660022009213466946D0F802
S31508012980C0005CF0D3FD10F1020F25D030B110F173
S31508012990030F1ED06FF00303019303E01023019385
S315080129A0009B0293D4F8C0300393019B102B7FF44C
S315080129B070AF029B1B68002B7FF46BAFA168606F39
S315080129C07EF0A4FD00283FF464AF032384F8713038
S315080129D05FE700230193E5E740230193E2E70B79DB
S315080129E013B980F8713054E70023C366806F5CF031
S315080129F0DDFD00283FF44DAF0223C4F8083104F584
S31508012A008473019300231A4601A9A06F5CF048FD5F
S31508012A10042384F871303CE70B791BB9062380F847
S31508012A20713036E70023C3660022009213466946D1
S31508012A30D0F8C0005CF07AFD10F1020F1CD030B15D
S31508012A4010F1030F15D06FF00303019303E0102370
S31508012A500193009B0293D4F8C0300393019B102B7A
S31508012A607FF417AF029B1B684BB9052384F87130B5
S31508012A700FE700230193EEE740230193EBE70623D3
S31508012A8084F8713005E70B68C3660B79002B7FF470
S31508012A9000AF037D1BB1062380F87130F9E60023E8
S31508012AA080F87130F5E60023C366806F5CF07EFD21
S31508012AB000283FF4EEAE0323C4F8083104F5847305
S31508012AC0019300231A4601A9A06F5CF0E9FC0723CC
S31508012AD084F87130DDE60023C366002200921346AE
S31508012AE06946D0F8C0005CF021FD10F1020F19D03B
S31508012AF030B110F1030F12D06FF00303019303E015
S31508012B0010230193009B0293D4F8C0300393019BD1
S31508012B10102B7FF4BEAE002384F87130B9E600238A
S31508012B200193F1E740230193EEE7002380F8713022
S31508012B30AFE6C06E704790F870007047F0B583B085
S31508012B40457D002D6DD00446437903F5C07003F524
S31508012B50207C03F5B0634A7B002A61D10A68824268
S31508012B6005D0624503D09A420ED0002559E004F1FA
S31508012B7048004FF015FE012384F8703004F118005F
S31508012B804CF075F800254CE0D4F81031012B04D02F
S31508012B90023B012B2ED9002543E04868224A904280
S31508012BA0F6D10E7A4B7A46EA03268B7A46EA03462B
S31508012BB0CB7A46EA036604F1480738464FF0F0FD3A
S31508012BC030467EF099FA19497EF0A2FB60673846CD
S31508012BD04FF036FE0026C4F80C6104F5867301939E
S31508012BE03346324601A9D4F8C0005CF059FCC4F852
S31508012BF0106116E04A680E4B9A4201D0002510E092
S31508012C000026C4F80C6104F58673019333463246EF
S31508012C1001A9D4F8C0005CF043FCC4F8106100E0D7
S31508012C200025284603B0F0BD4320200100007A4460
S31508012C3060142001437D03B9704770B58AB0044614
S31508012C4000220392134603A9806F5CF06FFC10F112
S31508012C50020F25D030B110F1030F1ED06FF0030318
S31508012C60079303E010230793039B0893A36F099324
S31508012C70079B102B17D0D4F81031002B5BD104F128
S31508012C80180528464BF0E9FFE3684FF47A7202FB10
S31508012C9003F398427DD80AB070BD00230793E5E790
S31508012CA040230793E2E7089B1B68C4F8103100220A
S31508012CB001920292012B16D093421FDD9A1E012A18
S31508012CC01CD82F228DF8042014228DF805202022E5
S31508012CD08DF8062001228DF80720022B29D0002322
S31508012CE08DF808300AE040238DF8043020238DF84A
S31508012CF005308DF8063001238DF80730637903F521
S31508012D00C06308228DF8182000228DF81A208DF844
S31508012D101920039304AB01AA92E8030083E8030090
S31508012D2003A9207929F096FF04F130004BF09FFFA3
S31508012D30A1E71346D4E704F130004BF08EFF23696F
S31508012D404FF47A7202FB03F3984298D9D4F81031FA
S31508012D50012B10D00223C4F80C3104F586730393B2
S31508012D6000231A4603A9D4F8C0005CF099FB002396
S31508012D70C4F8103183E704F1480528464FF010FDE1
S31508012D80134B636728464FF05BFD0023C4F80C31EB
S31508012D90E3E7002684F8706028464BF068FFADF833
S31508012DA0046001238DF8043063798DF80530022318
S31508012DB08DF818308DF81A608DF819600396BDF8EC
S31508012DC00430ADF8103003A9207929F043FF62E7F2
S31508012DD00000824210B50446074B40F8783B4FF095
S31508012DE050FD04F140004BF0BBFE04F128004BF006
S31508012DF0B7FE204610BD00BFE42C090810B50446ED
S31508012E00FFF7E8FFA02120464FF048FA204610BDFB
S31508012E10016042608360009BC360019B0361029B62
S31508012E204361039B8361049BC3619DF8143080F859
S31508012E3020309DF8183080F821309DF81C3080F834
S31508012E4022309DF8203080F823309DF8243080F810
S31508012E5024309DF8283080F825309DF82C3080F8EC
S31508012E6026309DF8303080F827309DF8343080F8C8
S31508012E7028309DF8383080F829307047F8B504466F
S31508012E80244B036000254560058100F12807384673
S31508012E904BF024FF04F1400630464BF01FFF84F83F
S31508012EA0585084F8595084F85A5084F85B5084F87D
S31508012EB05C5084F85D5084F85E50A4F86050A4F81C
S31508012EC06250A4F86450A4F86650A4F86850A4F8AF
S31508012ED06A50A4F86E50A4F87050A4F8725084F899
S31508012EE0745004F178004FF04DFC25730A4B2361A9
S31508012EF04FF07E536361094AA261E36184F8205069
S31508012F0084F8215038464BF036FE30464BF033FEF6
S31508012F102046F8BDE42C0908CDCCC44166669E411D
S31508012F2010B40A4C0C4444601909090201EB023138
S31508012F3089B21B0103F0F0030B449BB29DF80420F0
S31508012F4002F00F021344038110BC7047E0BADD7723
S31508012F5070B590F82150D5B104464B7BB3B90A68D0
S31508012F6040F205339A4201D0002510E000F17806B7
S31508012F7030464FF015FC012384F8583004F1280037
S31508012F804BF075FE30464FF05BFC00E00025284605
S31508012F9070BD000090F8213003B970472DE9F0475C
S31508012FA09EB0044600F1280528464BF056FED24B42
S31508012FB098420ADC04F1400948464BF04EFECF4BD5
S31508012FC0984211DC1EB0BDE8F08704F17806304658
S31508012FD04FF0E6FB002384F8583030464FF030FCBA
S31508012FE028464BF044FEE5E700230093019304F1DC
S31508012FF0780840464FF0D4FB94F859308DF80030E4
S3150801300094F85A308DF8013094F85B308DF8023017
S3150801301094F85C308DF8033094F820303BB994F875
S315080130205D308DF8043094F85E308DF807304046EF
S315080130304FF006FC4FF0080A8DF814A000268DF80B
S3150801304016608DF8156040F25933029303AB6F464B
S3150801305097E8030083E803000DEB0A052946207B60
S3150801306029F0F8FD40464FF09BFBB4F860308DF827
S31508013070003023FA0AF38DF80130B4F862308DF87E
S31508013080023023FA0AF38DF80330B4F864308DF868
S31508013090043023FA0AF38DF80530B4F866308DF852
S315080130A0063023FA0AF38DF8073040464FF0C8FB7D
S315080130B08DF824A08DF826608DF8256040F25133ED
S315080130C0069307AB97E8030083E8030006AB0FCB2B
S315080130D085E80F002946207B29F0BCFD40464FF0C4
S315080130E05FFBB4F868308DF8003023FA0AF38DF8DF
S315080130F00130B4F86A308DF8023023FA0AF38DF8F4
S3150801310003308DF804608DF805608DF806608DF83A
S31508013110076040464FF094FB8DF834A08DF8366071
S315080131208DF8356040F255330A930BAB97E80300E7
S3150801313083E803000AAB0FCB85E80F002946207BFD
S3150801314029F088FD40464FF02BFBB4F86E308DF818
S31508013150003023FA0AF38DF80130B4F970308DF88E
S315080131600230C3F307238DF80330B4F972308DF8B2
S315080131700430C3F307238DF8053040464FF060FB52
S315080131808DF844A08DF846608DF8456040F25633B7
S315080131900E930FAB97E8030083E803000EAB0FCB42
S315080131A085E80F002946207B29F054FD40464FF05B
S315080131B0F7FA94F874308DF800308DF801608DF8BF
S315080131C002608DF803608DF804608DF8056040464D
S315080131D04FF036FB8DF854A08DF856608DF8556082
S315080131E04FF45773129313AB97E8030083E8030070
S315080131F012AB0FCB85E80F002946207B29F02AFD63
S3150801320094F8203083BB4D238DF800304F238DF879
S31508013210013056238DF8023045238DF803304C23AF
S315080132208DF8043008238DF8643000238DF8663054
S315080132308DF8653040F25E33169317AB6A4692E80D
S31508013240030083E8030002AD16AB0FCB85E80F0038
S315080132502946207B29F0FEFC94F82030012B1AD050
S3150801326048464BF004FDADE64D238DF800304F235B
S315080132708DF8013056238DF8023045238DF8033039
S315080132804C238DF80430B4F86C308DF806301B0ADF
S315080132908DF80730C6E763688DF800301A0A8DF88D
S315080132A001201A0C8DF802201B0E8DF80330238994
S315080132B08DF804301B0A8DF8053000238DF8063089
S315080132C08DF8073008228DF874208DF876308DF840
S315080132D0753040F21C731A931BAB6A4692E80300D9
S315080132E083E803001EAB13E90F0085E80F002946A2
S315080132F0207B29F0AFFCB3E700093D0040420F00EF
S315080133000C30704738B5044600F1780528464FF069
S3150801331047FA94F8584028464FF092FA204638BDA5
S315080133202AB101229A400B7813430B707047012288
S315080133309A400B7823EA02030B7070472DE9F04196
S3150801334004460D4690F82130002B00F0BD8004F1AB
S31508013350780738464FF024FA04F15906012395F8FF
S31508013360252031462046FFF7DBFF022395F8242066
S3150801337031462046FFF7D4FF032395F82620314628
S315080133802046FFF7CDFF042395F82720314620462E
S31508013390FFF7C6FF072395F8232031462046FFF796
S315080133A0BFFF04F15A06002395F82320314620462B
S315080133B0FFF7B6FF032395F8282031462046FFF785
S315080133C0AFFF042395F8292031462046FFF7A8FFC9
S315080133D0002384F85B3084F85C30EB6984F85D304F
S315080133E095F8203084F85E304B4920697DF0DCFE83
S315080133F07EF0DCF8A4F86000474960697DF0D4FEE8
S315080134007EF0D4F8A4F862004349E0697DF0CCFE69
S315080134107EF0CCF8A4F864003F49A0697DF0C4FEAB
S315080134207EF0C4F8A4F866004FF07C5128697DF057
S31508013430B3FD7EF0BBF8A4F868004FF07C516869CB
S315080134407DF0AAFD7EF0B2F8A4F86A004FF07C512F
S31508013450A8697DF0A1FD7EF0A9F8A4F86C002F49B2
S3150801346028687DF0A1FE7EF0A1F8A4F86E002A492D
S3150801347068687DF099FE7EF073F8A4F87000E96833
S31508013480A8687DF089FD4FF07C517DF08DFE2249BB
S315080134907DF08AFE7EF064F8A4F8720004F17406E1
S315080134A0072395F8212031462046FFF739FF95F87D
S315080134B02180B8F1000F1BD0174928697EF01CF846
S315080134C0C0B94FF0000815E000F1780630464FF014
S315080134D067F9002384F8583004F128004BF0C7FB3C
S315080134E004F140004BF0C3FB30464FF0A9F92EE733
S315080134F04FF000080523424631462046FFF710FFE4
S31508013500062395F8222031462046FFF709FF38465B
S315080135104FF096F9BDE8F081000020410000C8424D
S3150801352010B50446034B40F8283B4FF0AAF920464C
S3150801353010BD00BFF42C090810B50446FFF7F0FFCB
S31508013540602120464EF0AAFE204610BDC0E90023A0
S31508013550009B83609DF8043003739DF8083043731C
S315080135609DF80C3083739DF81030C37370470000C3
S3150801357010B504460F4B40F8283B4FF003F90023DA
S31508013580E3642365002384F85430A4F85630A4F87C
S31508013590583084F85B302371074AA2604FF4C86239
S315080135A0E260237400220023C4E90623C4E9082340
S315080135B0204610BDF42C090833336742043070479E
S315080135C02DE9F8430446037C5BB10D46CB7BD3B9A1
S315080135D08B7B002B3BD14B7B002B3BD04FF001095A
S315080135E013E000F1280528464FF0DAF8002384F89D
S315080135F05B3000220023C4E90623C4E908232846D0
S315080136004FF01EF95BE04FF0020904F12806304637
S315080136104FF0C6F8E76C30464FF012F96B7BFBB1F9
S31508013620002138467DF054FF00284AD1D5F8088094
S31508013630394640467DF06AFF78B9234940467DF010
S31508013640B3FD39467DF064FE8046A7680AE04FF06F
S315080136500309DAE74FF00209D7E7DFF86C80F4E7E8
S315080136600027B84630464FF09BF828686A68A36970
S31508013670E1691B1842EB0102A361E26128686A68E5
S31508013680236A616A1B1842EB01022362626284F8AB
S3150801369054900E4940467DF087FD7DF087FFA4F8DA
S315080136A056000A4938467DF07FFD7DF07FFFA4F874
S315080136B058002B7B84F85A3030464FF0C1F8BDE8E4
S315080136C0F8830027B846CDE70000C842000020412C
S315080136D090F85B0070470000F8B5067C002E34D0E0
S315080136E005460C464B7B7BBB0A6840F2CB339A42B4
S315080136F001D0002629E00B7B052B01D8002624E002
S3150801370000F1280738464FF04BF8207A637A43EAE6
S3150801371000207DF0F5FC0E497DF046FDE864A079B0
S31508013720E37943EA00207DF0EBFC09497DF03CFD95
S315080137302865012385F85B3000220023C5E90623A5
S3150801374038464FF07DF800E000263046F8BD00BF48
S31508013750CDCCCC3D037C03B970472DE9F04387B046
S31508013760044600F1280528464FF01AF8A169E269CE
S31508013770E668F00E73019B1B60F10000800040EAC9
S3150801378093709B009B1940F10000C00040EA5370FA
S31508013790DB00994272EB000306D3002384F85B3001
S315080137A000220023C4E90623226A636A204991425A
S315080137B04FF0000272EB030336D200220023C4E95C
S315080137C0082394F85490B4F85670B4F8586094F8ED
S315080137D05A8028464FF034F80023009301938DF858
S315080137E000903A0A8DF801208DF80270320A8DF898
S315080137F003208DF804608DF8058008228DF81420C1
S315080138008DF816308DF8153040F2FF23029303AB7D
S315080138106A4692E8030083E8030002A9207929F0A1
S3150801382019FA07B0BDE8F08328464FF009F8F8E71A
S315080138303F0D0300C06C7047006D704710B5044614
S31508013840034B40F8283B4FF01CF8204610BD00BF3B
S31508013850042D090810B50446FFF7F0FF5821204644
S315080138604EF01CFD204610BDC0E90023009B836075
S315080138709DF804300373704710B50446104B40F8A1
S31508013880283B4EF07FFF0023A4F84C30A4F84E30B5
S3150801389084F8503084F85130237140F2C162E280D5
S315080138A04FF4FA62A2604FF47A72E260237400223E
S315080138B00023C4E90623C4E90823204610BD00BF36
S315080138C0042D090804307047F8B50446037C6BB328
S315080138D00D4600F1280630464EF062FF29686A68EF
S315080138E0A369E0695B1842EB0002A361E2612968FA
S315080138F06A68236A606A5B1842EB000223626262A5
S315080139002B7B2BB3B4F84E7017B31549A8687DF015
S315080139104BFC054638467DF0EFFB014628467DF00F
S31508013920F7FC7DF043FE84F8500014E000F1280509
S3150801393028464EF035FF002384F851300022002333
S31508013940C4E90623C4E9082328464EF079FF05E0B1
S31508013950002384F8503030464EF072FFF8BD00BFA0
S315080139600000C84290F851007047F8B5067C3EB38E
S3150801397004460D464B7B13BB0A6840F284539A42B0
S3150801398001D000261CE000F1280738464EF008FF52
S315080139902A7A6B7A43EA0223A4F84C30AA7AEB7A9C
S315080139A043EA0223A4F84E30012384F85130002259
S315080139B00023C4E9062338464EF042FF00E00026FC
S315080139C03046F8BD037C03B970472DE9F0418AB04A
S315080139D0044600F1280528464EF0E2FEA169E2698F
S315080139E0A668F00E73019B1B60F10000800040EA97
S315080139F093709B009B1940F10000C00040EA537088
S31508013A00DB00994272EB000306D3002384F8513098
S31508013A1000220023C4E90623216A626AE668F00ED9
S31508013A2073019B1B60F10000800040EA93709B00C4
S31508013A309B1940F10000C00040EA5370DB0099422F
S31508013A4072EB000336D300220023C4E9082394F855
S31508013A50508028464EF0F4FE00250095019508276A
S31508013A608DF814708DF816508DF8155040F20463D0
S31508013A70029303AB6E4696E8030083E803000DEB59
S31508013A800701207929F0E6F8E3888DF806808DF894
S31508013A9024708DF826508DF82550069307AB96E8C5
S31508013AA0030083E8030006A9207929F0D3F80AB0B0
S31508013AB0BDE8F08128464EF0C3FEF8E7B0F84C00A1
S31508013AC07047B0F84E00704710B50446074B40F8EA
S31508013AD0803B4EF0D6FE04F138004BF041F804F174
S31508013AE020004BF03DF8204610BD00BF142D0908F3
S31508013AF010B50446FFF7E8FFA82120464EF0CEFB95
S31508013B00204610BD016042608360009BC360019B33
S31508013B100361029B43619DF80C3003769DF81030D2
S31508013B2043769DF8143083769DF81830C3769DF850
S31508013B301C30037770470000F8B504460646274B44
S31508013B4046F8203B30464BF0C9F804F138073846A9
S31508013B504BF0C4F80025A4F85050A4F85250A4F824
S31508013B605450A4F85650A4F8585084F85A5084F87A
S31508013B705B50A4F85C50A4F85E5000232366636684
S31508013B80A366E3662367636784F8785084F87950F7
S31508013B9084F87A5084F87B5084F87C5084F87D50F8
S31508013BA084F87E5004F180004EF0ECFD257141F257
S31508013BB08833A360C822E260F62323820A2363823C
S31508013BC0A282E38201232376657630464AF0D3FF43
S31508013BD038464AF0D0FF2046F8BD00BF142D090823
S31508013BE010B5447E002C4ED04B7B002B4AD10B6876
S31508013BF040F20532934209D040F20632934221D06F
S31508013C0040F20732934239D000243CE04A790B79D5
S31508013C1043EA0223A0F85030CA798B7943EA022392
S31508013C20A0F852304A7A0B7A43EA0223A0F85430B4
S31508013C30CA7A8B7A43EA0223A0F8563020304BF031
S31508013C4016F820E04A790B7943EA0223A0F858309E
S31508013C508B7980F85A30CB7980F85B304A7A0B7ABF
S31508013C6043EA0223A0F85C30CA7A8B7A43EA022334
S31508013C70A0F85E3020304AF0FAFF04E020304AF01E
S31508013C80F6FF00E00024204610BD04307047437E4D
S31508013C9003B9704770B504460D4600F180063046F3
S31508013CA04EF07EFD2B6823666B686366AB68A36678
S31508013CB0237EEBB1E86803689B68984700F10040EA
S31508013CC0E0662B6923676B6963672B7E84F8783016
S31508013CD06B7E84F87930AB7E84F87A30EB7E84F893
S31508013CE07B302B7F84F87C3030464EF0A9FD70BDC1
S31508013CF0E86803689B689847E2E7B0F850007047A0
S31508013D00B0F952007047B0F954007047B0F8560040
S31508013D107047B0F85800704790F85A00704790F805
S31508013D205B007047B0F85C007047B0F85E007047FA
S31508013D30087840FA03FC1CF0030C06D0BCF1020F0C
S31508013D4003D0BCF1010F0ED07047002AF9D0032227
S31508013D509A4020EA020040B20870012202FA03F3EF
S31508013D60184308707047002AEED103229A4020EAC8
S31508013D70020C4FFA8CF20A70022000FA03F31A4376
S31508013D800A70E1E72DE9F04F93B00446437ED3B1BB
S31508013D9000F1200528464AF060FFA3684FF47A72BD
S31508013DA002FB03F3984216D804F1380840464AF054
S31508013DB054FFE3684FF47A7202FB03F3984221D861
S31508013DC013B0BDE8F08F20304AF051FF04F13800F6
S31508013DD04AF04DFFF4E70023A4F85030A4F8523016
S31508013DE0A4F85430A4F85630A4F8583084F85A3058
S31508013DF084F85B30A4F85C30A4F85E3028464AF0B3
S31508013E0036FFD1E7002500950195238A8DF8003004
S31508013E101B0A8DF80130638A8DF802301B0A8DF86A
S31508013E200330E38A8DF804301B0A8DF80530A38A1E
S31508013E308DF806301B0A8DF807304FF008038DF808
S31508013E4014308DF816508DF8155040F251330293FF
S31508013E5003AB6F4697E8030083E8030002AE3146D9
S31508013E60207928F0F7FE04F1800948464EF098FCBF
S31508013E7094F878308DF800308DF80150606E7DF039
S31508013E8095FB8DF802008DF803505C49206E7DF094
S31508013E908BF97DF065FB8DF8040000128DF805009D
S31508013EA048464EF0CDFC4FF0060A8DF824A08DF851
S31508013EB026508DF8255040F25533069306AB97E800
S31508013EC003000790ADF820100FCB86E80F003146A6
S31508013ED0207928F0BFFE48464EF062FC4749A06E9D
S31508013EE07DF062F97DF03CFB8DF8000000128DF83B
S31508013EF001004349E06E7DF057F97DF031FB8DF8FD
S31508013F00020000128DF803003D49206F7DF04CF93F
S31508013F107DF026FB8DF8040000128DF80500484651
S31508013F204EF08EFC8DF834A08DF836508DF835504C
S31508013F3040F256330A930AAB97E803000B90ADF8A3
S31508013F4030100FCB86E80F003146207928F082FE23
S31508013F5048464EF025FC04F17D0B022394F87B209C
S31508013F6059462046FFF7E4FE042394F87A20594679
S31508013F702046FFF7DDFE534694F87C205946204635
S31508013F80FFF7D6FE534694F8792004F17E012046C0
S31508013F90FFF7CEFE94F87D308DF8003094F87E3028
S31508013FA08DF801308DF802508DF803508DF80450C4
S31508013FB08DF805508DF806508DF8075048464EF095
S31508013FC03FFC4FF008038DF844308DF846508DF8C4
S31508013FD0455040F25A330E930FAB97E8030083E836
S31508013FE0030012AB13E90F0086E80F00314620796A
S31508013FF028F030FE40464AF03AFEE1E60000C842A3
S315080140000000204110B50446034B40F8303B4EF002
S3150801401038FC204610BD00BF242D090810B50446FA
S31508014020FFF7F0FF582120464EF038F9204610BD1B
S31508014030C0E90023009B8360019BC360029B036167
S31508014040039B4361049B8361BDF8143083839DF808
S31508014050183083779DF81C30C377704738B5044606
S31508014060124B03604FF6FF7303844384002580F8DF
S31508014070245080F82550802280F8262080F82720B1
S315080140800385438580F82C5030304EF07BFB2C237A
S315080140902371074BA3604FF07E53E360257400221A
S315080140A00023C4E90623204638BD00BF242D09088C
S315080140B0CDCCC4410430704738B5037C43B10446BE
S315080140C04B7B2BB9037903F500730A689A4201D031
S315080140D0002038BD00F1300528464EF061FB01236A
S315080140E084F82C3000220023C4E9062328464EF022
S315080140F0A7FBEDE72DE9F0410446037C6BB30D46BA
S3150801410000F1300630464EF04BFB2B686A68A16910
S31508014110E0695B1842EB0002A361E26194F82C1096
S3150801412061B1374999424FF00003934106D2002302
S3150801413084F82C3000220023C4E9062394F82C8045
S3150801414030464EF07DFBEB7FBBB92E49E8687DF022
S315080141502BF87DF02BFA80B211E000F130052846E4
S315080141604EF01EFB002384F82C3000220023C4E9FC
S31508014170062328464EF064FB40E04FF6FF70208484
S31508014180E66830467DF012FA60842F693946304672
S315080141907DF0A8F918B138467DF008FA6084AB7F3E
S315080141A093B1B8F1000F0FD0AB8B13F0010F0BD001
S315080141B0012384F824304FF0834128697CF0F4FF09
S315080141C07DF0F4F9608503E00023638584F82430E3
S315080141D0A8687DF0EBF984F8250068697DF0C0F9D7
S315080141E084F82600A8697DF0BBF984F827000549FB
S315080141F0A0687CF0D9FF7DF0D9F92085BDE8F0816A
S31508014200FF083D000000C84290F82C007047008C5A
S315080142107047408C704790F82400704790F8250045
S31508014220704790F92600704790F927007047008D6E
S315080142307047408D70470000014B0360704700BF0F
S31508014240342D090810B50446FFF7F6FF202120464C
S315080142504EF024F8204610BDC0E90023BDF8003011
S3150801426003819DF9043083729DF90830C372704742
S3150801427030B40A4A026000220283FF218176C176A0
S3150801428002774FF47A6141600121017241728272AB
S3150801429000240025C0E9044530BC7047342D0908BF
S315080142A004307047837A002B40D010B40C684A68F2
S315080142B003691B19446942EB0402036142610A89D5
S315080142C0038B9A4205D00123037700220023C0E914
S315080142D004230B890383426944684FEAD46C63015A
S315080142E01B1B6CF1000C4FEA8C0C4CEA937C9B006F
S315080142F01B194CF1000C4FEACC0C4CEA537CDB0041
S3150801430004699C4272EB0C0305D300230377002250
S315080143100023C0E90423037FABB191F90A20827611
S31508014320C3B191F90B30C37610BC704791F90A30C5
S31508014330837691F90B30C376002303770022002395
S31508014340C0E904237047027A12B991F90A20E6E70F
S315080143500122E4E7437A13B991F90B30E3E7012324
S31508014360E1E790F91A00704790F91B007047007F42
S3150801437070470000014B0360704700BF442D0908D0
S3150801438010B50446FFF7F6FF202120464DF086FFBB
S31508014390204610BDC0E900239DF90030037270471D
S315080143A030B4094A0260002202744FF47A714160FE
S315080143B00121816001734273827300240025C0E9DB
S315080143C0064530BC704700BF442D090804307047C4
S315080143D0007C0238C0B201288CBF0020012070473A
S315080143E091F90800003818BF0120704770B50446D6
S315080143F0037BABB1437BABB90B684D688669C26970
S315080144009E1945EB02058661C56191F90830002BB5
S315080144100BDB037C032B67D8DFE803F00A1533416E
S31508014420037470BD02230374FBE700230374F8E7E2
S31508014430FFF7D6FF0028F4D00123237400220023B6
S31508014440C4E90623EDE7FFF7CBFF10B90023237470
S31508014450E7E76168CA0E4B015B1A62F10002920036
S3150801446042EA93729B005B1842F10002D20042EACB
S315080144705372DB009E4275EB0203D2D302232374E7
S31508014480CFE7837B002BCCD1FFF7AAFF0028C8D141
S315080144900323237400220023C4E90623C1E7FFF797
S315080144A09FFF10B102232374BBE7A068C20E430124
S315080144B01B1A62F10002520242EAD3525B021B182E
S315080144C042F100024FEA821C4CEA936C9901CB1A1D
S315080144D06CEB02021B1842F100029E4275EB0203C5
S315080144E09FD3002323749CE70023037499E70000F4
S315080144F0014B0360704700BF542D090810B50446E7
S31508014500FFF7F6FF302120464DF0C8FE204610BDC4
S31508014510C0E90023009B83609DF80430037370474C
S3150801452030B40B4A02600022027680F82820094935
S31508014530416009498160C2600261012101754275C4
S31508014540827500240025C0E9084530BC704700BFC4
S31508014550542D090800005C420000484204307047A7
S31508014560007E0238C0B201288CBF002001207047A6
S3150801457090F82800704710B50C7B3CB10B46416892
S3150801458098687CF0CDFF10B9002400E0002420468D
S3150801459010BD10B50C7B3CB10B46816898687CF060
S315080145A0A1FF10B9002400E00024204610BDF8B58B
S315080145B00446037D93B10D46437D9BB90B684E684E
S315080145C0076A426ADF1946EB020607624662037EFC
S315080145D0032B78D8DFE803F00C19394D037680F8F8
S315080145E02830F8BD02230376012380F82830F8E73E
S315080145F0FFF7C1FF84F828000028F2D001232376AB
S3150801460000220023C4E90823EBE7FFF7B4FF84F887
S31508014610280010B900232376E3E7E168CA0E4B01A7
S315080146205B1A62F10002920042EA93729B005B18E0
S3150801463042F10002D20042EA5372DB009F4276EB56
S315080146400203CED302232376CBE7837D002BC8D181
S31508014650FFF791FF84F8280029462046FFF799FFBE
S315080146600028BED00323237600220023C4E90823A9
S31508014670B7E7FFF780FF84F8280029462046FFF7A9
S3150801468088FF10B902232376ABE72069C20E4301DE
S315080146901B1A62F10002520242EAD3525B021B184C
S315080146A042F10002950145EA93659901CB1A65EB3A
S315080146B002021B1842F100029F4276EB020390D3D5
S315080146C0002323768DE7002303768AE7014B0360EF
S315080146D0704700BF642D090810B50446FFF7F6FFB9
S315080146E0282120464DF0DAFD204610BDC0E90023F9
S315080146F0009B83609DF804300373704730B40A4AFF
S315080147000260002202760021416008498160C26088
S315080147100261012101754275827500240025C0E9EF
S31508014720084530BC704700BF642D09080000A04049
S3150801473004307047007E0238C0B201288CBF0020C1
S315080147400120704710B50C7B3CB10B46416898684F
S315080147507CF0C8FE10B9002400E00024204610BDF4
S3150801476010B50C7B3CB10B46816898687CF0D8FE85
S3150801477010B9002400E00024204610BD70B5044697
S31508014780037D8BB1437D8BB90B684D68066A426A16
S315080147909E1945EB020506624562037E032B64D822
S315080147A0DFE803F00712303E037670BD0223037675
S315080147B0FBE7FFF7C7FF0028F7D00123237600227E
S315080147C00023C4E90823F0E7FFF7BCFF10B900236B
S315080147D02376EAE7E168CA0E4B015B1A62F1000229
S315080147E0920042EA93729B005B1842F10002D200E2
S315080147F042EA5372DB009E4275EB0203D5D30223CC
S315080148002376D2E7837D002BCFD1FFF7A9FF0028B6
S31508014810CBD00323237600220023C4E90823C4E767
S31508014820FFF79EFF10B902232376BEE72069C20E61
S3150801483043011B1A62F10002520242EAD3525B0299
S315080148401B1842F100024FEA821C4CEA936C99014B
S31508014850CB1A6CEB02021B1842F100029E4275EB61
S315080148600203A2D3002323769FE7002303769CE75E
S31508014870014B0360704700BF742D090810B5044643
S31508014880FFF7F6FF382120464DF008FD204610BDFA
S31508014890C0E90023009B83607047000030B40E4ACC
S315080148A00260002280F8202080F83020DFF82CC032
S315080148B0C0F804C00A498160C0F80CC001614261B0
S315080148C00A21816101210177427782770024002537
S315080148D0C0E90A4530BC7047742D0908000020401C
S315080148E0CDCC0C400430704790F820000238C0B295
S315080148F001288CBF00200120704790F830007047CE
S3150801490038B504460D4688680368DB6898476168C8
S315080149107CF006FE58B9A86803681B699847E168E0
S3150801492001F100417CF0DEFD10B1012000E001201B
S3150801493038BD38B504460D4688680368DB6898476C
S31508014940A1687CF0CFFD58B1A86803681B69984730
S31508014950216901F100417CF0E3FD18B1012000E075
S31508014960002038BD0020FCE770B50446037F33B14B
S315080149700D46437F33B1022380F8203001E080F8E9
S31508014980203070BD09686A68836AC06A5B1842EBA1
S315080149900002A362E26229462046FFF7B1FF84F8C6
S315080149A0300094F82030032B69D8DFE803F0020CB5
S315080149B02C3D0028E5D0012384F82030002200236D
S315080149C0C4E90A23DDE718B9002384F82030D8E7BB
S315080149D0A16AE26A6569E80E6B015B1B60F100007A
S315080149E0800040EA93709B005B1940F10000C0000B
S315080149F040EA5370DB00994272EB0003C1D30223EC
S31508014A0084F82030BDE7A37F002BBAD1294620467A
S31508014A10FFF78FFF0028B4D0032384F82030002243
S31508014A200023C4E90A23ACE729462046FFF781FF9C
S31508014A3018B9022384F82030A3E7A06AE16AA669B7
S31508014A40F20E73019B1B62F10002520242EAD35233
S31508014A505B029B1942F100024FEA821C4CEA936CF5
S31508014A609D01EB1A6CEB02029B1942F10002984276
S31508014A7071EB020385D3002384F8203081E70023F4
S31508014A8084F820307DE70000014B0360704700BFC2
S31508014A90842D090810B50446FFF7F6FF3021204694
S31508014AA04DF0FCFB204610BDC0E90023009B836046
S31508014AB0019BC3609DF808300374704730B40B4AF4
S31508014AC002600022027680F82820094941600949D6
S31508014AD08160C26002610275012141758275C275E4
S31508014AE000240025C0E9084530BC7047842D090813
S31508014AF0000088406666864004307047007E0238AA
S31508014B00C0B201288CBF00200120704790F8280008
S31508014B10704710B50B46027D42B1C9681C7C3CB191
S31508014B2040687CF0DFFC20B9002402E08968F5E7DB
S31508014B300024204610BD10B50B46027D42B1C96856
S31508014B401C7C3CB180687CF0E1FC20B9002402E0C1
S31508014B508968F5E70024204610BDF8B50446437D6B
S31508014B6093B10D46837D8BB90B684E68076A426A15
S31508014B70DF1946EB020607624662037E032B76D8E7
S31508014B80DFE803F00A17374B0376F8BD02230376ED
S31508014B90012380F82830F8E7FFF7BBFF84F82800DF
S31508014BA00028F2D00123237600220023C4E9082332
S31508014BB0EBE7FFF7AEFF84F8280010B90023237648
S31508014BC0E3E7E168CA0E4B015B1A62F10002920043
S31508014BD042EA93729B005B1842F10002D20042EA54
S31508014BE05372DB009F4276EB0203CED30223237670
S31508014BF0CBE7C37D002BC8D1FFF78BFF84F82800CC
S31508014C0029462046FFF797FF0028BED003232376BF
S31508014C1000220023C4E90823B7E7FFF77AFF84F8DF
S31508014C20280029462046FFF786FF10B90223237676
S31508014C30ABE72069C20E43011B1A62F10002520258
S31508014C4042EAD3525B021B1842F10002950145EA7A
S31508014C5093659901CB1A65EB02021B1842F1000212
S31508014C609F4276EB020390D3002323768DE7002338
S31508014C7003768AE7014B0360704700BF942D090844
S31508014C8010B50446FFF7F6FF482120464DF006FB0E
S31508014C90204610BDC0E90023009B8360019BC360C9
S31508014CA09DF8083003749DF80C3043749DF8103054
S31508014CB083749DF91430C3749DF9183003759DF9F1
S31508014CC01C304375089B8361099BC3619DF8283095
S31508014CD080F820307047000030B4194A026000227B
S31508014CE080F82C2080F82D2080F82E2080F82F209F
S31508014CF080F8302080F8312000240025C0E90E45CF
S31508014D0080F8402080F8412080F842200D49416012
S31508014D104FF081418160C2600B4901610B494161D4
S31508014D200B4981610B49C1610B4901620B4941621A
S31508014D3080F8282080F8292080F82A2030BC70477E
S31508014D40942D09086666864000004040CDCC4C404B
S31508014D5005042300030002001B04410010000200A1
S31508014D600430704790F82C00704790F82E000128FF
S31508014D7014BF00200120704790F82E3013B990F81F
S31508014D80410070470020704790F84100704790F83D
S31508014D902F00704790F83100012814BF0020012028
S31508014DA07047087C40B9487C30B9887C20B991F9AC
S31508014DB01330002B00DD0120704782698B691A4286
S31508014DC009D1C269CB691A4207D190F8283033B1A3
S31508014DD091F8200070470120704701207047002094
S31508014DE070472DE9F04104460D46FFF7DAFF0646FE
S31508014DF084F82C0029462046FFF7DFFF074684F88A
S31508014E002D0094F82E3033B1012B3DD0002384F8C0
S31508014E102E30BDE8F08194F84080B8F1000F04D136
S31508014E206168E8687CF068FB08BBB8F1000F04D03C
S31508014E30A168E8687CF060FBC8B9E1680029E8D098
S31508014E402B686A68E06BD4F838C0B3EB0C0362EBE5
S31508014E500002C1EB011C4FEA8C0C634572F1000399
S31508014E60D7DB6168E8687CF03DFB0028D1D0002ECD
S31508014E70CFD1002FCDD1012384F8403084F82E30CC
S31508014E80002384F84130C4E76168E8687CF03EFB9A
S31508014E9050B1002384F82E30D5E90023C4E90E2346
S31508014EA0012384F84130B4E70EB9002FB1D00023AD
S31508014EB084F82E30D5E90001C4E90E0184F84130A1
S31508014EC0A7E7087C40B9487C30B9887C20B991F9B4
S31508014ED01430002B00DD0120704710B4024690F80B
S31508014EE0290088B1136A8869034003F40054C3F39F
S31508014EF0403092F82A303BB191F91500002802DDBD
S31508014F007CB9002000E000208B6923F40053146A61
S31508014F101C4208D140B9526ACB691A4204D0012011
S31508014F2002E01846F0E7012010BC70472DE9F04170
S31508014F3004460D46FFF7C5FF064684F82F002946A5
S31508014F402046FFF7CAFF074684F8300094F8313047
S31508014F5033B1012B21D0002384F83130BDE8F0812B
S31508014F6094F84280B8F1000F04D12169A8687CF051
S31508014F70CDFA40B9B8F1000FF0D06169A8687CF0A4
S31508014F80C5FA0028EAD0002EE8D1002FE6D1012380
S31508014F9084F8423084F83130E0E72169A8687CF06A
S31508014FA0ABFA10B90EB9002FD8D0002384F83130E6
S31508014FB0D4E738B504460D46FFF713FF29462046C0
S31508014FC0FFF7B4FF38BD0000014B0360704700BF0F
S31508014FD0A42D090810B50446FFF7F6FF402120461F
S31508014FE04DF05CF9204610BDC0E900239DF800305C
S31508014FF003729DF8043043729DF8083083729DF858
S315080150000C30C372704704307047052180F8381098
S31508015010002180F839108262C3620262436200226B
S315080150200023C0E90C2380F83A10704710B50446EE
S31508015030094B03600123436083604FF46162C260D8
S31508015040036143614FF4E153836100220023FFF7B3
S31508015050DCFF204610BD00BFA42D0908008F0128DA
S3150801506014BF002001207047008F022814BF0020BA
S3150801507001207047008F042814BF002001207047C3
S31508015080008F052814BF00200120704790F8393099
S315080150903BB990F83830032B05D0062B05D00020F4
S315080150A0704700207047012070470120704790F82B
S315080150B038007047006B704790F83A0070470B7AD2
S315080150C00BB14B7A2BB98B7A2BB1CB7A2BB9002042
S315080150D0704701207047002070470420704738B593
S315080150E004460D46FFF7EBFF2B686968002284F832
S315080150F03A2094F83920013A032A08D8DFE802F061
S315080151000228446101280DD0002284F8392094F838
S3150801511038506A1E052A00F2E480DFE802F06E873D
S3150801512087ABBEBEA26AE56A9A1A61EB0505D4F891
S3150801513004C0624575F10002E9DB002284F83920D2
S3150801514023626162012284F8382084F83A20DEE776
S31508015150B0B9A26AE56A9A1A61EB0505D4F808C0DE
S31508015160624575F10002D2DB002284F839202362F8
S315080151706162022284F83820012284F83A20C6E7BF
S31508015180002284F83920C2E7042803D0002284F8D3
S315080151903920BCE7A26AE56A9A1A61EB0505D4F8D3
S315080151A010C0624575F10002B1DB002284F839208E
S315080151B023626162042284F83820012284F83A20A5
S315080151C0A5E7B0B9A26AE56A9A1A61EB0505D4F8AA
S315080151D014C0624575F1000299DB002284F8392072
S315080151E023626162052284F83820012284F83A2074
S315080151F08DE7002284F8392089E794F839202AB9FD
S3150801520060B9A362E162022284F83920226A606ADF
S315080152109B1A61EB00012363616338BD0428F5D14C
S31508015220A362E162032284F83920EFE794F8392072
S31508015230002AEBD1012811D0042815D0022DE5D179
S31508015240226A606A9A1A61EB0000E568AA4270F15F
S315080152500002DBDB032284F83820D7E7A362E16288
S31508015260012284F83920D1E7A362E162032284F896
S315080152703920CBE794F83920002AC7D128B9A36287
S31508015280E162042284F83920C0E70128BED1A3626D
S31508015290E162012284F83920B8E794F83920002A16
S315080152A0B4D1012811D0042815D0052DAED1226A12
S315080152B0606A9A1A61EB0000A569AA4270F10002B8
S315080152C0A4DB062284F83820A0E7A362E162012262
S315080152D084F839209AE7A362E162032284F8392027
S315080152E094E723626162052284F838208EE701601B
S315080152F07047002141604FF0FF0C80F808C080F824
S3150801530009C04FF6FF724281C16080F810C080F86B
S3150801531011C042824161816102774277C28301628B
S3150801532080F8242080F82520C2848162C16280F831
S315080153303020416380F83820C1630022027070472B
S315080153402DE9F04F9DB00B680F934FF0000B00222B
S315080153501A92CDF860B04FF0FF331393119212935E
S3150801536010920192DA46099308931E46039207930F
S3150801537006931D4602920C92CDF814B01793169314
S315080153800E930B92159314930D930A921990BEE0FE
S315080153904FF00008C9E038464DF052FAB5E000254D
S315080153A055E0304609F0D6FC0A997CF09BF810B90D
S315080153B00D9B002B0BDA304609F0CCFC0A909DF9BF
S315080153C010300D9363B214930FFA8AF3159330468E
S315080153D009F0C0FC0B997CF0A3F810B90E9B002BC1
S315080153E00BDA304609F0B6FC0B909DF910300E9396
S315080153F063B216930FFA8AF31793304609F0AAFC9B
S3150801540001460C987BF0C8FD0C90059B013305936A
S315080154102CE0304609F09CFC03909DF9107063B2AC
S3150801542008930FFA8AF30993304609F091FC01466D
S3150801543001987BF0B1FD01900AF1010A0134112CA2
S3150801544034DCACD804EB44056D00203545442146CF
S31508015450484609F0B9FC064628460AF030FB0028FA
S31508015460ECD028460AF03BFB00289AD1304609F0D1
S315080154706FFC02997CF036F810B9BBF1000F0ADA15
S31508015480304609F065FC02909DF910B063B20693A7
S315080154900FFA8AF30793304609F05AFC03997CF010
S315080154A03FF80028B5D1002FBEDAB2E75D463E4681
S315080154B0DDF810B01B9F484609F090FC10997CF066
S315080154C011F810B9129B002B06DA484609F086FC3A
S315080154D010904FFA8BF31293484609F07FFC119905
S315080154E07CF01EF810B9139B002B06DA484609F022
S315080154F075FC11904FFA8BF31393B8F8103013F02B
S31508015500080F29D038464DF09BF90BF1010BBBF179
S31508015510000F2DDC0F9809F094FCBBF1000F7FF406
S3150801552037AF4FF0B00808FB0B0859460F9809F03A
S3150801553009FE814608F18C0738464DF031F998F88D
S31508015540003013F0040F3FF426AF0024CDF810B055
S31508015550AB461B97374672E7484609F03FFC0146BA
S315080155601A987BF019FD1A90189B01331893C9E70D
S31508015570199F0A9B7B600D9B3B72149B7B72159B43
S315080155807B810B9BFB600E9B3B74169B7B74179B65
S315080155907B820598002837D07BF0B2FD01460C982E
S315080155A07BF0B6FE7861029BBB613D77069B7B77F4
S315080155B0079BFB83039B3B6287F82460089B87F85C
S315080155C02530099BFB84BAF1000F1FD050467BF0AA
S315080155D097FD014601987BF09BFEB862109BFB6222
S315080155E0129B87F83030119B7B63139B87F8383001
S315080155F0189868B17BF084FD01461A987BF088FEFD
S31508015600F8631DB0BDE8F08F0020CBE70020E4E782
S315080156100020F5E74068704790F90800704790F94F
S3150801562009007047C068704790F91000704790F9F3
S3150801563011007047406970478069704790F91C00EE
S31508015640704790F91D007047006A704790F9240069
S31508015650704790F925007047806A7047014B0360CF
S31508015660704700BFB42D090810B50446FFF7F6FFC9
S31508015670302120464CF012FE204610BDC0E9002319
S31508015680009B8360019BC3609DF8083003747047D3
S3150801569030B40B4A02600022027680F828200949B4
S315080156A0416009498160C260026102750121417543
S315080156B08275C27500240025C0E9084530BC7047CB
S315080156C0B42D090833333340000040400430704795
S315080156D0007E0238C0B201288CBF00200120704725
S315080156E090F82800704710B50B46027D42B1C9688B
S315080156F01C7C3CB140687BF013FF20B9002402E012
S315080157008968F5E70024204610BD10B50B46027DD1
S3150801571042B1C9681C7C3CB180687BF0EDFE20B9BA
S31508015720002402E08968F5E70024204610BDF8B593
S315080157300446437D93B10D46837D8BB90B684E684C
S31508015740076A426ADF1946EB020607624662037E6A
S31508015750032B78D8DFE803F00A17394D0376F8BD2D
S3150801576002230376012380F82830F8E7FFF7BBFF09
S3150801577084F828000028F2D001232376002200238A
S31508015780C4E90823EBE7FFF7AEFF84F8280020B940
S31508015790002384F828302376E1E7E168CA0E4B0135
S315080157A05B1A62F10002920042EA93729B005B184F
S315080157B042F10002D20042EA5372DB009F4276EBC5
S315080157C00203CCD302232376C9E7C37D002BC6D1B6
S315080157D0FFF789FF84F8280029462046FFF795FF39
S315080157E00028BCD00323237600220023C4E908231A
S315080157F0B5E7FFF778FF84F8280029462046FFF722
S3150801580084FF10B902232376A9E72069C20E430152
S315080158101B1A62F10002520242EAD3525B021B18BA
S3150801582042F10002950145EA93659901CB1A65EBA8
S3150801583002021B1842F100029F4276EB02038ED345
S31508015840002323768BE70023037688E710B5044601
S31508015850074B40F8203B05F097F904F1180005F0CD
S3150801586093F904F1100005F08FF9204610BD00BF29
S31508015870C42D090810B50446FFF7E8FF282120467C
S315080158804CF00CFD204610BDC0E90023009B836047
S315080158909DF8043003739DF8083043739DF80C3066
S315080158A083739DF81030C3739DF8143003749DF803
S315080158B0183043747047000038B504460B4B036033
S315080158C00025C5602946103005F05AF9294604F124
S315080158D0180005F055F9294604F1200005F050F99C
S315080158E0034B636001232372204638BDC42D090882
S315080158F0CDCC0C402DE9F04387B004460D4617463A
S315080159001E46DDF8388021F00049414948467BF0BA
S3150801591011FE002872D13E4948467BF001FE002857
S315080159206CD127F000493A4948467BF003FE002826
S3150801593066D1374948467BF0F3FD002860D126F049
S315080159400049334948467BF0F5FD00285AD13049CC
S3150801595048467BF0E5FD002854D128F000492C493A
S3150801596048467BF0E7FD00284ED1294948467BF099
S31508015970D7FD002848D1E560D4F804904FF07C5152
S3150801598048467BF011FC29467BF0CAFD40B94FF029
S315080159907F5148467BF008FC29467BF0A3FD08B1F8
S315080159A0C4F80C906D463946284605F0E9F804F125
S315080159B0100395E8030083E80300284605F0E4F898
S315080159C002AD3146284605F0DBF804F1180395E8DF
S315080159D0030083E80300284605F0D6F804AD4146DE
S315080159E0284605F0CDF8203495E8030084E803003D
S315080159F0284605F0C9F807B0BDE8F083656890E761
S31508015A0000279CE70026A8E74FF00008B3E700BF88
S31508015A10FFFF7F7F04307047037A002B00F0FC807C
S31508015A202DE9F0438BB004460D460B7C002B63D160
S31508015A304B7C002B60D1D1E900017BF06FFB7749E4
S31508015A407BF066FC0646A86803689B689847074684
S31508015A5000217BF05BFD10B16B7B002B4FD107F169
S31508015A600041684605F08CF83146684605F076F936
S31508015A706B49684605F072F904F11008684605F0A5
S31508015A8084F80146404605F0CFF8684605F083F8E4
S31508015A900146404605F0C8F8404605F076F800216B
S31508015AA07BF020FD00283AD1684605F06DF82B7B7E
S31508015AB0002B44D1AB7B002B6ED00DF118080021C9
S31508015AC0404605F05DF804F1200398E8030083E8F1
S31508015AD00300404605F058F8EB7B002B7DD008AD56
S31508015AE00021284605F04CF8183495E8030084E8A7
S31508015AF00300284605F048F80BB0BDE8F0830DF120
S31508015B0008080021404605F03BF804F1100398E81F
S31508015B10030083E80300404605F036F8C7E70DF1B0
S31508015B2010080021404605F02BF804F1100398E807
S31508015B30030083E80300404605F026F8B4E704F1BC
S31508015B401008404605F023F800217BF0E9FC0028FF
S31508015B50B0D0404605F01BF881464FF07C5160688D
S31508015B607BF022FB014648467BF0D0FC0028A1D0F9
S31508015B70404605F00CF881464FF07F5160687BF08E
S31508015B8013FB014648467BF0B7FC002892D04046F5
S31508015B9004F0FDFFE0608DE707F10041684604F077
S31508015BA0EFFF3146684605F0D9F81D49684605F004
S31508015BB0D5F804F12008684604F0E7FF0146404697
S31508015BC005F032F8684604F0E6FF0146404605F05E
S31508015BD02BF8684604F0D8FF7EE73946684604F094
S31508015BE0CFFF3146684605F0B9F80D49684605F014
S31508015BF0B5F81834684604F0C8FF0146204605F092
S31508015C0013F8684604F0C7FF0146204605F00CF86C
S31508015C10684604F0B9FF6FE7704700BF002474496E
S31508015C20B4A29139C068704708B5103004F0AFFFC7
S31508015C3008BD08B5183004F0AAFF08BD08B520301C
S31508015C4004F0A5FF08BD0000014B0360704700BFC3
S31508015C50502E090810B50446FFF7F6FF28212046FD
S31508015C604CF01CFB204610BDC0E90023009B836055
S31508015C70019BC360029B03619DF80C3003759DF877
S31508015C80103043759DF8143083759DF81830C37527
S31508015C909DF81C300376704730B40C4A0260002226
S31508015CA042618261002101774177094A42604FF0DA
S31508015CB07A5282600122C260027442748274C1748B
S31508015CC000240025C0E9084530BC7047502E090854
S31508015CD0CDCCCC3D04307047007F7047407F70477C
S31508015CE0007F0138C0B205288CBF0020012070470B
S31508015CF02DE9F04F87B0037C8DF81030437C8DF881
S31508015D001130837C23B9BDF81030ADF8143067E043
S31508015D108B6803934FF0000ACDF808A0CDF804A0CC
S31508015D20DFF8D49031E000273BE058464CF088FD77
S31508015D3029E0002408E00135112D21DCF9D805EB0D
S31508015D404504640020343C442946404609F03CF8A1
S31508015D500646204609F0B3FE0028ECD0304608F086
S31508015D60F7FF49467BF0BEFB0028E4D0304608F031
S31508015D70EFFF81460AF1010301936B1C0293DAE7EF
S31508015D8058464CF05DFD0AF1010ABAF1000F18DC1C
S31508015D90039809F056F8BAF1000FC4D1B02707FBEA
S31508015DA00A075146039809F0CDF9804607F18C0B8D
S31508015DB058464CF0F5FC3B7813F0040FB5D0002596
S31508015DC0BAE70D4948467BF083FB28B9019B8DF854
S31508015DD01030029B8DF81130BDF81030ADF8143033
S31508015DE000209DF8143063F307009DF8153063F31E
S31508015DF00F2007B0BDE8F08F9AF9794410B50B4624
S31508015E00144611780139986809F09CF938B1617816
S31508015E10013908F0D9FF20B108F09AFF00E0002007
S31508015E2010BD0020FCE710B50B4614461178013960
S31508015E30D86809F04BFB38B16178013909F0B1F935
S31508015E4020B109F09AF900E0002010BD0020FCE716
S31508015E50F0B593B006460C46154611A81FF0E6F9AB
S31508015E603649204670F032F9002862D004460EA859
S31508015E704CF070FB05A90EA871F06AF82946304660
S31508015E80FFF736FFADF8100004AA29463046FFF79A
S31508015E90B5FF074604AA29463046FFF7C4FF06465A
S31508015EA0059B0393069B0293079B01930A9B03F2A7
S31508015EB06C730093099B0133089A2149204649F0DE
S31508015EC098FF28697AF0C2FC02460B461D4920460E
S31508015ED049F08FFF1C4D9DF810202946204649F0B0
S31508015EE088FF9DF811202946204649F082FF384649
S31508015EF07AF0ACFC02460B461449204649F079FF74
S31508015F0030467AF0A3FC02460B461149204649F071
S31508015F1070FF2346022201210E4870F0D3FF204666
S31508015F206FF064FE012411A81FF0FCF9204613B096
S31508015F30F0BD11A81FF0CCF80024F4E734430B0890
S31508015F40CC2D0908EC2D0908F42D0908F82D0908A6
S31508015F50002E0908A4E20B0870B582B004460D4666
S31508015F6008684968226A636A801841EB030320625C
S31508015F706362227F072A00F20A81DFE812F008002D
S31508015F8010005D007500A600B600EB0000010023B5
S31508015F906377E37C002B46D00123237743E0002374
S31508015FA0637701A81FF042F97A497B4870F08EF8A9
S31508015FB00646002839D0034605220121774870F0A4
S31508015FC081FF334604220121754870F07BFF334671
S31508015FD006220121734870F075FF33460522012117
S31508015FE0714870F06FFF3346042201216F4870F043
S31508015FF069FF33460A2201216D4870F063FF334673
S31508016000022201216B4870F05DFF30466FF0EEFD0C
S31508016010616828697AF0C0FF6061042323770DEB74
S3150801602003001FF07FF902B070BD01A81FF050F8F8
S3150801603001A81FF077F9F6E701236377E37C0BB92B
S315080160402377F0E72B7E002BEDD129462046FFF773
S315080160504FFEADF8040001AA29462046FFF7CEFEF9
S31508016060A06103232377DEE701236377E37C0BB97A
S315080160702377D8E729462046FFF73AFEADF804000C
S3150801608001AA29462046FFF7B9FE06466B7D1BB9CC
S31508016090AB7D0BB9EB7D13B107232377C3E72B7DC3
S315080160A013B106232377BEE7616928697BF02EFAC7
S315080160B040B93146A0697AF06DFFA1687BF026FAEE
S315080160C00028B0D004232377ADE700236377E37C68
S315080160D00BB92377A7E72B7E002BA4D005232377BB
S315080160E000220023C4E908239DE700226277E27CA7
S315080160F012B90023237796E7E668F10E7201921B1F
S3150801610061F10001490241EAD2515202921941F163
S3150801611000014FEA811E4EEA926E4FEA821CBCEBE1
S3150801612002026EEB0101921941F1000190428B4185
S31508016130FFF479AF2A4618492046FFF789FE002859
S315080161403FF471AF616828697AF026FF606102231E
S31508016150237768E700236377E37C0BB9237762E744
S315080161602B7E002B3FF45FAF2A460B492046FFF7EB
S315080161706FFE00283FF457AF0723237753E7002321
S315080161806377E37C002B7FF44EAF23774BE700233D
S31508016190237748E704640908082E0908202E090808
S315080161A0282E0908302E0908382E0908402E090814
S315080161B0A4400B08A4E20B08014B0360704700BF1B
S315080161C0602E09080B8802889B1A1BB2002B01DD79
S315080161D00120704701DB002070474FF0FF30704700
S315080161E010B50446FFF7E8FF282120464CF056F87B
S315080161F0204610BD0170427083709DF90030C3704E
S3150801620070470000104B0360002343620F4A426047
S315080162100F4A82600F4AC2600F4A02610F4A426101
S315080162200122027643768376C361002B05DCC21808
S31508016230002182F820100133F7E7012380F8213085
S31508016240002380F822307047602E090800008C422E
S315080162509A9979400AD7A33C0AD7233C8FC285402D
S3150801626004307047406A0028D4BF002001207047D7
S31508016270406A7047F8B50C46C06908F0E2FD6CB98A
S31508016280B02606FB040606F18C0738464CF088FA58
S31508016290337813F0040F03D0002508E00026F2E74F
S315080162A038464CF0CDFA24E0002408E00135112DDA
S315080162B01CDCF9D805EB4504640020343444204637
S315080162C009F0FDFB0028F1D00021204609F04BFC1E
S315080162D0204609F034FC0028E8D00021204609F0C0
S315080162E022FC0121204609F00EFCDFE738464CF076
S315080162F0A7FAF8BD2DE9F04F85B0019003914FF04B
S31508016300000B0027DA4632E04FF000083DE002981C
S315080163104CF096FA29E000240DE0504608F018FDE5
S31508016320074626460135112D1BDCF4D805EB450435
S315080163306400203444442946484608F045FD82460F
S31508016340204609F0BCFB04460028EBD0504608F06D
S31508016350FFFC39467BF0C6F80028DED1002EE1D1D4
S31508016360DBE7B24602984CF06BFA0BF1010BBBF175
S31508016370000F1EDC019BD86908F063FDBBF1000F15
S31508016380C2D14FF0B00808FB0B085946019BD869E2
S3150801639008F0D8FE814608F18C03029318464CF0A2
S315080163A0FFF998F8003013F0040FB0D000255646CF
S315080163B0B9E7BAF1000F03D1504605B0BDE8F08F31
S315080163C0039B1F60F8E72DE9F84F05460C469246F0
S315080163D0C06908F036FD64B94FF0B00808FB040837
S315080163E02146E86908F0AEFE074600250026A946BB
S315080163F00AE04FF00008F3E700240DE0584608F0DC
S31508016400A7FC0646A1460135112D1CDCF4D805EB7F
S3150801641045046400203444442946384608F0D4FC2F
S315080164208346204609F04BFB04460028EBD0584624
S3150801643008F08EFC31467BF055F80028DED1B9F11B
S31508016440000FE0D1DAE7B9F1000F02D14846BDE8FD
S31508016450F88FCAF80060F9E738B50569C4682946AE
S3150801646020467BF03FF800B92C46204638BD00008F
S315080164702DE9F84304460E4617461D46437E012B71
S3150801648028D0022B1AD07BB14FF00008A37E6BB33C
S31508016490012B2ED196F90390B9F1000FD4BF4FF015
S315080164A000094FF0010926E00B78B3B991F801808C
S315080164B0B8F1000FEAD04FF00108E7E70B787BB98E
S315080164C04B7883B991F80280B8F1000FDED04FF00E
S315080164D00108DBE74FF00108D8E74FF00108D5E7D7
S315080164E04FF00108D2E74FF00108CFE74FF0010955
S315080164F001E04FF00009284608F02AFC39467AF0EF
S3150801650049FD0746284608F023FCA1687AF0FEFFF4
S3150801651078B13946E0687AF0EFFF20BB96F9033087
S31508016520002B06DD2046FFF797FF39467AF0E4FF90
S31508016530D8B9284608F00CFC61697AF0E7FF40B93A
S315080165400020B8F1000F12D0B9F1000F10D10020C8
S315080165500EE0284608F0FCFB06497AF0C3FF00283E
S31508016560EFD00120EDE70120EBE70120E9E7002064
S31508016570BDE8F8830000A0402DE9F041044617461E
S315080165801E46437EB3B1022B1BD00025A37E012BE9
S3150801659026D04FF00008304608F0DAFB61697AF038
S315080165A0A1FF38BB0023002D41D1B8F1000F3DD121
S315080165B01D463CE00D786DB94B78002BE6D10125D7
S315080165C0E4E70D7845B94B78002BDFD18A782AB1F3
S315080165D01D46DBE70025D9E70025D7E70125D5E7DD
S315080165E091F90380B8F1000FCCBF4FF000084FF0C6
S315080165F00108D0E7304608F0ABFBA1687AF072FFD4
S3150801660008B10123CFE7304608F0A2FB39467AF0F4
S31508016610C1FC06462046FFF71FFF014630467AF0C1
S3150801662061FF08B90023BEE70123BCE745462846B2
S31508016630BDE8F0812DE9F04F99B080468A461546A6
S3150801664004921C46C06908F0FCFB75BB4FF0B00B01
S315080166500BFB050B0499D8F81C0008F073FD81465D
S315080166600BF18C03059318464CF09AF89DF888703F
S315080166703F1BFFB20137FFB20025AF4218DD2146A5
S31508016680484608F0A1FB08F063FB68497AF08CFDDF
S3150801669018AB03EB85067AF063FF26F8480C631CF2
S315080166A006F8464C0135DCB2E7E74FF0000BD1E7B7
S315080166B0D8F804505E4928467AF06CFC04460297DD
S315080166C0BBF8103013F0280F2ED1239928467AF0FB
S315080166D013FF002830D1239920467AF003FF28B307
S315080166E0214623987AF056FC0646214628467AF032
S315080166F051FC014630467AF00BFE01464FF07E50BA
S315080167007AF048FC044638467AF0F6FC21467AF0D7
S315080167104BFD7AF04BFF0446464B0422394606A840
S3150801672071F0E6FD029401E000230293002503952A
S315080167303B464F4699461CE000230293F6E70024A0
S3150801674025E00021204609F00EFA204609F017FA3D
S3150801675010B1029B002B4CD1204609F0F0F9002814
S3150801676053D1204609F0EBF910B1039B013303938A
S315080167700135A94552DD18AB03EB850313F8461C11
S315080167801129DCD801EB4104640020345C44384605
S3150801679008F01AFB0646204609F091F90028E7D0C9
S315080167A03346249A51464046FFF762FE0190334626
S315080167B0249A51464046FFF7DFFE064698F82230EE
S315080167C033B9019B43B1049B434493F820301BB969
S315080167D00121204609F0C7F998F82230002BB4D1D7
S315080167E0002EAED1049B434493F82030002BACD045
S315080167F0A7E70121204609F096F90121204609F06B
S3150801680082F9029B013B0293ABE70021204609F07E
S315080168108AF90121204609F076F9A2E705984CF094
S315080168200FF8039819B0BDE8F08F00BF00007A444D
S315080168300000A040C5610108C369002B00F0B880BB
S315080168402DE9F04F87B00446884690F8213073B990
S315080168500025002D05DC29462046FFF70BFD0135ED
S31508016860F7E700266662666207B0BDE8F08F002387
S315080168700493037E012B02D000252E4641E090F8B1
S315080168802230002BF8D104A9FFF734FD0028F3D1F3
S3150801689000236362E8E700273DE058464BF0D0FF46
S315080168A02EE005AA29462046FFF78DFD002849D185
S315080168B058464BF0C5FF23E0012B43D1049B0593B2
S315080168C040E00C235FFA83FA12F0010F03D0FB892B
S315080168D0B3F5417F41D2484608F080FA0746584643
S315080168E04BF0AEFF059B029301970AF1FF33DBB22A
S315080168F0009300232A4641462046FFF79BFE06449D
S315080169000135002DAFDCE06908F09BFA002DC2D1F4
S31508016910B02707FB05072946E06908F013FC8146FD
S3150801692007F18C0B58464BF03BFF3B7813F0040FED
S31508016930B3D000230593237E002BBDD194F82230D2
S31508016940002BAED07A8812F01C0FBAD112F0010FC3
S3150801695001D10C23B6E71223B4E7484608F041FAF9
S315080169600746484608F040FA814658464BF068FF04
S315080169704FEA5A0B059B029301970BF1FF33DBB2E2
S31508016980009300232A4641462046FFF753FE064454
S31508016990059B0293CDF804900AF1FF33DBB200930D
S315080169A05B462A4641462046FFF744FE0644A7E7CA
S315080169B070470000014B0360704700BF702E09083D
S315080169C010B50446FFF7F6FF202120464BF066FC7A
S315080169D0204610BDC0E90023BDF8003003819DF8AB
S315080169E0043083727047000030B4094A02600022FD
S315080169F00275012181804FF47A748460C160027442
S31508016A004274827400240025C0E9064530BC7047EB
S31508016A10702E090804307047007D0238C0B201287B
S31508016A208CBF0020012070478B7A3BB90A8983887D
S31508016A309A4201D001207047002070470020704714
S31508016A4070B50446037C8BB1437C8BB90B684D68E2
S31508016A508669C2699E1945EB02058661C561037D92
S31508016A60032B64D8DFE803F00712303E037570BDC7
S31508016A7002230375FBE7FFF7D7FF0028F7D00123A9
S31508016A80237500220023C4E90623F0E7FFF7CCFFAC
S31508016A9010B900232375EAE7A168CA0E4B015B1AF0
S31508016AA062F10002920042EA93729B005B1842F17E
S31508016AB00002D20042EA5372DB009E4275EB0203E2
S31508016AC0D5D302232375D2E7837C002BCFD1FFF7D9
S31508016AD0ABFF0028CBD10323237500220023C4E989
S31508016AE00623C4E7FFF7A0FF10B102232375BEE70B
S31508016AF0E068C20E43011B1A62F10002520242EA21
S31508016B00D3525B021B1842F100024FEA821C4CEA7F
S31508016B10936C9901CB1A6CEB02021B1842F1000225
S31508016B209E4275EB0203A2D3002323759FE7002338
S31508016B3003759CE7024A0260024A0260704700BF79
S31508016B40982E0908802E090810B5044640687AF07F
S31508016B502BFBA06010BD8068704710B50446FFF78F
S31508016B60E9FF0C2120464BF099FB204610BD000099
S31508016B70044A0260044A0260002282604FF07E5293
S31508016B8042607047802E0908982E0908043070471C
S31508016B90014B0360704700BFB02E090810B50446C3
S31508016BA0FFF7F6FF702120464BF078FB204610BD13
S31508016BB0C0E900239DF9003003729DF90430437240
S31508016BC09DF9083083729DF80C30C3729DF8103018
S31508016BD003739DF8143043739DF8183083739DF839
S31508016BE01C30C3739DF8203003749DF82430437418
S31508016BF09DF8283083749DF82C30C3740C9B43612F
S31508016C000D9B83619DF838300377704730B41D4A70
S31508016C100260002280F8582080F8682080F86920F0
S31508016C2080F86A2080F86B200121017141714FF4C7
S31508016C307A748460C4600174427442618261C2617B
S31508016C40026242628262C262026342638263C26311
S31508016C50026480F8442080F8452080F8462080F8B0
S31508016C60472080F84820084CC464084C046580F81D
S31508016C70542080F8551000240025C0E9184530BC79
S31508016C80704700BFB02E090805042300030002005F
S31508016C900430704790F85800B0FA80F04009704700
S31508016CA090F86800704790F858000338C0B2012878
S31508016CB08CBF00200120704790F86A00704790F851
S31508016CC0690070470379013BDBB2012B01D900202A
S31508016CD0704790F854300BB1CB7C3BB191F9093030
S31508016CE0002B01DD01207047002070470020704706
S31508016CF00379013BDBB2012B01D900207047887C5F
S31508016D007047034690F854200AB1C87C00E0012078
S31508016D101B7923B1012B03D0022B0AD0002070471F
S31508016D2028B191F90830002BF9DC002070470020C2
S31508016D30704728B191F90A30002BF0DC0020704722
S31508016D40002070470346887C00283AD1B3F804C06E
S31508016D5040F2011294451BD093F8442032B393F8BC
S31508016D6045201AB310B44C6914F4005F03D18C7B27
S31508016D709CB1CA7B9AB193F8463093B14A6912F429
S31508016D80004F0FD10A7C7AB14A7C5AB9184609E0F4
S31508016D904A7B002AE0D010467047104602E020469A
S31508016DA000E0184610BC70471846FBE793F84630D2
S31508016DB043B14A6912F4004F03D10A7C22B14A7CD5
S31508016DC022B17047184670471846704718467047EB
S31508016DD0C26C4B691A4208D1026D8B691A4206D1F7
S31508016DE090F847302BB1087F704701207047012082
S31508016DF070470020704730B40346144612B1027C2E
S31508016E00002A69D1D868002C67D05A7C002A64D038
S31508016E10DC6C4A69224012F0040F03D05C69844293
S31508016E2000D8204612F0010F03D09C69844200D88D
S31508016E3020461C6D8D692C4014F0010F03D0DD69C5
S31508016E40854200D8284614F0020F03D01C6A8442F2
S31508016E5000D8204693F8444034B112F4005F03D0B9
S31508016E605C6A844200D8204693F8464034B112F44D
S31508016E70004F03D09C6A844200D8204693F84740C5
S31508016E8034B112F0005F03D0DD6A854200D8284686
S31508016E902CB1097F19B1196B814200D8084612F441
S31508016EA0803F03D0596B814200D8084612F4003F4F
S31508016EB003D0996B814200D8084612F4001F03D00B
S31508016EC0D96B814200D8084612F4806F05D01B6C35
S31508016ED0834202D8184600E0002030BC70472DE9ED
S31508016EE0F843044690F85530DBB10D460B684F68F8
S31508016EF0026E416E13EB020847EB0107C0F860808A
S31508016F0047662946FFF764FF064684F86B0094F83E
S31508016F105830042B00F21A81DFE803F00A3C8BBBD8
S31508016F20E80080F8683080F8693080F858302FE03A
S31508016F30002384F8683029462046FFF7C3FE20B1AE
S31508016F4029462046FFF7D4FE48B129462046FFF7D1
S31508016F50D8FE90B129462046FFF7F4FE68B966B90E
S31508016F60012384F86930EB7A53B1012384F8583048
S31508016F7000220023C4E9182302E0002384F86930BB
S31508016F8094F85830032B00F0E580002384F86A3022
S31508016F90BDE8F883002384F8683029462046FFF7C0
S31508016FA091FE814620B129462046FFF7A1FE48B148
S31508016FB029462046FFF7A5FE98B329462046FFF73E
S31508016FC0C1FE70BB6EBBA168CA0E4B015B1A62F1AA
S31508016FD00002920042EA93729B005B1842F100029A
S31508016FE0D20042EA5372DB00984577EB0203C7D316
S31508016FF094F84830CBB1B9F1000F04D029462046A0
S31508017000FFF776FE48B129462046FFF77AFE60B1BA
S3150801701029462046FFF796FE38B9022384F85830E8
S31508017020AEE7002384F85830AAE7032384F85830DA
S31508017030A6E7012384F8683029462046FFF742FE71
S3150801704020B129462046FFF753FE48B12946204676
S31508017050FFF757FEC8B129462046FFF773FEA0B9C8
S315080170609EB92B7B002B8BD029462046FFF749FE7C
S31508017070002885D029462046FFF764FE00287FF4BC
S315080170807FAF032384F858307AE7002384F8583011
S3150801709076E794F848705FB129462046FFF712FE55
S315080170A0074628B129462046FFF722FE00B10027E8
S315080170B084F86870237C23B11EB1002384F8583004
S315080170C05EE729462046FFF71CFE38B129462046C9
S315080170D0FFF738FE10B9002E3FF452AF042384F8A7
S315080170E0583000220023C4E9182349E7002384F80D
S315080170F0683029462046FFF704FE28B1294620466E
S31508017100FFF720FE00B9EEB1324629462046FFF7C1
S3150801711072FEC20E43011B1A62F10002920042EA94
S3150801712093729B001B1842F10002D20042EA537285
S31508017130DB00984577EB0203FFF422AF002384F8BE
S3150801714058301DE7032384F8583019E7002384F8DB
S31508017150583015E7EB7C19E7014B0360704700BF10
S31508017160C02E090810B50446FFF7F6FF5021204640
S315080171704BF094F8204610BDC0E900239DF9003074
S3150801718003729DF9043043729DF9083083729DF9A3
S315080171900C30C3729DF8103003739DF81430437395
S315080171A09DF8183083739DF81C30C3739DF8203001
S315080171B003749DF8243043749DF8283083749DF830
S315080171C02C30C3749DF8303003759DF834304375FF
S315080171D09DF8383083759DF83C30C375109B8361E3
S315080171E0119BC3617047000030B41B4A026000223C
S315080171F080F8382080F8392080F83A2080F848202D
S3150801720080F8492080F84A2080F84B2080F84C20E5
S3150801721080F84D2080F84E2080F84F2002714FF4F7
S315080172207A718160C1600121017442740B4C446119
S315080172300B4C84610B4CC4610B4C04624262826242
S31508017240C262026380F8342080F8351000240025D4
S31508017250C0E9104530BC7047C02E09080504230053
S31508017260030002001B0441001000020004307047AD
S3150801727090F84900704790F84800704790F839002F
S31508017280704790F84A00704790F84B00704790F89D
S315080172904C00704790F84D00704790F84E007047C3
S315080172A090F83830032B00F28580DFE803F0022FCF
S315080172B04B6491F90830002B19DD4B7B13B303237B
S315080172C080F8383090F83830012B79D0032B75D0F7
S315080172D0002380F83930002380F84E3080F84D308D
S315080172E080F84C3080F84B3080F84A30704791F975
S315080172F00930002BE1DCCB7B002BE3D0012380F89E
S315080173003830DFE7022380F83830DBE791F90830B7
S31508017310002B05DD4B7B73B1032380F83830D1E7A9
S3150801732091F90930002BF5DC8B7B002BCAD00023A1
S3150801733080F83830C6E70B7B002BC3D0022380F8D0
S315080173403830BFE791F90830002B06DD4B7B002B5F
S31508017350B8D0032380F83830B4E791F90930002B07
S31508017360F4DCCB7B1BB1012380F83830AAE7002374
S3150801737080F83830A6E791F90830002B06DD4B7BFB
S31508017380002B9FD1022380F838309BE791F9093009
S31508017390002BF4DC0B7B002B94D0CB7B1BB1012398
S315080173A080F838308EE78B7B002B8BD0002380F852
S315080173B0383087E7002380F8383083E7012388E7E8
S315080173C0012386E791F90A000028D4BF002001208D
S315080173D07047002070470379012B11D0022B01D089
S315080173E00020704791F90930002B01DD0120704713
S315080173F091F90B30002B01DD012070470020704701
S31508017400012070478B7D0BB1C87D704700207047FE
S31508017410F0B403464269446A22EA04008D692842A7
S3150801742012D19E69D3F828C026EA0C00CF693842E2
S3150801743025D1087D28B32240154206D106EA0C0655
S31508017440374202D1002000E00120DA69DC6A22EA2B
S31508017450040C15EA0C0F16D11E6AD3F830C026EAB9
S315080174600C03CF693B4213D14B7D9BB12240154298
S315080174700AD106EA0C06374206D1002304E00120A8
S31508017480E3E70020E1E7012300B91846F0BC70479D
S315080174900123F9E70023F7E742698B691A4207D105
S315080174A0CA69D0F818C01CEA020F0DD0012200E003
S315080174B00122D0F81CC013EA0C0F07D1006ACB6968
S315080174C0184208D0012302E00022F2E7012322B97B
S315080174D02BB1002070470023F9E7002070470120EF
S315080174E070472DE9F84304460D460B684F68066C4C
S315080174F0426C9E1947EB02080664C0F84480FFF700
S3150801750087FF074694F83A30042B00F24B81DFE8EF
S3150801751013F005005C00B000E8001701002384F8A9
S31508017520483029462046FFF74DFF20B12946204617
S31508017530FFF74FFF48B129462046FFF74CFF60B1D8
S3150801754029462046FFF75EFF38B994F84F304BB30A
S3150801755029462046FFF7A0FF30BB002384F84930AF
S3150801756094F83A20D31EDBB2012B8CBF00230123EA
S3150801757084F8393094F83410002900F01B8184F816
S315080175804B3084F84A30B2FA82F35B0984F84D30FD
S3150801759084F84C30032A00F00B81002384F84E301E
S315080175A0BDE8F883002FD8D1012384F84930AB7C94
S315080175B0002BD5D0012384F83A30002384F84F30C4
S315080175C000220023C4E91023CAE7002384F84830BF
S315080175D029462046FFF7F6FE814620B12946204670
S315080175E0FFF7F7FE48B129462046FFF7F4FE90B3A8
S315080175F029462046FFF706FF68BB67BBA168CA0E86
S315080176004B015B1A62F10002920042EA93729B00F7
S315080176105B1842F10002D20042EA5372DB009E4235
S3150801762078EB02039CD3637CFBB1B9F1000F04D05C
S3150801763029462046FFF7CDFE48B129462046FFF7E1
S31508017640CAFE90B129462046FFF7DCFE68B9022337
S3150801765084F83A3084E7002384F83A30002F3FF45F
S315080176607FAF012384F84F307AE7032384F83A3051
S3150801767076E7012384F8483029462046FFF7A2FE1B
S3150801768020B129462046FFF7A4FE48B129462046DF
S31508017690FFF7A1FED8B129462046FFF7B3FEB0B9D8
S315080176A0AFB9EB7C002B3FF45BAF29462046FFF7C9
S315080176B092FE00283FF454AF29462046FFF7A2FE62
S315080176C000287FF44DAF032384F83A3048E70023B6
S315080176D084F83A30002F3FF443AF012384F84F3042
S315080176E03EE7667C5EB129462046FFF76BFE0646F5
S315080176F028B129462046FFF76CFE00B1002684F81A
S315080177004860237C3BB137B1002384F83A30012322
S3150801771084F84F3024E729462046FFF75CFE38B146
S3150801772029462046FFF76EFE10B9002F3FF418AF21
S31508017730042384F83A3000220023C4E910230FE712
S31508017740002384F8483029462046FFF744FE28B12D
S3150801775029462046FFF756FE00B9FFB1E168CA0E71
S315080177604B015B1A62F10002920042EA93729B0096
S315080177705B1842F10002D20042EA5372DB009E42D4
S3150801778078EB0203FFF4ECAE002384F83A30002FBD
S315080177903FF4E6AE012384F84F30E1E6032384F88B
S315080177A03A30DDE6002384F83A3084F84F30D7E6DC
S315080177B02B7CF3E6002384F84E3084F84D3084F8A8
S315080177C04C3084F84B3084F84A30E9E610B5044663
S315080177D090F8353053B10379013B012B21D9FFF7D5
S315080177E05FFD00220023C4E9102310BD80F838305C
S315080177F080F83A3080F8493080F8483080F83930D6
S3150801780080F84A3080F84B3080F84C3080F84D309B
S3150801781080F84E3080F84F3000220023C0E910234B
S31508017820E3E7FFF75EFEE0E7014B0360704700BF41
S31508017830D02E090810B50446FFF7F6FF3821204671
S315080178404AF02CFD204610BDC0E90023DDE90023DE
S31508017850C0E902239DF808300374704730B40F4A13
S31508017860026000220276C26180F82020426200246A
S315080178700025C0E90A450A2141604FF496618160F5
S315080178804FF47A71C1604FF4167101610275427540
S315080178908275C0E90C4530BC704700BFD02E090877
S315080178A004307047C16170472DE9F04190F82030E6
S315080178B023B90B7C13B1C3690133C3610B7C80F80F
S315080178C02030057D002D2ED0477D002F2FD10B6846
S315080178D04E68046B426B1C1946EB02020463426351
S315080178E08E68D1F80CC08368F31A6CF1000EC16A70
S315080178F0D0F82880984571EB0E0304DA8662C0F841
S315080179002CC0C3694362D0F81CE0436AAEEB03039B
S3150801791041688B4200D23D46037E032B59D8DFE8E6
S3150801792003F009122A3400230376BDE8F081022305
S315080179300376FAE7002DF8D0012303760022002307
S31508017940C0E90C23F1E7C568E90E6B015B1B61F120
S315080179500001890041EA93719B005B1941F100011D
S31508017960C90041EA5371DB009C4272EB0103DCD387
S3150801797002230376D9E7837D002BD6D10323037629
S3150801798000220023C0E90C23CFE70569E90E6B0144
S315080179905B1B61F10001490241EAD3515B025B19A4
S315080179A041F100014FEA811848EA93689F01FB1AE1
S315080179B068EB01015B1941F100019C4272EB01037D
S315080179C0B3D38662C0F82CC0C0F824E0002303763E
S315080179D0ABE700230376A8E7007E0238C0B2012888
S315080179E08CBF002001207047C0697047014B0360B6
S315080179F0704700BFE02E090810B50446FFF7F6FFE9
S31508017A00202120464AF04AFC204610BDC0E9002341
S31508017A109DF8003003729DF90430437270470000E7
S31508017A2030B4094A0260002202744FF47A71416047
S31508017A304FF46161816002734273827300240025E9
S31508017A40C0E9064530BC7047E02E09080430704786
S31508017A50007C0238C0B201288CBF00200120704783
S31508017A60087A10B191F9093043B120B991F9093071
S31508017A70012B02D07047002070470120704770B56E
S31508017A800446037BABB191F90930002B11DB437B2B
S31508017A9093B90B684D688669C2699E1945EB02055B
S31508017AA08661C561037C032B65D8DFE803F00813FB
S31508017AB0313F0023237470BD02230374FBE7FFF7EC
S31508017AC0CFFF0028F7D00123237400220023C4E93D
S31508017AD00623F0E7FFF7C4FF10B900232374EAE78A
S31508017AE06168CA0E4B015B1A62F10002920042EA12
S31508017AF093729B005B1842F10002D20042EA53726C
S31508017B00DB009E4275EB0203D5D302232374D2E729
S31508017B10837B002BCFD1FFF7A3FF0028CBD103230B
S31508017B20237400220023C4E90623C4E7FFF798FF5C
S31508017B3010B102232374BEE7A068C20E43011B1AC3
S31508017B4062F10002520242EAD3525B021B1842F169
S31508017B5000024FEA821C4CEA936C9901CB1A6CEB32
S31508017B6002021B1842F100029E4275EB0203A2D3E0
S31508017B70002323749FE7002303749CE7014B0360EA
S31508017B80704700BFF02E090810B50446FFF7F6FF47
S31508017B90282120464AF082FB204610BDC0E9002371
S31508017BA0009B83607047000030B4094A02600022D6
S31508017BB002760849416008498160C260026102751E
S31508017BC04275827500240025C0E9084530BC704716
S31508017BD0F02E09080000B4420000AA42043070479A
S31508017BE0007E0238C0B201288CBF002001207047F0
S31508017BF010B50B464FF001044168986879F090FC7E
S31508017C0008B94FF0000404F0010010BD10B50B4689
S31508017C104FF001048168986879F064FC08B94FF05F
S31508017C20000404F0010010BD70B50446037D8BB154
S31508017C30437D8BB90B684D68066A426A9E1945EB06
S31508017C40020506624562037E032B64D8DFE803F06A
S31508017C500712303E037670BD02230376FBE7FFF772
S31508017C60C7FF0028F7D00123237600220023C4E9A1
S31508017C700823F0E7FFF7BCFF10B900232376EAE7EC
S31508017C80E168CA0E4B015B1A62F10002920042EAF0
S31508017C9093729B005B1842F10002D20042EA5372CA
S31508017CA0DB009E4275EB0203D5D302232376D2E786
S31508017CB0837D002BCFD1FFF7A9FF0028CBD0032363
S31508017CC0237600220023C4E90823C4E7FFF79EFFB1
S31508017CD010B902232376BEE72069C20E43011B1A97
S31508017CE062F10002520242EAD3525B021B1842F1C8
S31508017CF000024FEA821C4CEA936C9901CB1A6CEB91
S31508017D0002021B1842F100029E4275EB0203A2D33E
S31508017D10002323769FE7002303769CE7014B036044
S31508017D20704700BF002F090810B50446FFF7F6FF94
S31508017D30382120464AF0B2FA204610BDC0E9002390
S31508017D40009B8360019BC360029B0361704700002F
S31508017D5030B40E4A0260002280F8202000214162D8
S31508017D604FF0FF318162C162094941600949816069
S31508017D70C26002610849416182610277427782776E
S31508017D8000240025C0E90C4530BC7047002F0908BE
S31508017D900000204200000C420B0401000430704729
S31508017DA090F820000238C0B201288CBF00200120BB
S31508017DB0704700002DE9F04F87B0049205938B6850
S31508017DC001934FF00009CDF80C90CDF80890DFF833
S31508017DD020A1B9F1000F77DC019807F032F8B9F163
S31508017DE0000F19D1B02707FB09074946019807F083
S31508017DF0A9F9804607F18C0B58464AF0D1FC3B7825
S31508017E0013F0040F0AD013F0100F0BD13B7813F0BF
S31508017E10200F18D100252AE00027E6E758464AF040
S31508017E200FFD4EE0404606F0E2FF514679F078FB39
S31508017E300028EBD0404606F0DAFF8246CDF80890D6
S31508017E4000230393E2E7404606F0D4FF514679F052
S31508017E5067FB0028DED0404606F0CCFF8246CDF807
S31508017E60089001230393D5E7002408E00135112D75
S31508017E7024DCF9D805EB4504640020343C44294642
S31508017E80404606F0A1FF0646204607F018FE0028E0
S31508017E90ECD0204607F023FE0028E7D0304606F04E
S31508017EA059FF514679F03CFB0028DFD0304606F0F1
S31508017EB051FF82460395CDF80890D7E758464AF010
S31508017EC0BFFC09F1010984E70949504679F000FB2D
S31508017ED018B1002007B0BDE8F08F049BC3F800A0D5
S31508017EE0059B029A1A60109B039A1A600120F1E712
S31508017EF09AF979C44269CB681A4205D182690B6934
S31508017F001A4203D0012070470120704700207047AC
S31508017F1010B54FF001041146406879F0E3FA08B943
S31508017F204FF0000404F0010010BD10B54FF0010434
S31508017F301146806879F0F4FA08B94FF0000404F0A4
S31508017F40010010BD30B583B00446037FA3B10D46C9
S31508017F50437FABB909686A68036B406B5B1842EBF0
S31508017F6000022363626394F82030032B00F2CA806F
S31508017F70DFE803F00A2C668D80F8203003B030BDA7
S31508017F80022380F82030F9E704F12C03009304F169
S31508017F90280304F1240229462046FFF70BFF00288F
S31508017FA0ECD029462046FFF7A5FF0028E6D1626AEC
S31508017FB029462046FFF7ACFF0028DFD0012384F8C5
S31508017FC0203000220023C4E90C23D7E704F12C034F
S31508017FD0009304F1280304F1240229462046FFF7F9
S31508017FE0E9FE70B129462046FFF784FF48B9626A5F
S31508017FF029462046FFF78CFF38B9002384F820303C
S31508018000BCE7002384F82030B8E7216B626BE5688A
S31508018010E80E6B015B1B60F10000800040EA93707B
S315080180209B005B1940F10000C00040EA5370DB0079
S31508018030994272EB0003A1D3022384F820309DE70D
S31508018040A37F002B9AD104F12C03009304F1280392
S3150801805004F1240229462046FFF7ACFE98B12946C9
S315080180602046FFF747FF70B9626A29462046FFF79F
S315080180705CFF002882D0032384F8203000220023E5
S31508018080C4E90C237AE7002384F8203076E704F163
S315080180902C03009304F1280304F1240229462046FF
S315080180A0FFF788FE70B129462046FFF723FF48B936
S315080180B0626A29462046FFF738FF38B9022384F851
S315080180C020305BE7002384F8203057E7216B626B89
S315080180D02569E80E6B015B1B60F10000800040EA30
S315080180E093709B005B1940F10000C00040EA537091
S315080180F0DB00994272EB0003FFF440AF002384F8DA
S3150801810020303BE7002384F8203037E7014B036032
S31508018110704700BF102F090810B50446FFF7F6FF90
S31508018120202120464AF0BAF8204610BDC0E90023AE
S315080181309DF8003003729DF8043043729DF80830AB
S3150801814083729DF80C30C3729DF8103003739DF845
S31508018150143043739DF8183083739DF81C30C3732C
S315080181609DF8203003749DF8243043749DF8283017
S3150801817083749DF82C30C3749DF8303003759DF8CF
S31508018180343043759DF8383083759DF83C30C37596
S315080181909DF8403003769DF8443043769DF8483083
S315080181A083769DF84C30C3769DF8503003779DF859
S315080181B0543043779DF8583083779DF85C30C37700
S315080181C09DF8603080F820307047000030B4084AC6
S315080181D002600022027442600121816001734273C8
S315080181E0827300240025C0E9064530BC704700BFEC
S315080181F0102F090804307047007C0238C0B20128E4
S315080182008CBF002001207047087A002831D1487AAE
S3150801821000282ED1887A00282BD1C87A48BB087B3A
S3150801822038BB487B28BB887B18BBC87B08BB087C46
S31508018230F8B9487CE8B9887CD8B9C87CC8B9087D3A
S31508018240B8B9487DA8B9887D98B9C87D88B9087E26
S3150801825078B9487E68B9887E58B9C87E48B9087F12
S3150801826038B9487F28B9887F18B9C87F08B991F8FD
S315080182702000704770B50446037B8BB1437B8BB9ED
S315080182800B684D688669C2699E1945EB02058661C8
S31508018290C561037C032B64D8DFE803F00712303E7F
S315080182A0037470BD02230374FBE7FFF7ADFF0028D3
S315080182B0F7D00123237400220023C4E90623F0E73B
S315080182C0FFF7A2FF10B900232374EAE76168CA0E13
S315080182D04B015B1A62F10002920042EA93729B001B
S315080182E05B1842F10002D20042EA5372DB009E4259
S315080182F075EB0203D5D302232374D2E7837B002BC4
S31508018300CFD1FFF781FF0028CBD1032323740022A5
S315080183100023C4E90623C4E7FFF776FF10B1022359
S315080183202374BEE7A068C20E43011B1A62F100025C
S31508018330520242EAD3525B021B1842F100024FEA8B
S31508018340821C4CEA936C9901CB1A6CEB02021B183E
S3150801835042F100029E4275EB0203A2D30023237465
S315080183609FE7002303749CE7014B0360704700BF36
S31508018370202F090810B50446FFF7F6FF18212046F5
S3150801838049F08CFF204610BD01607047054A02601E
S3150801839000220275427504494160044A8260C1603F
S315080183A002617047202F09089A99193ECDCCCC3D18
S315080183B00430704738B504460D46037DC3B10868D5
S315080183C00368DB689847A16879F08CF808B100233F
S315080183D02375637DC3B1286803681B6998472169BA
S315080183E001F1004179F09CF808B10023637538BDA5
S315080183F008680368DB689847616879F091F800288E
S31508018400E7D001232375E4E7286803681B699847C1
S31508018410E16801F1004179F065F80028E7D0012308
S315080184206375E4E7007D7047407D70470346007D2C
S3150801843000B9587D70470000014B0360704700BFC3
S31508018440302F090810B50446FFF7F6FF30212046FC
S3150801845049F024FF204610BDC0E90023009B836034
S31508018460019BC3609DF808300374704730B40E4A07
S3150801847002600022027780F828200C4941600C49E5
S3150801848081600C49C1604FF47A7101613C214161F7
S315080184900121017642768276C27600240025C0E95A
S315080184A0084530BC704700BF302F09080000484214
S315080184B0000020400000A04004307047007F0238C9
S315080184C0C0B201288CBF00200120704770B506464E
S315080184D00D46886803689B6898470446337E0BB93E
S315080184E000F100440021204679F01AF830B12146FE
S315080184F0E86878F0F7FF10B1012000E0002070BDB0
S3150801850070B505460E46886803689B689847044611
S315080185102B7E0BB900F100440021204679F000F8C2
S3150801852008B32146686878F0DDFF90B1F6680F490F
S31508018530E86878F039FE4FF07E5178F02DFD014656
S31508018540304678F031FE214678F0CCFF60B1012043
S315080185500AE0A968F06878F01FFD214678F0C2FFA5
S3150801856010B1012000E0002070BD00BF0AD7233CEE
S3150801857070B50446437E43B10D46837E4BB1012354
S3150801858080F828300223037702E080F82830037741
S3150801859070BD09686A68036A406A5B1842EB0002A3
S315080185A02362626229462046FFF790FF84F8280075
S315080185B0237F032B72D8DFE803F0021237472B7C9F
S315080185C0002BE5D029462046FFF79AFF0028DFD081
S315080185D00123237700220023C4E90823D8E72B7C4B
S315080185E013B900232377D3E729462046FFF788FFE7
S315080185F00028F6D0216A626A2569E80E6B015B1BC1
S3150801860060F10000800040EA93709B005B1940F11D
S315080186100000C00040EA5370DB00994272EB000388
S31508018620B6D302232377B3E7E37E002BB0D12946DD
S315080186302046FFF765FF0028AAD1032323770022E6
S315080186400023C4E90823A3E729462046FFF758FF74
S3150801865010B1022323779BE7206A616A6669F20EE5
S3150801866073019B1B62F10002520242EAD3525B027A
S315080186709B1942F100024FEA821C4CEA936C9D0158
S31508018680EB1A6CEB02029B1942F10002984271EB5C
S315080186900203FFF47DAF0023237779E700232377CD
S315080186A076E7C0E90023009B8360019BC360029BB8
S315080186B00361039B4361049B8361059BC361704707
S315080186C030B5A9B084460023C0F8AC30604A0260D0
S315080186D04360604A6B4607CA03C31A800023042B0A
S315080186E009DC28AA02EB430232F9A01C1A1D2CF850
S315080186F012100133F3E703AB574A07CA03C31A80BB
S315080187000023042B10DC28AA02EB430232F9941C3D
S3150801871003F108020CEB4202518003F124020CEB2F
S315080187204202D1800133ECE70DF16C0E4B4C0FCCB4
S31508018730AEE80F000FCCAEE80F000FCCAEE80F0085
S315080187402368AEF8003000210FE001EB81031344E2
S3150801875028A800EB430030F9340C0C330CEB430327
S3150801876098800132042AF0DD0131042901DC002256
S31508018770F8E706AB3A4A07CA03C31A800023042B53
S315080187800ADC28AA02EB430232F9881C03F12C02FF
S315080187902CF812100133F2E72E4C09AD04F15803F7
S315080187A00FCB07C52B800DAD04F168030FCB07C5A9
S315080187B02B800023062B11DC28AA02EB430131F991
S315080187C07C0C03F130020CEB4202508031F96C1C2F
S315080187D003F138022CF812100133EBE71D4C0DF1A9
S315080187E0440E04F178050FCDAEE80F002B68CEF8DC
S315080187F000300DF1580E8C340FCCAEE80F0023680B
S31508018800CEF800300023092B12DC28AA02EB43011B
S3150801881031F95C0C03F13C020CEB4202D08031F9D0
S31508018820481C03F148020CEB420251800133EAE786
S3150801883001238CF8A63000238CF8A7308CF8A830D1
S315080188408CF8A9308CF8AA30604629B030BD00BF33
S31508018850CDCC0C40382F0908442F0908502F090898
S31508018860842F090870477047D0F8AC0070472DE986
S31508018870F0410546069C04F10040013832F910C062
S31508018880B2F90060B44543DDAE4204DAAC4506DD13
S315080188904FF0000C08E0B3F90000BDE8F08133F9A8
S315080188A01000FAE70CF1010C601E60456ADD4FEA1B
S315080188B04C0E32F91C60AE42F4DC0CF101004FEAB1
S315080188C0400832F91070AF42ECDB33F9080033F98E
S315080188D00E80A0EB080078F013FC0446B81B78F06C
S315080188E00FFC0146204678F013FD0446A81B78F0D4
S315080188F007FC214678F058FC0446404678F000FC0F
S315080189000146204678F048FB78F02AFE00B2C4E713
S31508018910AE4204DDAC4505DA04F1FF3C07E0B3F9E4
S315080189200000BAE733F91000B7E70CF1FF3CBCF1D8
S31508018930000F29DD4FEA4C0032F91C60AE42F4DC27
S315080189400CF10044013C670032F91440AC42ECDBFF
S31508018950DA5F1F5ED01BA41B90FBF4F078F0D0FB06
S315080189600446A81B78F0CCFB214678F01DFC04468A
S31508018970384678F0C5FB214678F00EFB78F0F0FD15
S3150801898000B28AE7084688E7084686E72DE9F04FE8
S315080189908BB005460391144622F000464E493046EF
S315080189A078F0C8FD002840F095804B49304678F0AC
S315080189B0B7FD002840F08E80B5F9120078F0A0FBCB
S315080189C00646214678F0ACFD48B9B5F91A0078F0A3
S315080189D097FB0646214678F085FD00B92646002410
S315080189E007940894ADF8244000E00134032C5DDCBB
S315080189F004F1080305EB4303B3F90270384678F02E
S31508018A007FFB8146314678F077FD0028EDD004F1E9
S31508018A10010A04F1090305EB4303B3F90280404651
S31508018A2078F06EFB314678F071FD0028DDD0CDF87F
S31508018A3010904FF000090596B9F1040F36DC0AEBE0
S31508018A408A034B440C3305EB4303B3F9040004EBE7
S31508018A5084034B440C3305EB4303B3F904B0A0EB91
S31508018A600B0078F04DFB0646A8EB070078F048FBAB
S31508018A700146304678F04CFC06460499059878F08C
S31508018A8089FA314678F090FB0646584678F038FB65
S31508018A900146304678F080FA0AAB03EB490678F0CE
S31508018AA05FFD26F80C0C09F10109C5E7083503989D
S31508018AB078F056FD0523009307AB2A46642100B2D8
S31508018AC0FFF7D5FE78F01CFB044978F021FC0BB0C2
S31508018AD0BDE8F08F0020F7E7FFFF7F7F0000C8425F
S31508018AE030B583B000F17E0500F19204084678F0AE
S31508018AF037FD0A23009323462A46642100B2FFF76D
S31508018B00B6FE78F0FDFA024978F002FC03B030BDF2
S31508018B100000C8422DE9F04383B0044690F8AA3014
S31508018B20002B00F098800E46056890F8A630B3B180
S31508018B30CF680A693946FFF729FF804672693946BF
S31508018B402046FFF723FF07460146404678F0E8FC32
S31508018B5000B947463946284678F026FB054694F873
S31508018B60A73043B3D6F8188028F000475D49384640
S31508018B7078F0E0FC002874D15A49384678F0D0FCE0
S31508018B8000286ED104F14E0704F15809404678F0E1
S31508018B90E7FC052300934B463A46642100B2FFF7EA
S31508018BA066FE78F0ADFA504978F0B2FB01462846E0
S31508018BB078F0FAFA054694F8A8305BB3D6F81C8023
S31508018BC028F000474749384678F0B4FC00284AD1CE
S31508018BD04449384678F0A4FC002844D14349404624
S31508018BE078F0E2FA04F1620704F1700878F0B8FC4B
S31508018BF00723009343463A46642100B2FFF737FE3E
S31508018C0078F07EFA384978F083FB0146284678F0F1
S31508018C10CBFA054694F8A930A3B131692046FFF786
S31508018C205FFF804671692046FFF75AFF07460146EE
S31508018C30404678F075FC00B947463946284678F02B
S31508018C40B3FA054667680021384678F041FC60B1F9
S31508018C50C4F8AC5002E00023C0F8AC3003B0BDE85C
S31508018C60F08300209FE70020CCE7D6F80890294634
S31508018C70484678F041FC002830D04FF07E584146EE
S31508018C80384678F091FA0746D6E9000178F046FAAF
S31508018C90394678F089FA164978F03AFB014648468A
S31508018CA078F07AF90646C4F8AC000021404678F017
S31508018CB037FC20B12946304678F032FC58B90021F4
S31508018CC0404678F00FFC0028C8D02946304678F08F
S31508018CD009FC0028C2D0C4F8AC50BFE7DFF81480FD
S31508018CE0CDE700BFFFFF7F7F0000C84200007A443E
S31508018CF000247449000080BF014B0360704700BF20
S31508018D00E02F090810B50446FFF7F6FF282120468B
S31508018D1049F0C4FA204610BDC0E90023009B8360D0
S31508018D20019BC3607047000030B40E4A02600022FE
S31508018D3002770D4941604FF07C5181604FF07A51BD
S31508018D40C1604FF47A7101613C21416102760121CA
S31508018D5041768276C27600240025C0E9084530BCF2
S31508018D60704700BFE02F09080000904004307047A3
S31508018D70007F0238C0B201288CBF0020012070474D
S31508018D802DE9F04104460D468E6847683946304656
S31508018D9078F0BCFB30B9A168304678F0ADFBA8B1D4
S31508018DA0012600E0012694F81880B8F1000F10D0CA
S31508018DB07EB9ED682946384678F09EFB40B9A16828
S31508018DC0284678F099FB20B1464602E00026EAE7F4
S31508018DD046463046BDE8F0812DE9F04104460E4687
S31508018DE08F68D0F80C804146406878F0D3F805467C
S31508018DF00146384678F076FB50B1A168404678F0CE
S31508018E00CBF80146384678F08BFBB0B9002700E06D
S31508018E100027237EA3B197B1F6683146284678F034
S31508018E207FFB80B1A168404678F0B6F80146304626
S31508018E3078F076FB20B9002702E00127E9E7002749
S31508018E403846BDE8F0810027FAE770B50446437E47
S31508018E508BB1837E8BB90B684D68066A426A9E1987
S31508018E6045EB020506624562037F032B64D8DFE8FA
S31508018E7003F00712303E037770BD02230377FBE741
S31508018E80FFF77EFF0028F7D001232377002200236E
S31508018E90C4E90823F0E7FFF773FF10B90023237726
S31508018EA0EAE72169CA0E4B015B1A62F100029200D8
S31508018EB042EA93729B005B1842F10002D20042EA31
S31508018EC05372DB009E4275EB0203D5D30223237747
S31508018ED0D2E7C37E002BCFD1FFF77EFF0028CBD088
S31508018EE00323237700220023C4E90823C4E7FFF7F5
S31508018EF073FF10B902232377BEE76069C20E4301E7
S31508018F001B1A62F10002520242EAD3525B021B1893
S31508018F1042F100024FEA821C4CEA936C9901CB1A82
S31508018F206CEB02021B1842F100029E4275EB02032A
S31508018F30A2D3002323779FE7002303779CE700004A
S31508018F40024A0260024A0260704700BF08300908F7
S31508018F50802E0908F8B504460D464169284678F079
S31508018F6019F8064667682946384678F01DF9606299
S31508018F703146384678F018F9216978F0C9F9E16877
S31508018F8078F012F9054620F00041A06878F0C8FA91
S31508018F9010BB637E0BB3237E9BB14FF00106002104
S31508018FA0284678F09FFA08B94FF00006F6B294F809
S31508018FB0202092B18EB1E169284678F0F5F8054688
S31508018FC00BE04FF001060021284678F0A9FA08B906
S31508018FD04FF00006F6B2EAE700252846F8BD406AD2
S31508018FE070470000024A0260024A0260704700BFE9
S31508018FF0F02F0908802E09088068704710B50446C5
S31508019000FFF79EFF2821204649F048F9204610BD62
S3150801901010B50446FFF7E6FF0C21204649F03EF954
S31508019020204610BD0C4A02600C4A026000224262C8
S315080190304FF07E5141608260DFF824C0C0F80CC051
S31508019040DFF820C0C0F810C04261002202764276DD
S31508019050C16180F820207047802E09080830090868
S31508019060000070410000203F0430704738B50546BE
S315080190700C464068FFF7F8FF04616868FFF7F4FFDC
S315080190802146006878F090F8A860204638BD0000AF
S31508019090034A0260034A0260416000228260704707
S315080190A0802E0908F02F0908024A0260024A026066
S315080190B0704700BF40300908203009080069704729
S315080190C040697047806970470B4621B9023300EB46
S315080190D08300406870470020704710B50446FFF7C3
S315080190E0E3FF2421204649F0D9F8204610BD016046
S315080190F042608360009BC360019B03617047000067
S315080191000C4B03600C4B03600023036143618361CD
S31508019110C361036243600123038100238372002B29
S3150801912006DC9A1C00EB8202002151600133F6E746
S31508019130704700BF203009084030090804307047DD
S315080191402DE9F04104460D46867A731E042B00F27A
S31508019150C080DFE803F0031C411C79008968686850
S3150801916077F01AFF296877F015FF0023002B05DC35
S315080191709A1C04EB820250600133F7E7A061606133
S3150801918020616B68E361AB682362BDE8F0814F68D3
S3150801919027F00041406878F0AFF910B9022E0DD0DA
S315080191A0EF682968384677F0F5FE0023002B07DCBF
S315080191B09A1C04EB820250600133F7E7AF68F0E7C7
S315080191C0A061606120616B68E361022E02D0EB68E1
S315080191D02362DAE7AB68FBE70023002B06DC696844
S315080191E09A1C04EB820251600133F6E72289134681
S315080191F0B3EB420F06DAA868991C04EB81014860B3
S315080192000133F5E7A968686877F0C6FE4FF07C5127
S3150801921077F0CAFF20616F68AE683146384678F044
S3150801922075F968B167616F68AE683146384678F096
S3150801923063F938B1A7616B68E361AB682362A4E798
S315080192406661F0E7A661F6E7D1F80C804E6826F06C
S3150801925000414768384678F04FF900B94646002379
S31508019260002B05DC9A1C04EB820256600133F7E7F2
S31508019270D5F81080AD6825F00041384678F03CF9FC
S3150801928000B9454622891346B3EB420F05DA991C04
S3150801929004EB81014D600133F6E72946304677F044
S315080192A07BFE4FF07C5177F07FFF206129463046DF
S315080192B078F02CF948B166612946304678F01CF9F0
S315080192C028B1A661E66125625FE76561F4E7A561F4
S315080192D0F8E70968686877F05DFE03460022002A08
S315080192E005DC911C04EB81014B600132F7E7A361B0
S315080192F0636123616B68E3610023236245E700002C
S31508019300014B0360704700BF6030090810B5044679
S31508019310FFF7F6FF1421204648F0C0FF204610BD8E
S315080193200160027170470000054A026000228260EE
S31508019330C260002202744274024A4260704700BF4A
S31508019340603009080000A04204307047816000239C
S3150801935003744374704738B504460B46027C22B140
S31508019360012A0CD00023037438BD0A79002AFBD0E0
S315080193700B68C3600023437401230374F4E70A7975
S31508019380002AF1D1C168186877F004FE0546002164
S3150801939078F0C6F850B16168284677F0B9FF0146FA
S315080193A0A06877F0F9FDA060012363740023237494
S315080193B0DAE7806870470000014B0360704700BF19
S315080193C0D030090810B50446FFF7F6FF6821204694
S315080193D048F064FF204610BDC0E90023DDE90023FB
S315080193E0C0E90223029B0361039B4361049B8361DA
S315080193F0059BC361069B0362079B4362089B8362C5
S315080194009DF8243080F82C309DF8283080F82D30CE
S315080194109DF82C3080F82E309DF8303080F82F30AA
S315080194209DF8343080F830307047000030B41A4A5D
S31508019430026000240025C0E90E45C0E91045002256
S3150801944080F8502080F8512080F85220002141658B
S3150801945080F85820A0F85A20C1654FF0FF310166FF
S315080194604166032181800D4981600D49C1600D491D
S3150801947001610D4941611E2101764FF47A71C1617D
S3150801948080F82020094941623C21816280F82C201C
S31508019490C0E90C4530BC7047D0300908000060406F
S315080194A00AD7A33C000096439A993940CDCCCC3DC6
S315080194B00430704790F85000704700F14001D1E937
S315080194C00001704790F95100704790F852007047B3
S315080194D0406D704790F858007047C06D7047006E30
S315080194E07047406E7047B0F85A00704710B582B0A1
S315080194F00C4601A81BF09AFE284920466CF0E6FDA9
S31508019500002844D0044603460522012124486DF06B
S31508019510D9FC23460622012122486DF0D3FC2346B5
S315080195200422012120486DF0CDFC23460B2201219E
S315080195301E486DF0C7FC2346092201211C486DF01F
S31508019540C1FC2346082201211A486DF0BBFC2346BB
S315080195500B22012118486DF0B5FC23460922012189
S3150801956016486DF0AFFC23460822012114486DF018
S31508019570A9FC23460222012112486DF0A3FC2046CC
S315080195806CF034FB01A81BF0CDFE02B010BD01A89A
S315080195901BF09EFD01A81BF0C5FEF6E70464090849
S315080195A0202E090868300908282E0908703009088C
S315080195B07C3009088830090894300908A030090860
S315080195C0AC300908A4E20B08F0B58FB007460C4683
S315080195D015460DA81BF02AFE364920466CF076FD85
S315080195E000285FD0044604A905F108006DF0B0FC17
S315080195F0049B0393059B0293069B0193099B03F224
S315080196006C730093089B0133079A2B49204646F051
S31508019610F0FB2A4EB7F85A203146204646F0E9FBB8
S31508019620286977F013F902460B462549204646F084
S31508019630E0FB686977F00AF902460B46214F39467D
S31508019640204646F0D6FBEA6901323146204646F005
S31508019650D0FB2A6A01323146204646F0CAFBA86980
S3150801966077F0F4F802460B463946204646F0C1FB28
S315080196706A6A01323146204646F0BBFBAA6A0132C4
S315080196803146204646F0B5FB2346022201210E4803
S315080196906DF018FC20466CF0A9FA0DA81BF042FEE5
S315080196A00FB0F0BD0DA81BF013FD0DA81BF03AFE77
S315080196B0F6E700BF34430B08CC2D0908F42D090839
S315080196C0EC2D0908F82D0908A4E20B08F8B504469B
S315080196D090F82C301BB30D4690F8501051B105295E
S315080196E008D0AB68EA68806B1B1AE06B62EB000274
S315080196F0236462642A68206B636B1218686840EBFE
S31508019700030322636363062900F28881DFE811F007
S3150801971022005400B500D7004701750175010020E4
S315080197200021C4E90C0184F85030FF2284F8512045
S3150801973084F852300022626584F85830C4E90E0173
S31508019740C4E91001A4F85A30E2654FF0FF332366E5
S315080197506366F8BD002384F8513084F8523000223C
S31508019760626584F8583095F83030002BF1D095F8B9
S315080197702E30002BEDD1D5E90223C4E91223C4E921
S315080197800E2300220023C4E91023012384F8503054
S315080197900023A4F85A300023E3654FF0FF3323660C
S315080197A06366A04E31462046FFF7A0FE2A4631469B
S315080197B02046FFF709FFCCE795F830301BB902239D
S315080197C084F85030C5E7012384F8513084F85230C3
S315080197D000236365002384F85830B4F85A20A38817
S315080197E09A4208D395F82C20237E9A42B1D30523B1
S315080197F084F85030ADE76969A86977F0CBFB20F0AA
S315080198000041606A77F08CFE18B1D5E90223C4E9F4
S315080198101223AB68EA68A16CE06C5B1A62EB000282
S31508019820A16A8B4272F100031EDA6F69A668314696
S31508019830384677F06BFE00288BD0AD69294630464D
S3150801984077F05AFE002884D03946284677F0A2FBDD
S3150801985020F00041E06877F059FE00283FF479AF1F
S31508019860022384F8503074E72A466E492046FFF7EA
S31508019870ABFE062384F850306BE7012384F8513098
S31508019880002384F852300022626584F8583095F82E
S315080198902D30002B7FF45DAF95F830305BB1D5E9FB
S315080198A00223C4E91223032384F85030002200233B
S315080198B0C4E90C234DE7002384F8503049E795F8AD
S315080198C0301019B9042384F8503042E7002184F88E
S315080198D0511084F8521094F8581049B9002161655D
S315080198E095F82F10002939D100220023C4E90C2349
S315080198F094F858306BB12369636595F82F3043B9ED
S3150801990000236365002384F8583000220023C4E944
S315080199100C236969A86977F03DFB20F00041606A6C
S3150801992077F0FEFD18B1D5E90223C4E91223AB6825
S31508019930EA68A16CE06C5B1A62EB0002A16A8B42D1
S3150801994072F1000322DA6169686977F0D5FD0028AA
S315080199503FF4FFAE042384F85030FAE6E669F00EC8
S315080199607101891B60F10000800040EA917089004D
S31508019970891940F10000C00040EA5170C9008A42C5
S315080199808341B5D3012384F85830B1E72A462549DE
S315080199902046FFF719FE062384F85030D9E600233E
S315080199A084F8513084F852300022626584F85830C0
S315080199B095F82E30002B7FF4CCAE95F830301BB9D4
S315080199C0002384F85030C4E6B4F85A300133A4F8B9
S315080199D05A302A4613492046FFF7F6FD2E69E16DEE
S315080199E0304677F093FD20B1E665EB6923662B6A6D
S315080199F06366012384F85030ABE6002384F85130BE
S31508019A0084F852300022626584F8583095F830306F
S31508019A10002B7FF49EAE84F850309AE6002384F832
S31508019A20503096E6B8300908014B0360704700BF0D
S31508019A30E030090810B50446FFF7F6FF2C21204649
S31508019A4048F02CFC204610BD0160426083609DF8F9
S31508019A5000300373019B0361029B43617047000059
S31508019A600D4A0260002280F8282001210171142183
S31508019A70417119218171C271084981600849C16022
S31508019A80027408494161084981610849C161026254
S31508019A9080F82420704700BFE030090800004040E4
S31508019AA06666464000002842000070421304010021
S31508019AB00430704790F82800012814BF00200120BF
S31508019AC070472DE9F04104460D4616460B7B002BDF
S31508019AD032D10127237953B1002E2FD0A07977F0FF
S31508019AE00BFB0146286877F0FDFC00B10027E379F6
S31508019AF033B146B3E168A86877F0F4FC00B10027F2
S31508019B00237C33B3606906B34FF07E58414677F03C
S31508019B1043FA06464146A06977F03CFA04466D6861
S31508019B203146284677F0DEFC90B92146284677F07B
S31508019B30F7FC70B100270CE00027CBE7607977F0D6
S31508019B40DBFA0146CEE7A168D5E74FF00008DDE765
S31508019B5000273846BDE8F081C2690B691A4205D16A
S31508019B60026A4B691A4203D00120704701207047E7
S31508019B70002070472DE9F04104460D460F7B067912
S31508019B8056B1D1F80080407977F0BAFA01464046D5
S31508019B9077F0B2FC00B13746E6792EB1A168A8681C
S31508019BA077F0AAFC00B13746267C6EB16D6861690B
S31508019BB0284677F0A1FC30B9A169284677F0A6FCBA
S31508019BC010B1374600E037463846BDE8F08138B56A
S31508019BD0044690F824305BB10D4690F82830012BE5
S31508019BE018D0022B23D033B1002380F8283001E0A6
S31508019BF080F8283038BD0022FFF763FF0028F9D026
S31508019C0029462046FFF7A8FF0028F3D1012384F847
S31508019C102830EFE7FFF7AEFF28B929462046FFF7B8
S31508019C209BFF0028E6D0022384F82830E2E70122C8
S31508019C30FFF747FF0028DDD029462046FFF78CFFAE
S31508019C400028D7D1012384F82830D3E7014B0360D4
S31508019C50704700BFF030090810B50446FFF7F6FF54
S31508019C608021204648F01AFB204610BDC0E9002392
S31508019C70BDF800300381BDF8043043819DF90830F1
S31508019C8003739DF90C3043739DF9103083739DF866
S31508019C901430C3739DF8183003749DF81C3043744F
S31508019CA09DF82030C3749DF8243003759DF828303B
S31508019CB043759DF82C3083759DF83030C3759DF832
S31508019CC0343003769DF8383043769DF83C308376F8
S31508019CD0109BC361119B03627047000030B4224A8E
S31508019CE00260002280F8602080F8702080F87120D8
S31508019CF080F8722080F87320426780F87820012165
S31508019D00017141714FF47A748460C46002744274BB
S31508019D1042618261C261026242628262C262026316
S31508019D2042638263C2630264426480F84820A0F8F1
S31508019D304A2080F84C2080F84D1080F84E2080F893
S31508019D404F2080F8502080F85120084C4465084C73
S31508019D50846580F85C2080F85D1000240025C0E940
S31508019D601A4530BC704700BFF03009081B04410092
S31508019D70100002000430704790F86000B0FA80F0D5
S31508019D804009704790F87300704790F860000338EF
S31508019D90C0B201288CBF00200120704790F86000EE
S31508019DA0042814BF00200120704790F86000052898
S31508019DB014BF00200120704790F87000704790F892
S31508019DC07100704790F87200704790F878007047F4
S31508019DD04379022B01D00020704790F85C300BB113
S31508019DE08B7E3BB191F90D30002B01DD01207047C7
S31508019DF000207047002070474379022B01D00020CC
S31508019E007047487E7047034690F85C200AB1887E01
S31508019E1000E001205B7923B1012B03D0022B0AD084
S31508019E200020704728B191F90C30002BF9DD00208C
S31508019E3070470020704728B191F90E30002BF0DCED
S31508019E4000207047002070470346487E90B99888DD
S31508019E5040F2011290420ED093F84E200AB1C87C06
S31508019E6040B993F850200AB1087D18B993F8510002
S31508019E7000B1487D7047487C0028EDD0FAE710B458
S31508019E80024690F84E0088B1536DC869034003F441
S31508019E900054C3F3403092F84F303BB191F90C00AE
S31508019EA0002802DD7CB9002000E00020CB6923F4FC
S31508019EB00053546D1C4208D140B9926D0B6A1A427F
S31508019EC004D0012002E01846F0E7012010BC7047D3
S31508019ED070B40346144612B1027C002A7BD1D868B5
S31508019EE0002C79D05A7C002A76D05C6DCA6922404A
S31508019EF012F0020F03D05C69844200D8204612F0A2
S31508019F00040F03D09C69844200D8204612F0010F41
S31508019F1003D0DC69844200D8204612F0080F03D02A
S31508019F201C6A844200D8204612F0100F03D05C6ADE
S31508019F30844200D8204693F84E408CB102F400566C
S31508019F40C2F3403593F84F402CB191F90C40002CDF
S31508019F5006DD0EB904E01DB19C6A844200D820468C
S31508019F6093F8504034B112F4004F03D0DC6A8442AE
S31508019F7000D8204693F8514034B112F0005F03D05F
S31508019F801C6B844200D8204612F4803F03D05C6BD8
S31508019F90844200D8204612F4003F03D09C6B8442C9
S31508019FA000D820469C6D096A0C4014F0100F03D0A6
S31508019FB0D96B814200D8084612F4800F03D0196C78
S31508019FC0814200D8084612F4806F05D05B6C834243
S31508019FD002D8184600E0002070BC70472DE9F84306
S31508019FE0044690F85D30EBB10D460B684968876EFB
S31508019FF0C26EDF1941EB02088766C0F86C802946F4
S3150801A000FFF73DFF064684F8720094F86030052B89
S3150801A01000F2D381DFE813F00E004900C200FD000B
S3150801A0204201AB0180F8733080F8783080F86030EF
S3150801A030BDE8F883002384F8733029462046FFF7E4
S3150801A040C7FE20B129462046FFF7D6FE48B1294664
S3150801A0502046FFF7D8FEB0B129462046FFF7F4FEA1
S3150801A06088B986B9012384F87830EB7B002BDFD0D9
S3150801A07094F84C308BB194F84D3043B194F8713063
S3150801A080002BD5D106E0002384F87830D0E70023E9
S3150801A09084F87130012384F87030012384F8603024
S3150801A0A000220023C4E91A23C2E7002384F8733087
S3150801A0B029462046FFF78CFE814620B129462046CF
S3150801A0C0FFF79AFE48B129462046FFF79CFE68B37A
S3150801A0D029462046FFF7B8FE40BB3EBBA168CA0E1B
S3150801A0E04B015B1A62F10002920042EA93729B00ED
S3150801A0F05B1842F10002D20042EA5372DB009F422A
S3150801A10078EB020394D394F84C3053B32B89D3B12B
S3150801A1106A89C2B19B1A002BB8BF5B42B4F84A20C0
S3150801A120934210DC022384F8603081E794F84C30BE
S3150801A1302BB1002384F87030012384F87130002391
S3150801A14084F8603074E7002384F87030012384F8BA
S3150801A1507130052384F8603000220023C4E91A23EC
S3150801A16066E794F84830ABB1B9F1000F04D0294637
S3150801A1702046FFF741FE48B129462046FFF743FE30
S3150801A18040B129462046FFF75FFE18B9022384F835
S3150801A19060304DE7032384F8603049E7012384F8EA
S3150801A1A0733029462046FFF713FE20B1294620467B
S3150801A1B0FFF722FE48B129462046FFF724FED8B10B
S3150801A1C029462046FFF740FEB0B9AEB92B7C002BD5
S3150801A1D03FF42EAF29462046FFF715FE00283FF427
S3150801A1E027AF29462046FFF72FFE00287FF420AF28
S3150801A1F0032384F860301BE794F84C302BB1002315
S3150801A20084F87030012384F87130002384F86030B3
S3150801A2100EE794F848705FB129462046FFF7D8FD46
S3150801A220074628B129462046FFF7E6FD00B1002773
S3150801A23084F87370237C6BB166B194F84C302BB1FA
S3150801A240002384F87030012384F87130002384F8E0
S3150801A2506030EDE694F84C7027B16A89B4F84A3053
S3150801A2609A420CD929462046FFF7CDFD38B1294631
S3150801A2702046FFF7E9FD10B9002E3FF4D9AE2FB1FC
S3150801A280002384F87030012384F87130042384F89C
S3150801A290603000220023C4E91A23C9E6002384F8A2
S3150801A2A0733094F84C3053B929462046FFF7ABFD75
S3150801A2B028B129462046FFF7C7FD00B906B332463D
S3150801A2C029462046FFF704FE86B294F85130DBB9D9
S3150801A2D073019B1B62EB0202920042EA93729B0096
S3150801A2E09B1942F10002D20042EA5372DB009F42F7
S3150801A2F078EB0203FFF49CAE002384F8603097E6FE
S3150801A300032384F8603093E6636F0BBB95F81890C6
S3150801A310B9F1000F1CD02B4B03FB09F3FB1848F1CD
S3150801A3200001E2684FF47A7C0CFB02F2934271F168
S3150801A330000319D24FF47A7200233846414677F062
S3150801A340A5F94FF47A7303FB090303F57A73636777
S3150801A350636F03B19EB2EB7D13B9AB7D002BB7D00A
S3150801A360002384F8603063E680B26067F0E7002373
S3150801A37084F8733094F84D30002B7FF459AE0246B9
S3150801A38029462046FFF7A4FD80B243011B1A62EB5A
S3150801A3900202920042EA93729B001B1842F10002E4
S3150801A3A0D20042EA5372DB009F4278EB0203FFF4C4
S3150801A3B03FAE002384F860303AE6002384F8603023
S3150801A3C036E600BF40420F0010B504461B4B40F865
S3150801A3D0683B00F0D9FB04F1600000F0D5FB04F1FD
S3150801A3E0580000F0D1FB04F1500000F0CDFB04F158
S3150801A3F0480000F0C9FB04F1400000F0C5FB04F178
S3150801A400380000F0C1FB04F1300000F0BDFB04F197
S3150801A410280000F0B9FB04F1200000F0B5FB04F1B7
S3150801A420180000F0B1FB04F1100000F0ADFB04F1D7
S3150801A430080000F0A9FB204610BD00BF003109083D
S3150801A44010B50446FFF7C0FF8021204647F026FFD6
S3150801A450204610BDC0E90023009B8360019BC360B1
S3150801A4609DF8083003749DF80C3043749DF910303B
S3150801A47083749DF91430C3747047000038B50446D7
S3150801A480264B40F8083B0025294600F079FB29466A
S3150801A49004F1100000F074FB294604F1180000F0DD
S3150801A4A06FFB294604F1200000F06AFB294604F1F6
S3150801A4B0280000F065FB294604F1300000F060FB36
S3150801A4C0294604F1380000F05BFB294604F14000F7
S3150801A4D000F056FB294604F1480000F051FB2946D5
S3150801A4E004F1500000F04CFB294604F1580000F035
S3150801A4F047FB294604F1600000F042FB294604F1B6
S3150801A500680000F03DFBA567002384F87C302371C1
S3150801A51000220023C4E91C23204638BD003109085E
S3150801A52004307047F0B589B0044617461E466D4695
S3150801A530284600F025FB04F1500395E8030083E85B
S3150801A5400300284600F020FB02AD3946284600F0F4
S3150801A55017FB04F1580395E8030083E8030028462E
S3150801A56000F012FB04AD3146284600F009FB04F160
S3150801A570600395E8030083E80300284600F004FB1E
S3150801A58006AD0E99284600F0FBFA04F1680395E832
S3150801A590030083E80300284600F0F6FA00220023A8
S3150801A5A0C4E91C2309B0F0BD2DE9F04F87B08046F8
S3150801A5B08946D1E9000176F0B1FD814976F0A8FE18
S3150801A5C00090002102A800F0DBFA4FF0000A5EE0D5
S3150801A5D0002769E05146D9F80C0004F0B3FD83461B
S3150801A5E0002531E0002437E0314604A800F0C8FA16
S3150801A5F0314604A800F0B2FBF9694FF07E5076F0B7
S3150801A60087FE014604A800F0A9FB009904A800F0FA
S3150801A610A5FB6C4904A800F0A1FB08F1680404A88D
S3150801A62000F0B5FA0146204600F0FEFA04A800F04B
S3150801A630B4FA04A800F0ABFA0146204600F0F4FA91
S3150801A64004A800F0A1FA0135112D1BDCCAD805EBC7
S3150801A6504504640020343C44204605F030FA0028BD
S3150801A660F1D02946584604F0AFFB04F071FB0646C3
S3150801A670014602A800F0D8FA204605F060FA00283B
S3150801A680E1D0B1E7019848F0DBF80AF1010ABAF11D
S3150801A690000F17DCD9F80C0004F0D3FBBAF1000F50
S3150801A6A096D1B02707FB0A0707F18C0401942046C7
S3150801A6B048F076F83B7813F0040F8BD1204648F022
S3150801A6C0BFF8E2E799F810301BB999F81130002B59
S3150801A6D048D002A800F058FA99F810305BBB99F8EF
S3150801A6E0113043BBD9F8080003689B68984720F0E6
S3150801A6F0004104A800F044FA009904A800F02EFBD2
S3150801A700D9F8080003689B689847002176F008FF86
S3150801A710A8B304A800F03BFA014608F1100000F0BE
S3150801A72083FA98F804301BB199F91230002B2FDD02
S3150801A73004A800F029FAD9F80000D9F80410D8F8C5
S3150801A7407030D8F87420C01841EB0201C8F87000BF
S3150801A750C8F874101C4B984271F1000336D207B041
S3150801A760BDE8F08F009902A800F0F8FA02A800F0F7
S3150801A7700EFA014608F1080000F056FAA9E704A8FE
S3150801A78000F005FA014608F1180000F04DFAC8E78D
S3150801A79099F91330002BCBDCD9F8080003689B68BC
S3150801A7A09847002176F0BCFE0028C1D004A800F025
S3150801A7B0EEF9014608F1200000F036FAB8E700BFC5
S3150801A7C000247449B4A291390087930376F0A6FC54
S3150801A7D0584976F09DFD074600220023C8E91C2347
S3150801A7E008F1080A01464FF07E5076F091FD814640
S3150801A7F00146504600F0B2FA08F1100549462846C6
S3150801A80000F0ACFA08F118044946204600F0A6FA09
S3150801A81008F120064946304600F0A0FA284600F01D
S3150801A820B4F98146204600F0B0F90146484676F06B
S3150801A830B1FBC8F878003946284600F08FFADFF8E8
S3150801A840F8904946284600F089FA3946204600F02C
S3150801A85085FA4946204600F081FA3946304600F025
S3150801A8607DFA4946304600F079FA284600F08FF914
S3150801A870014608F1280000F0D7F9204600F087F9CB
S3150801A880014608F1300000F0CFF9504600F07FF993
S3150801A8900146284600F062FA504600F078F901466A
S3150801A8A0204600F05BFA504600F071F90146304641
S3150801A8B000F054FA284600F06AF9014608F1380012
S3150801A8C000F0B2F9204600F062F9014608F14000AD
S3150801A8D000F0AAF9304600F05AF9014608F1480095
S3150801A8E000F0A2F9284600F052F9014608F1500095
S3150801A8F000F09AF9204600F04AF9014608F1580095
S3150801A90000F092F9304600F042F9014608F160007C
S3150801A91000F08AF9504600F040F9284600F03DF962
S3150801A920204600F03AF9304600F037F9012388F855
S3150801A9307C3014E700247449B4A2913908B528304B
S3150801A94000F025F908BD08B5303000F020F908BD3A
S3150801A95008B5383000F01BF908BD08B5403000F0DD
S3150801A96016F908BD08B5503000F011F908BD08B54B
S3150801A970583000F00CF908BD08B5683000F007F941
S3150801A98008BD90F87C007047002380F87C3070473A
S3150801A990014B0360704700BF1031090810B5044622
S3150801A9A0FFF7F6FF2821204647F078FC204610BD20
S3150801A9B0C0E90023DDE90023C0E902239DF8083038
S3150801A9C003749DF80C30437470474269C06910449A
S3150801A9D07047C0697047016000224260704730B510
S3150801A9E083B004464160DDE90601C4E902016D460A
S3150801A9F011462846FFF7EFFF04F1140395E8030013
S3150801AA0083E803000023E3612362237403B030BDA6
S3150801AA1010B582B00446064B036000220023CDE937
S3150801AA2000231146FFF7DBFF204602B010BD00BF29
S3150801AA301031090830B40E4BA3FB012C4FEA9C4494
S3150801AA40026802EB9C4202600A4D05FB1411446838
S3150801AA5021444160A3FB0143074CA14205D99B0C44
S3150801AA601A44026005FB1311416030BC704700BFF0
S3150801AA7083DE1B4340420F003F420F0010B40C68AF
S3150801AA8003681C4404604B68426813444360074AE0
S3150801AA90A2FB031206498B4206D9920C14440460A0
S3150801AAA0013101FB1233436010BC704783DE1B433F
S3150801AAB03F420F00F8B504460E4600231370037C87
S3150801AAC0012B0CD0022B2FD003B1F8BD0B7C002B28
S3150801AAD0FBD001230374436801334360F5E7154648
S3150801AAE04B7C43B14368013B43600023C361036266
S3150801AAF002230374E9E700F11C0789683846FFF762
S3150801AB0099FF337C002BE0D1394604F11400FFF795
S3150801AB10B5FF0021E1612162D6E90023C4E90223D8
S3150801AB2001232B702174D0E70B7C002BCDD1037444
S3150801AB30CBE70000024A0260024A0260704700BF82
S3150801AB40383109082031090808467047704710B599
S3150801AB500446FFF7EFFF0421204647F09FFB2046F6
S3150801AB6010BD0000024A0260024A0260704700BF37
S3150801AB70203109083831090800220260426070470D
S3150801AB80016000224260704770470068704708B547
S3150801AB90FFF7FBFF08BD4068704743680360002361
S3150801ABA04360704710B504460021006876F090FCB2
S3150801ABB030B10021606876F08BFC10B1012000E00D
S3150801ABC0002010BD2DE9F0470C46164698469DF81B
S3150801ABD020901146204676F0DFF90546214676F0A3
S3150801ABE0D9F907460146284676F0D4F98246394608
S3150801ABF0304676F0CFF906465146204676F0CAF930
S3150801AC000146304676F0C8F90146B9F1000F04D07D
S3150801AC10C8F800002846BDE8F087D8F8000076F0A5
S3150801AC20BBF9C8F80000F5E730B583B004460A4613
S3150801AC30054655F8041B002300932B46FFF7C2FF70
S3150801AC4002462060012300932B4661682046FFF7E0
S3150801AC50B9FF206003B030BDF8B50C461D46104655
S3150801AC6075F0F4FD02460B4600204FF0804169F06D
S3150801AC70B5FF00220F4B75F08BFC06460F462046A2
S3150801AC8075F0E4FD02460B463046394675F036FE48
S3150801AC9076F02CF90646214676F07CF901463046CF
S3150801ACA076F078F901462860204676F073F9069B16
S3150801ACB01860F8BD0000F03F2DE9F04387B006465D
S3150801ACC0884617461D461146404676F06DFA0446F3
S3150801ACD0DFF8849004AB009305AB4A4641463046FB
S3150801ACE0FFF7BAFF02AB009303AB4A463946304633
S3150801ACF0FFF7B2FFDDF81480DDF80C9049464046AF
S3150801AD0076F052FA0146204676F044F90646049F43
S3150801AD103946484676F048FA0146304676F03AF919
S3150801AD200646DDF808904946404676F03DFA014662
S3150801AD30304676F02FF906464946384676F034FA13
S3150801AD40314676F027F90146286876F025F9286014
S3150801AD50204607B0BDE8F0830000404130B583B016
S3150801AD6004460A46054655F8041B2B46FFF7A4FF79
S3150801AD7002462060012300932B4661682046FFF7AF
S3150801AD8021FF206003B030BD014B0360704700BF4F
S3150801AD905031090810B50446FFF7F6FF2821204669
S3150801ADA047F07CFA204610BDC0E90023009B83606A
S3150801ADB0019BC3607047000030B40A4A0260002252
S3150801ADC00276426001218160074CC4601324046144
S3150801ADD001754275827500240025C0E9084530BC15
S3150801ADE0704700BF503109081F040100043070473D
S3150801ADF0007E0238C0B201288CBF002001207047AE
S3150801AE00C2688B681A4205D10269CB681A4203D017
S3150801AE1001207047012070470020704770B504462D
S3150801AE20037D8BB1437D8BB90B684D68066A426A0F
S3150801AE309E1945EB020506624562037E032B64D81B
S3150801AE40DFE803F00712303E037670BD022303766E
S3150801AE50FBE7FFF7D5FF0028F7D001232376002269
S3150801AE600023C4E90823F0E7FFF7CAFF10B9002356
S3150801AE702376EAE76168CA0E4B015B1A62F10002A2
S3150801AE80920042EA93729B005B1842F10002D200DB
S3150801AE9042EA5372DB009E4275EB0203D5D30223C5
S3150801AEA02376D2E7837D002BCFD1FFF7A9FF0028B0
S3150801AEB0CBD10323237600220023C4E90823C4E760
S3150801AEC0FFF79EFF10B102232376BEE7A068C20EE4
S3150801AED043011B1A62F10002520242EAD3525B0293
S3150801AEE01B1842F100024FEA821C4CEA936C990145
S3150801AEF0CB1A6CEB02021B1842F100029E4275EB5B
S3150801AF000203A2D3002323769FE7002303769CE757
S3150801AF10014B0360704700BF6031090810B504464C
S3150801AF20FFF7F6FF3821204647F0B8F9204610BD4D
S3150801AF30C0E90023009B83609DF804300373029BDC
S3150801AF400361039B4361704730B40E4A02600022D5
S3150801AF5080F82020002141624FF0FF318162C162F1
S3150801AF600949416009498160C26002610849416134
S3150801AF70826102774277827700240025C0E90C4571
S3150801AF8030BC704760310908000020C10000A0C02C
S3150801AF90130401000430704790F820000238C0B24B
S3150801AFA001288CBF00200120704700002DE9F04FD1
S3150801AFB087B0049205938B6801934FF00009CDF889
S3150801AFC00C90CDF80890DFF820A1B9F1000F77DCD5
S3150801AFD0019803F036FFB9F1000F19D1B02707FB25
S3150801AFE009074946019804F0ADF8804607F18C0B2C
S3150801AFF0584647F0D5FB3B7813F0040F0AD013F0F7
S3150801B000100F0BD13B7813F0200F18D100252AE039
S3150801B0100027E6E7584647F013FC4EE0404603F0A2
S3150801B020E6FE514676F05EFA0028EBD0404603F07C
S3150801B030DEFE8246CDF8089000230393E2E74046F8
S3150801B04003F0D8FE514676F04DFA0028DED0404688
S3150801B05003F0D0FE8246CDF8089001230393D5E785
S3150801B060002408E00135112D24DCF9D805EB450447
S3150801B070640020343C442946404603F0A5FE0646B2
S3150801B080204604F01CFD0028ECD0204604F027FDDC
S3150801B0900028E7D0304603F05DFE514676F022FAE5
S3150801B0A00028DFD0304603F055FE82460395CDF8D9
S3150801B0B00890D7E7584647F0C3FB09F1010984E729
S3150801B0C00949504676F004FA18B1002007B0BDE8E0
S3150801B0D0F08F049BC3F800A0059B029A1A60109B87
S3150801B0E0039A1A600120F1E79AF9794442690B69D2
S3150801B0F01A4205D182694B691A4203D00120704769
S3150801B100012070470020704708B50B7B33B91146FB
S3150801B110406876F005FA10B1012000E0002008BD6C
S3150801B12010B50C7B2CB91146806876F0DBF900B1B5
S3150801B1300124204610BD30B583B00446037FA3B170
S3150801B1400D46437FABB909686A68036B406B5B18A8
S3150801B15042EB00022363626394F82030032B00F26A
S3150801B160CA80DFE803F00A2C668D80F8203003B028
S3150801B17030BD022380F82030F9E704F12C0300934F
S3150801B18004F1280304F1240229462046FFF70EFF9D
S3150801B1900028ECD029462046FFF7A8FF0028E6D16B
S3150801B1A0626A29462046FFF7AFFF0028DFD0012350
S3150801B1B084F8203000220023C4E90C23D7E704F1E0
S3150801B1C02C03009304F1280304F12402294620469E
S3150801B1D0FFF7ECFE70B129462046FFF787FF48B90D
S3150801B1E0626A29462046FFF78FFF38B9002384F89B
S3150801B1F02030BCE7002384F82030B8E7216B626B66
S3150801B200E568E80E6B015B1B60F10000800040EA0F
S3150801B21093709B005B1940F10000C00040EA53702F
S3150801B220DB00994272EB0003A1D3022384F8203094
S3150801B2309DE7A37F002B9AD104F12C03009304F117
S3150801B240280304F1240229462046FFF7AFFE98B1E8
S3150801B25029462046FFF74AFF70B9626A2946204601
S3150801B260FFF75EFF002882D0032384F820300022EE
S3150801B2700023C4E90C237AE7002384F8203076E713
S3150801B28004F12C03009304F1280304F1240229464E
S3150801B2902046FFF78BFE70B129462046FFF726FFA9
S3150801B2A048B9626A29462046FFF73AFF38B90223A8
S3150801B2B084F820305BE7002384F8203057E7216BB8
S3150801B2C0626B2569E80E6B015B1B60F1000080006B
S3150801B2D040EA93709B005B1940F10000C00040EA08
S3150801B2E05370DB00994272EB0003FFF440AF002371
S3150801B2F084F820303BE7002384F8203037E7000044
S3150801B300014B0360704700BF7031090810B5044648
S3150801B310FFF7F6FF2821204646F0C0FF204610BD5C
S3150801B320C0E90023009B83607047000030B40A4AD5
S3150801B330026000220276094941604FF0804181602E
S3150801B340C2600261012101754275827500240025DA
S3150801B350C0E9084530BC704770310908CDCC0C40AE
S3150801B36004307047007E0238C0B201288CBF002025
S3150801B3700120704738B5044688680368DB68984732
S3150801B3804FF00105616876F0CBF808B94FF0000572
S3150801B39005F0010038BD38B5044688680368DB68DE
S3150801B3A098474FF00105A16876F09CF808B94FF067
S3150801B3B0000505F0010038BD70B50446037DD3B11B
S3150801B3C00D46437DCBB909686A68036A406A5B180A
S3150801B3D042EB000223626262A8680368DB68984749
S3150801B3E0002176F07FF858B9237E032B73D8DFE85E
S3150801B3F003F00A173949037670BD02230376FBE782
S3150801B40000232376F8E729462046FFF7B3FF0028ED
S3150801B410F2D00123237600220023C4E90823EBE7AF
S3150801B42029462046FFF7A6FF10B900232376E3E74E
S3150801B430216A626AE568E80E6B015B1B60F1000030
S3150801B440800040EA93709B005B1940F10000C00040
S3150801B45040EA5370DB00994272EB0003CCD3022316
S3150801B4602376C9E7A37D002BC6D129462046FFF7D7
S3150801B47092FF0028C0D00323237600220023C4E9C3
S3150801B4800823B9E729462046FFF785FF10B90223A5
S3150801B4902376B1E7206A616A2669F20E73019B1B5E
S3150801B4A062F10002520242EAD3525B029B1942F14F
S3150801B4B000024FEA821C4CEA936C9D01EB1A6CEB75
S3150801B4C002029B1942F10002984271EB020393D3DF
S3150801B4D00023237690E7002323768DE72DE9F04FA5
S3150801B4E083B007460191164600930C9C04F18045EA
S3150801B4F0013D52F82590D2F800804146484676F03B
S3150801B5000FF800284BD03946404675F0FFFF30B991
S3150801B5103946484675F0F0FF30B9002509E0009B29
S3150801B520186803B0BDE8F08F009B53F82500F8E7CB
S3150801B5300135631EAB427DDD4FEA850956F8258044
S3150801B5403946404675F0D8FF0028F1D06B1C4FEA02
S3150801B550830B56F823A03946504675F0D7FF0028C5
S3150801B560E6D0009B53F80950294653F80B0075F0AD
S3150801B57011FD04464146504675F00CFD014620462C
S3150801B58075F0C6FE04464146384675F003FD214668
S3150801B59075F00AFE0146284675F0FEFCC1E73946F4
S3150801B5A0404675F0A9FF30B93946484675F0AEFFF1
S3150801B5B020B9013C07E0009B1868B2E7009B53F8E5
S3150801B5C02500AEE7013C002C36DD4FEA840856F823
S3150801B5D024503946284675F08FFF0028F2D004F129
S3150801B5E08043013B4FEA830A56F823903946484679
S3150801B5F075F08CFF0028E5D0009B53F808603146AA
S3150801B60053F80A0075F0C6FC04462946484675F003
S3150801B610C1FC0146204675F07BFE0446294638469C
S3150801B62075F0B8FC214675F0BFFD0146304675F048
S3150801B630B3FC76E7019874E7019872E7014B03605A
S3150801B640704700BF8031090810B50446FFF7F6FFB9
S3150801B6502821204646F022FE204610BDC0E90023D7
S3150801B6609DF9003003729DF9043043729DF9083043
S3150801B6708372704730B40B4A02600022027480F864
S3150801B68020204FF47A7141604FF461618160027341
S3150801B690427382730122C27300240025C0E906455C
S3150801B6A030BC70478031090804307047007C023885
S3150801B6B0C0B201288CBF00200120704790F82000F5
S3150801B6C0704710462AB191F90830002B02DC002098
S3150801B6D070470020704770B50446437B5BB1807B99
S3150801B6E068B9227B012A28D0022A33D06AB10123FC
S3150801B6F084F820300CE0037480F8203070BD0223F2
S3150801B7002374012384F82030F8E7012384F82030D4
S3150801B7100B684D68A669E2699E1945EB0205A661A3
S3150801B720E56191F90830002B21DB237C032B00F21C
S3150801B7308C80DFE803F0212F506191F90920002A56
S3150801B74002DD84F82030E3E791F90A20002AF8DCC3
S3150801B7500346F6E791F90920002A02DD84F820005C
S3150801B760D6E791F90A20002AF8DC1846F6E70023FD
S3150801B770237484F82030C1E794F820202046FFF787
S3150801B780A0FF0028BAD00123237400220023C4E9AC
S3150801B7900623B3E794F820202046FFF792FF10B955
S3150801B7A000232374AAE76168CA0E4B015B1A62F18A
S3150801B7B00002920042EA93729B005B1842F1000272
S3150801B7C0D20042EA5372DB009E4275EB020395D31F
S3150801B7D00223237492E7E37B002B8FD194F8202070
S3150801B7E02046FFF76EFF002888D103232374002221
S3150801B7F00023C4E9062381E794F820202046FFF7B1
S3150801B80060FF10B10223237478E7A068C20E4301D2
S3150801B8101B1A62F10002520242EAD3525B021B185A
S3150801B82042F100024FEA821C4CEA936C9901CB1A49
S3150801B8306CEB02021B1842F100029E4275EB0203F1
S3150801B840FFF45CAF0023237458E70023237455E7FC
S3150801B850014B0360704700BF9031090810B50446D3
S3150801B860FFF7F6FF1421204646F018FD204610BDC5
S3150801B870094B0360094B4360094B8360012303733A
S3150801B880002343738373002B04DCC218002111744F
S3150801B8900133F8E7704700BF9031090800008C4270
S3150801B8A000008242014B0360704700BFA0310908BE
S3150801B8B010B50446FFF7F6FF2021204646F0EEFCB8
S3150801B8C0204610BDC0E90023009B83609DF8043023
S3150801B8D00373704730B40A4A0260002202744FF0BB
S3150801B8E0FF31416142F210714160012181600173AA
S3150801B8F04273827300240025C0E9064530BC7047AF
S3150801B900A031090804307047007C0238C0B201280A
S3150801B9108CBF0020012070472DE9F8430F7B67BBD8
S3150801B9200C4690460026002E20DCA06803F089FA12
S3150801B9309EB9B02505FB060505F18C09484646F072
S3150801B9402FFF2B7813F0010F02D013F0020F06D048
S3150801B950484646F075FF0136E5E70025ECE7484617
S3150801B96046F06EFFC8F80060012703E04FF0FF3389
S3150801B970C8F800303846BDE8F8830027FAE738B535
S3150801B9800446037B8BB1437B8BB908684A68A36974
S3150801B9901B18E06942EB0002A361E261237C032BD9
S3150801B9A076D8DFE803F007153849037438BD022352
S3150801B9B00374FBE704F114022046FFF7ADFF0028E4
S3150801B9C0F4D00123237400220023C4E90623EDE7FA
S3150801B9D004F114022046FFF79FFF10B900232374D0
S3150801B9E0E4E7A169E2696568E80E6B015B1B60F132
S3150801B9F00000800040EA93709B005B1940F100004B
S3150801BA00C00040EA5370DB00994272EB0003CDD3C4
S3150801BA1002232374CAE7A37B002BC7D104F11402BE
S3150801BA202046FFF779FF0028C0D10323237400229B
S3150801BA300023C4E90623B9E704F114022046FFF7F7
S3150801BA406BFF10B102232374B0E7A069E169A56809
S3150801BA50EA0E6B015B1B62F10002520242EAD35203
S3150801BA605B025B1942F100024FEA821E4EEA936EAF
S3150801BA704FEA831CBCEB03036EEB02025B1942F12E
S3150801BA800002984271EB020390D3002323748DE7D9
S3150801BA90002323748AE70000014B0360704700BF47
S3150801BAA0B031090810B50446FFF7F6FF28212046EC
S3150801BAB046F0F4FB204610BDC0E90023009B8360D5
S3150801BAC07047000030B40A4A02600022027609492A
S3150801BAD0416009498160C2600261012101754275AF
S3150801BAE0827500240025C0E9084530BC704700BFAF
S3150801BAF0B03109080000A0410000C8410430704770
S3150801BB00007E0238C0B201288CBF00200120704790
S3150801BB1010B50B464FF001044168986875F0E2FCD0
S3150801BB2008B94FF0000404F0010010BD10B50B462A
S3150801BB304FF001048168986875F0F2FC08B94FF076
S3150801BB40000404F0010010BD70B50446037D8BB1F5
S3150801BB50437D8BB90B684D68066A426A9E1945EBA7
S3150801BB60020506624562037E032B64D8DFE803F00B
S3150801BB700712303E037670BD02230376FBE7FFF713
S3150801BB80C7FF0028F7D00123237600220023C4E942
S3150801BB900823F0E7FFF7BCFF10B900232376EAE78D
S3150801BBA0E168CA0E4B015B1A62F10002920042EA91
S3150801BBB093729B005B1842F10002D20042EA53726B
S3150801BBC0DB009E4275EB0203D5D302232376D2E727
S3150801BBD0837D002BCFD1FFF7A9FF0028CBD0032304
S3150801BBE0237600220023C4E90823C4E7FFF79EFF52
S3150801BBF010B902232376BEE72069C20E43011B1A38
S3150801BC0062F10002520242EAD3525B021B1842F168
S3150801BC1000024FEA821C4CEA936C9901CB1A6CEB31
S3150801BC2002021B1842F100029E4275EB0203A2D3DF
S3150801BC30002323769FE7002303769CE7014B0360E5
S3150801BC40704700BFC031090810B50446FFF7F6FF73
S3150801BC502821204646F022FB204610BDC0E90023D4
S3150801BC609DF8003003729DF9043043729DF808303F
S3150801BC7083729DF90C30C3729DF9103003739DF8D8
S3150801BC80143043739DF8183083739DF81C30C373C1
S3150801BC909DF820300374099B43610A9B83610B9BC2
S3150801BCA0C3610C9B0362704730B40B4A02600022E1
S3150801BCB00276426042F21071816040F21741C1601A
S3150801BCC01221016102750121417582750024002541
S3150801BCD0C0E9084530BC7047C031090804307047CF
S3150801BCE0007E0138C0B202288CBF002001207047AF
S3150801BCF0007E0238C0B201288CBF0020012070479F
S3150801BD000346887AF0B91B7D012B06D0022B06D093
S3150801BD104B7BD3B98B7BBBB17047087A70474B7B9A
S3150801BD209BB98B7B8BB991F90B30002B0DDC91F903
S3150801BD300C30002B09DC91F90930002B01DD0120BB
S3150801BD40704770470020704701207047C268CB6969
S3150801BD501A4205D102690B6A1A4203D001207047BB
S3150801BD6001207047002070470346C87B80B9087CCC
S3150801BD7070B94A69D3F80CC01CEA020F07D18A695F
S3150801BD80D3F810C01CEA020F02D0012000E00120FE
S3150801BD901B7D012B06D0022B08D04B7B13BB8B7B5B
S3150801BDA013BB7047087A80F0010070474B7B9BB93B
S3150801BDB08B7B9BB991F90B30002B01DD0120704774
S3150801BDC091F90C30002B01DD0120704791F90930FA
S3150801BDD0002B05DD002070470020704700207047C2
S3150801BDE0012070470020704700207047F8B50446C7
S3150801BDF0437D8BB10D460B684F68066A426A9E19E8
S3150801BE0047EB020706624762037E042B6CD8DFE81C
S3150801BE1003F00516384361000376F8BDFFF770FF96
S3150801BE200028FAD029462046FFF790FF0028F4D1CA
S3150801BE300123237600220023C4E90823EDE7FFF74F
S3150801BE405FFF20B129462046FFF780FF08B100238E
S3150801BE5023766168CA0E4B015B1A62F100029200F1
S3150801BE6042EA93729B005B1842F10002D20042EA51
S3150801BE705372DB009E4277EB0203CED3022323766D
S3150801BE80CBE7FFF771FF0028C7D0032323760022EB
S3150801BE900023C4E90823C0E7FFF766FF10B90223A8
S3150801BEA02376BAE7A168CA0E4B015B1A62F1000252
S3150801BEB0920042EA93729B005B1842F10002D2009B
S3150801BEC042EA5372DB009E4277EB0203A5D30423B1
S3150801BED02376A2E7837D002B9FD1FFF745FF002834
S3150801BEE09BD10023237698E70023037695E7000084
S3150801BEF0014B0360704700BFD031090810B50446ED
S3150801BF00FFF7F6FF5021204646F0C8F9204610BD36
S3150801BF10C0E90023009B8360019BC360029B036108
S3150801BF209DF80C300375704730B41A4A0260002236
S3150801BF3080F83420012180F8351080F83610002465
S3150801BF4044604FF07E5484604FF4FA64C460026121
S3150801BF5001754FF47A7484613C24C46180F8202009
S3150801BF6080F821200C4C44620C4C84624FF4FA741C
S3150801BF70C46280F8301080F8312080F8322000241D
S3150801BF800025C0E90E45C0E91045C0E9124530BC97
S3150801BF90704700BFD03109080000704200002041F7
S3150801BFA00430704790F83400032814BF002001209C
S3150801BFB0704790F83430012B05D0032B01D00020AF
S3150801BFC07047012070470120704790F83400042813
S3150801BFD014BF002001207047F8B505460C4688684D
S3150801BFE003689B6898470646A06803689B68984754
S3150801BFF00146304675F0D8F86F6A394675F0D4F8B7
S3150801C0000646E168206974F0C5FF95F820307BB1D2
S3150801C01004464FF07C51384675F078FA88B12146C6
S3150801C020204675F0C1F8394675F072F9044600E004
S3150801C03000243146204675F055FA00B134462046AB
S3150801C040F8BD0024F5E700002DE9F04182B0044669
S3150801C0500D4690F83030002B2BD090F83160002E29
S3150801C06039D10B684F68826BC16B9B1847EB010787
S3150801C0708363C76328686968226C1218606C41EB90
S3150801C08000012264616469680191A26CE06C296807
S3150801C0905218019941EB0001A264E16494F8342035
S3150801C0A0042A13D8DFE812F0230037000D013701FF
S3150801C0B055010B7D6BB1012384F83430002200232E
S3150801C0C0C4E90E23C4E91023C4E9122302B0BDE86A
S3150801C0D0F0810023F0E7042380F83430002200239E
S3150801C0E0C0E90E23C0E91023C0E91223EEE72B7D30
S3150801C0F0002BEBD0012384F8343084F83530237DC6
S3150801C10084F8363000220023C4E90E23C4E910233B
S3150801C110C4E91223DAE72F7D1FB9002384F83430E6
S3150801C120D4E794F8213053BBD4F804809B494046A0
S3150801C13075F0E2F9002849D094F82030002B45D152
S3150801C140A16BE26BE568E80E6B015B1B60F1000011
S3150801C150800040EA93709B005B1940F10000C00023
S3150801C16040EA5370DB00994272EB0003AED3032316
S3150801C17084F8343000220023C4E90E23A6E72946B1
S3150801C1802046FFF729FFA16A75F0ACF920B1002214
S3150801C1900023C4E91223C7E7A16CE26AD00E530152
S3150801C1A09B1A60F10000800040EA93709B009B187F
S3150801C1B040F10000C00040EA5370DB009942E36C8D
S3150801C1C08341B1D3042384F834307FE77349404669
S3150801C1D075F0A6F9F0B93E4694F8203073B129698D
S3150801C1E0E86874F0D7FE20F000414FF00107A06817
S3150801C1F075F08CF908B94FF00007FFB2002E35D05B
S3150801C200002F33D0032384F8343000220023C4E9F5
S3150801C2100E235BE794F83530012B06D0022B15D097
S3150801C220012384F835303E46D6E7226C636C5C49B7
S3150801C23091424FF0000272EB0303CDD20022002394
S3150801C240C4E91023022384F83530C5E7A8680368D2
S3150801C2509B68984720F000414FF00106606875F029
S3150801C26055F908B94FF00006F6B2B5E7A16BE26BCE
S3150801C270E568E80E6B015B1B60F10000800040EA8F
S3150801C28093709B005B1940F10000C00040EA5370AF
S3150801C290DB00994272EB0003FFF418AF94F83630CD
S3150801C2A0013BDBB284F836303BB1022384F83430E3
S3150801C2B000220023C4E90E2308E7042384F8343056
S3150801C2C0F6E72A7D1AB9002384F83430FEE6206998
S3150801C2D0C10E4201121A61F10001890041EA927107
S3150801C2E09200121841F10001C90041EA5271D200C7
S3150801C2F0934277EB0103FFF4E9AE012384F8343066
S3150801C30084F8353000220023C4E90E23C4E910233A
S3150801C310C4E91223DAE62A7D002A7FF4D7AEA0699A
S3150801C320C10E4201121A61F10001890041EA9271B6
S3150801C3309200121841F10001C90041EA5271D20076
S3150801C340934277EB0103FFF4C1AE002384F834303E
S3150801C350BCE694F83220002A7FF4B8AEE569E90E06
S3150801C3606A01521B61F10001490241EAD2515202A6
S3150801C370521941F100018E0146EA92669001821A2C
S3150801C38066EB0101521941F10001934277EB010372
S3150801C390FFF49CAE002384F8343097E66F12833A93
S3150801C3A09F860100014B0360704700BFE031090811
S3150801C3B010B50446FFF7F6FF3021204645F06EFF1B
S3150801C3C0204610BDC0E90023009B8360019BC36022
S3150801C3D09DF8083003749DF90C3043749DF91030AB
S3150801C3E083749DF81430C3749DF8183003759DF84D
S3150801C3F01C3043759DF8203083759DF82430C3752C
S3150801C4009DF828300376704730B40C4A0260002242
S3150801C410027580F828200A49416082604FF47A71D2
S3150801C420C160027442740122827400240025C0E9A5
S3150801C4300645C0E9084530BC704700BFE031090828
S3150801C4400000904104307047F8B50446837CD3B1A7
S3150801C4500D460B684E688769C269DF1946EB020605
S3150801C4608761C6610B684968006A626A1B1841EBF5
S3150801C470020223626262217D032900F2CB80DFE892
S3150801C48001F0061D96C580F828300375F8BD00230E
S3150801C49084F82830237C53B195F91230002BF5DC4A
S3150801C4A00123237500220023C4E90623EEE70123AD
S3150801C4B0237500220023C4E90623E7E7617C29B135
S3150801C4C0E97C21B300220023C4E9082394F8283023
S3150801C4D0002B3ED195F91230002B36DDE168CA0EE4
S3150801C4E04B015B1A62F10002920042EA93729B00C9
S3150801C4F05B1842F10002D20042EA5372DB009F4206
S3150801C50076EB020325D3012384F8283021E0D4F8F9
S3150801C5100CC04FEADC604FEA4C11B1EB0C0160F13B
S3150801C5200000800040EA9170890011EB0C0140F18E
S3150801C5300000C00040EA5170C9008B4272EB00034B
S3150801C540C4D3012384F82830C0E700220023C4E9B4
S3150801C550062394F828301BB12B7D0BB16B7D6BB983
S3150801C560A36873B1AA7D1AB9EA7D0AB92A7E42B1CE
S3150801C570EA68C3EB0313B2EB830F02D303232375D4
S3150801C58084E72B7C002B81D16168A86874F0B4FF1D
S3150801C59000283FF47BAF95F91130002B3FF776AFB2
S3150801C5A00223237500220023C4E906236EE72B7CA8
S3150801C5B023B96168A86874F0B3FF18B995F9113001
S3150801C5C0002B02DD0123237560E7637C23B1EB7C35
S3150801C5D013B90323237559E794F8283033B995F924
S3150801C5E01230002B02DD012384F8283094F8283014
S3150801C5F01BB12B7D0BB16B7D2BB9084B9F4276F195
S3150801C6000003FFF443AF032323753FE7012384F8AF
S3150801C61028303BE70123237538E700BF00879303DA
S3150801C62090F828007047007D032814BF00200120D8
S3150801C6307047007D02288CBF00200120704700004A
S3150801C640024A0260024A0260704700BF10320908B6
S3150801C650F03109080369002B00F0BD802DE9F0418E
S3150801C66004468069F8B1A568E168226C636C5219C1
S3150801C67041EB030322646364A36CE26C5B1941EB2F
S3150801C6800201A364E16403689B689847064694F827
S3150801C690515055B1012D23D0002384F85030002282
S3150801C6A0E26384F85130BDE8F08194F833304BB138
S3150801C6B094F8323033B9A063E063012384F850302B
S3150801C6C084F8523094F83230002BECD00022002343
S3150801C6D0C4E91023C4E91223012384F85130E2E79F
S3150801C6E094F8323033B984F850300022E26384F882
S3150801C6F05130D8E7D4F838803749404674F054FDAC
S3150801C70007464146304674F045FC20F0004027F0C4
S3150801C710004174F005FF20B1A66300220023C4E995
S3150801C7201023216C626C666AF00E73019B1B60F123
S3150801C7300000800040EA93709B009B1940F10000BD
S3150801C740C00040EA5370DB00994272EB0003AAD39A
S3150801C75094F8503023B90021E06B74F0B9FE88BB18
S3150801C760E16BA06B74F016FC20F000461B49E069EA
S3150801C77074F01AFD314674F0B5FE18B3002384F837
S3150801C7805030A16CE26CA66AF00E73019B1B60F136
S3150801C7900000400240EAD3505B029B1940F10000B9
S3150801C7A04FEA801C4CEA936C9F01FB1A6CEB000064
S3150801C7B09B1940F10000994272EB000300D2022551
S3150801C7C084F85250A36BE36300220023C4E91023C3
S3150801C7D0C4E9122367E77047CDCC4C3DCDCC4C3E1E
S3150801C7E090F85200022814BF002001207047002348
S3150801C7F080F85230704710B50446FFF721FF5821DB
S3150801C800204645F04BFD204610BD00002DE9F04FAE
S3150801C81083B00446006938B10F4615461E4663695A
S3150801C82013B194F8523013B903B0BDE8F08F0C99DF
S3150801C83002F088FC0D9902F0C7FA02F089FA8046DF
S3150801C84094F85230022B04D0C5F80080A36B3360EC
S3150801C850EAE70C99606903F0FFF80D9902F087FE83
S3150801C86002F068FEFEF791F974F0A0FE5FFA80F90E
S3150801C870D5F800A02AF0004B2C49584674F05AFE08
S3150801C8800028E1D12949584674F04AFE0028DBD12F
S3150801C8903368019323F0004B2449584674F04AFE45
S3150801C8A00028D1D12149584674F03AFE0028CBD147
S3150801C8B094F830304B45C7D894F831304B45C3D33B
S3150801C8C05146404674F066FB81460199A06B74F0A7
S3150801C8D061FB0146484674F01BFD20F000491349E7
S3150801C8E0484674F027FE0028AED11049484674F030
S3150801C8F017FE0028A8D1D4F820B0E16A584674F08A
S3150801C90053FC8246494674F0EDFD10B1C7F800A004
S3150801C9109AE74FF07C51584674F046FC494674F044
S3150801C920EBFD002890D0C7F800908DE7FFFF7F7FC9
S3150801C93030B4184A0260184A026000228263C26350
S3150801C940002280F8502080F8512080F852200024D7
S3150801C9500025C0E902450261426182610F49C16150
S3150801C9600F49016241F2883141621E2181624FF00D
S3150801C970804CC0F82CC080F83010642180F8311042
S3150801C98080F8322080F83320C0E91045C0E9124505
S3150801C99030BC7047F031090810320908CDCC0C407B
S3150801C9A00AD7A33D08307047014B0360704700BFA3
S3150801C9B03032090810B50446FFF7F6FF6021204614
S3150801C9C045F06CFC204610BDC0E90023DDE90023D3
S3150801C9D0C0E902239DF9083003749DF80C304374AD
S3150801C9E09DF8103083749DF81430C374704708306D
S3150801C9F0704710B50446E0E9082304F128016AF0F6
S3150801CA00A7FABDF80830A4F84C3010BD10B582B0AD
S3150801CA100446114B0360002180F84E1080F8581027
S3150801CA204FF461620023C0E90223032303821E2314
S3150801CA3043820123037543758375C375037643766C
S3150801CA408376C17600220023C0E914230091FFF7FB
S3150801CA50D0FF204602B010BD3032090890F84E00CA
S3150801CA600138C0B201288CBF00200120704790F818
S3150801CA704E00022814BF00200120704700F1200152
S3150801CA80D1E900017047B0F84C00704770B58AB01B
S3150801CA9004460D464B7C4BB991F91030002B38DD15
S3150801CAA090F95830002B36DD002600E0002601A952
S3150801CAB005F108006AF04CFA079B0BB9A27E62B928
S3150801CAC0012B2AD0022B2CD0032B2ED0042B30D0AD
S3150801CAD0052B32D0062B34D00022E16B069B9942F6
S3150801CAE031D00120AB68E968656AD4F820C0B3EB98
S3150801CAF00C0361EB0501A568E468002E38D0002A0D
S3150801CB0039D0002839D0AB4271EB040331DA002061
S3150801CB102FE00026CBE70126C9E7227D002ADCD1D2
S3150801CB20D0E7627D002AD8D1CEE7A27D002AD4D1EA
S3150801CB30CCE7E27D002AD0D1CAE7227E002ACCD1F1
S3150801CB40C8E7627EC9E7A16B059B994201D001201E
S3150801CB50C8E7616B049B994201D00120C2E7B4F88A
S3150801CB604C10238A994201D20120BBE70020B9E77C
S3150801CB7000200AB070BD0020FBE70020F9E700009D
S3150801CB8070B58AB004460D46C37EC3B10A684868C3
S3150801CB90216D636D511840EB03032165636594F8B4
S3150801CBA04E20012A20D0022A03D07AB1002384F824
S3150801CBB04E3095F9103084F858300AB070BD80F8B7
S3150801CBC04E3091F9103080F85830F6E7294620465C
S3150801CBD0FFF75CFF0028ECD0012384F84E300022D1
S3150801CBE00023C4E91423E4E7AA7C3AB9EA7C2AB902
S3150801CBF0234A8A424FF000029A411ED3B4F812E042
S3150801CC004FEA4E12B2EB0E0260EB0000400240EA18
S3150801CC10D250520212EB0E0240F1000C4FEA8C166A
S3150801CC2046EA92669001821A66EB0C0012EB0E0236
S3150801CC3040F1000091428341BBD301A905F10800E7
S3150801CC406AF086F9E36B069A9A420AD00123A4F898
S3150801CC504C30D5E90223C4E90823022384F84E306F
S3150801CC60A7E7A36B059A9A42F0D1636B049A9A4295
S3150801CC70ECD1B4F84C300133A4F84C30E9E700BFE5
S3150801CC803F420F00014B0360704700BF403209085D
S3150801CC9010B50446FFF7F6FF2021204645F0FEFAB7
S3150801CCA0204610BDC0E90023009B83607047000041
S3150801CCB030B40A4A02600022027500240025C0E940
S3150801CCC00645074941604FF4616181607821C16079
S3150801CCD002744274827430BC704700BF403209083E
S3150801CCE000009643043070472DE9F0410446037C61
S3150801CCF0E3B10D46437CE3B90F68D1F8048088682F
S3150801CD000368DB68984720F00046A86803681B6932
S3150801CD10984720F00041304667F032FF0146237DEF
S3150801CD20032B4DD8DFE803F0081328360375BDE851
S3150801CD30F08102230375FAE7606874F0D3FB0028D3
S3150801CD40F5D001232375A761C4F81C80EFE7606855
S3150801CD5074F0E6FB10B100232375E8E7A369E269DD
S3150801CD60FB1A68EB0202A16899424FF0000393414E
S3150801CD70DDDA02232375DAE7A37C002BD7D16068B5
S3150801CD8074F0CEFB0028D2D003232375A761C4F81B
S3150801CD901C80CCE7606874F0A5FB10B102232375EB
S3150801CDA0C5E7A369E269FF1A68EB0208E368BB42B3
S3150801CDB04FF0000373EB0803B9DA00232375B6E7CE
S3150801CDC000232375B3E7007D0238C0B201288CBF62
S3150801CDD00020012070470000024A0260024A0260F0
S3150801CDE0704700BF50320908802E0908C06A70478B
S3150801CDF00020704710B50446FFF7EEFF382120469C
S3150801CE0045F04CFA204610BDC0E900239DF80030D4
S3150801CE1003729DF804304372029BC3609DF90C307E
S3150801CE2003749DF810304374059B436170470000F5
S3150801CE3030B4114A0260114A0260002280F82820A3
S3150801CE4080F829200021C16280F8302080F831203D
S3150801CE5080F832204FF4C871416009498160094957
S3150801CE60C1600274427400240025C0E90645C0E980
S3150801CE70084530BC704700BF802E090850320908A2
S3150801CE800AD7233DCDCC4C3E002380F8293080F8C3
S3150801CE90283080F8323080F8313080F8303000237D
S3150801CEA0C36200220023C0E90623C0E908237047AC
S3150801CEB004307047F8B50446437C83B30D460968C8
S3150801CEC06A688369C0695B1842EB0002A361E26183
S3150801CED094F830309BBB94F828202B7A9A4203D0D9
S3150801CEE000220023C4E90623A169E2696668F00EF7
S3150801CEF073019B1B60F10000800040EA93709B0060
S3150801CF009B1940F10000C00040EA5370DB009942CA
S3150801CF1072EB00031FD3012384F830301BE0002293
S3150801CF200023C0E90623C0E908230023C3620023BE
S3150801CF3080F8323080F8313080F830306CE094F87F
S3150801CF4028202B7A9A4206D000220023C4E9062318
S3150801CF50002384F830302B7A84F8283029686A68E7
S3150801CF60236A606A5B1842EB00022362626294F8E4
S3150801CF703130ABB994F829206B7C9A4203D0002250
S3150801CF800023C4E90823226A636A264991424FF0BD
S3150801CF90000272EB03030FD2012384F831300BE050
S3150801CFA094F829206B7C9A4206D000220023C4E912
S3150801CFB00823002384F831306B7C84F829306B7A96
S3150801CFC0003B18BF012384F8323094F83030EBB9AE
S3150801CFD094F831300BBBE86874F092F8124974F092
S3150801CFE097F9064620F000473946E06874F098FA42
S3150801CFF068B13946A06874F07FFA80B1686974F03F
S3150801D0007FF8094974F084F9064600E00026237C76
S3150801D0100BB106F10046E662F8BD0026F7E70026E1
S3150801D020F5E700BFFF083D0000007A44C06A704773
S3150801D030034690F8300008B993F83100704790F824
S3150801D04032007047014B0360704700BF98320908E8
S3150801D05010B50446064B036000F59C70FFF7F2FF16
S3150801D06004F58C70FFF7EEFF024B2360204610BDD6
S3150801D070A832090868320908054BC0F80831C0F812
S3150801D0800C31002380F8103180F81131704700BF48
S3150801D0900000C07FD0F800017047D0F8080170473A
S3150801D0A0D0F80C0170470000024A0260024A026089
S3150801D0B0704700BFD83209086832090810B5044616
S3150801D0C000F10801D1E9000174F028F8044974F067
S3150801D0D01FF9C4F88000606803689B68984710BD0B
S3150801D0E000247449D0F88400704708B5406803687D
S3150801D0F05B69984708BD08B5406803689B69984706
S3150801D10008BD08B540680368DB69984708BD08B5D6
S3150801D110406803681B6A984708BD08B540680368F4
S3150801D1205B6A984708BD10B50446FFF78BFF2021B7
S3150801D130204645F0B3F8204610BD10B50446FFF762
S3150801D14087FF4FF4AC71204645F0A8F8204610BD7C
S3150801D15010B50446FFF7A8FF8821204645F09EF83A
S3150801D160204610BD30B4064A0260017600224260AC
S3150801D170826000240025C0E9044530BC704700BF21
S3150801D180983209080430704710B49DF804400169C3
S3150801D1905218416941EB030302614361017E29BBD0
S3150801D1A0F4B144684FEAD46C6101091B6CF1000CB7
S3150801D1B04FEA8C0C4CEA917C890009194CF1000C58
S3150801D1C04FEACC0C4CEA517CC9008A4273EB0C033A
S3150801D1D00AD30123037600220023C0E9042303E0CE
S3150801D1E000220023C0E9042310BC7047F4B98468FF
S3150801D1F04FEAD46C6101091B6CF1000C4FEA8C0CE7
S3150801D2004CEA917C890009194CF1000C4FEACC0CC7
S3150801D2104CEA517CC9008A4273EB0C03E4D3002320
S3150801D220037600220023C0E90423DDE70022002358
S3150801D230C0E90423D8E7000030B583B00446D0F826
S3150801D240085125F000451A49284674F073F930BB90
S3150801D2501749284674F064F908BBD4F80C5125F02F
S3150801D26000451349284674F065F9E0B9104928467E
S3150801D27074F056F9B8B994F810310093D4E9022339
S3150801D28004F58C70FFF780FF94F811310093D4E907
S3150801D290022304F59C70FFF777FF03B030BD002326
S3150801D2A0C4F80831D9E70023C4F80C31E3E700BF15
S3150801D2B0FFFF7F7F007E704708B500F58C70FFF78A
S3150801D2C0F9FF08BD08B500F59C70FFF7F3FF08BD27
S3150801D2D02DE9F8430746384B0360384B03600023B2
S3150801D2E0C0F80831C0F80C3100F58C7900214846A0
S3150801D2F0FFF738FF07F59C7800214046FFF732FF14
S3150801D3000023142B0ADCC3EB8332C3EB820264329B
S3150801D31003F1080127F811200133F2E70024032C51
S3150801D3200FDC04EB840000EB800073F0E9FE24496E
S3150801D33073F030FE04F10E0307EB830358600134E2
S3150801D340EDE7002600E00136142E19DC0025032D31
S3150801D350F9DC304673F0D4FE1A4973F025FF01460D
S3150801D360194873F017FE05EB4503C3EBC3043444B0
S3150801D370243407EB440474F019F9A0800135E6E773
S3150801D3800024C7F8F440C7F8F840C7F8FC400F4B2B
S3150801D390C7F800310E4BC7F804314846FFF7F2FECD
S3150801D3A04FF4FA65056044604046FFF7EBFE0560F9
S3150801D3B044603846BDE8F88368320908A832090886
S3150801D3C00000C8418FC2753D66668640CDCC0C40CB
S3150801D3D00000C8420830704770B504462D4B0360FB
S3150801D3E02D4B036041600023C0F88030C0F88430BB
S3150801D3F000220023C0E90223002513E005EB85007E
S3150801D40000EB800073F07CFE0146244873F0C2FDF0
S3150801D4102B1D44F8230005F108034FF07E5244F80A
S3150801D42023200135032DE9DD002510E005F10C0661
S3150801D4304FF4FA7005FB00F073F062FE44F826001B
S3150801D44005F110034FF07E5244F823200135032DD0
S3150801D450ECDD002323656365A365E365104A22664F
S3150801D4606266104AA266104AE266226784F8743038
S3150801D47084F8753084F8763084F8773084F8783013
S3150801D48084F8793084F87A3084F87B3084F87C30F3
S3150801D490204670BD68320908D83209080000C8411B
S3150801D4A0CDCC0C400000C842CDCC6C40083070474A
S3150801D4B02DE9F0410546069C04F10040013832F891
S3150801D4C010C01688B44542D9AE4204D2AC4505D936
S3150801D4D04FF0000C07E01888BDE8F08133F810001A
S3150801D4E0FAE70CF1010C601E604569DD4FEA4C0E46
S3150801D4F032F81C60AE42F4D80CF101004FEA40083C
S3150801D50032F81070AF42ECD333F8080033F80E80C6
S3150801D510A0EB080073F0F4FD0446B81B73F0F0FDA8
S3150801D5200146204673F0F4FE0446A81B73F0E8FD95
S3150801D530214673F039FE0446404673F0DDFD014687
S3150801D540204673F029FD74F031F880B2C4E7AE4283
S3150801D55004D9AC4504D204F1FF3C06E01888BBE7C0
S3150801D56033F81000B8E70CF1FF3CBCF1000F29DDD8
S3150801D5704FEA4C0032F81C60AE42F4D80CF1004474
S3150801D580013C670032F81440AC42ECD3DA5B1F5A0F
S3150801D590D01BA41B90FBF4F073F0B2FD0446A81B44
S3150801D5A073F0AEFD214673F0FFFD0446384673F06D
S3150801D5B0A7FD214673F0F0FC73F0F8FF80B28BE704
S3150801D5C0084689E7084687E72DE9F04F95B00491A3
S3150801D5D0D0F8F480B8F1000F00F07D8104461546B5
S3150801D5E01E46D0F8F870002F00F07581D0F8FC308F
S3150801D5F0002B00F070811146404601F0A3FD31462B
S3150801D60001F0E2FB01F0A4FB81462946384601F008
S3150801D6105DFF314601F0C5FD01F0AFFD0746D4F8BF
S3150801D620FC0003685B6929469847394673F0BCFDD7
S3150801D6300146484673F0AEFC0390404601F001FCF2
S3150801D64055BBB02303FB0500112E27D806EB46036D
S3150801D6505B002033184402F042FA08B329464046D3
S3150801D66001F070FD314601F0AFFB01F073FB814615
S3150801D670E76B4946384673F053FF30B9A76C4946FC
S3150801D680384673F02FFF00B94F462A22002107A812
S3150801D6906AF056FA002565E00020D5E70020DAE7AA
S3150801D6A0404601F0CEFB75B9B02303FB05000378AC
S3150801D6B013F0100F09D02946404601F043FD01F049
S3150801D6C096FB8146D4E70020F1E7404601F0B9FB15
S3150801D6D075B9B02303FB0500037813F0200F09D0B1
S3150801D6E02946404601F02EFD01F084FB8146BFE73D
S3150801D6F00020F1E7404601F0A4FB55B94FF0B00B05
S3150801D7000BFB050B00274FF0120ADFF8D0910594A1
S3150801D71005E04FF0000BF5E7002008E00137112F6F
S3150801D7201BDCF9D807EB470040002030584402F0CB
S3150801D730D6F90028F2D0BC1B002CB8BF6442A2451A
S3150801D7400DDD2946404601F0FDFC394601F03CFB5A
S3150801D75001F000FB8146A246E0E7059C88E7059CA7
S3150801D76086E70135022D55DC05F10E0304EB83032B
S3150801D770D3F804803946404673F0BEFE0028F0D03F
S3150801D78005F1010B05F10F0304EB83035E683946C6
S3150801D790304673F0BBFE0028E3D005960026142E0A
S3150801D7A038DC0BEB4B03C3EBC3033344243304EBE1
S3150801D7B04303988805EB4503C3EBC303334424337A
S3150801D7C004EB4303B3F804A0A0EB0A0073F098FC3A
S3150801D7D081464146059873F0DDFB0146484673F0DC
S3150801D7E097FD81464146384673F0D4FB494673F0A6
S3150801D7F0DBFC8146504673F07FFC0146484673F0D0
S3150801D800CBFB14AB03EB460973F0D0FE29F8340CB5
S3150801D8100136C4E7D4F8086126F0004530492846A0
S3150801D82073F088FE48B92E49284673F079FE20B967
S3150801D8300399304673F074FE10B1039BC4F808319E
S3150801D840D4F80C6126F000452549284673F072FE86
S3150801D85048B92349284673F063FE20B9039930462F
S3150801D86073F040FE10B1039BC4F80C311D490398AF
S3150801D87073F09AFC73F09AFE80B2BDF84430984270
S3150801D88002D8012384F81031BDF81C30984202D31E
S3150801D890012384F811311523009304F1100307AA13
S3150801D8A00021FFF705FE73F027FC0F4973F030FDE1
S3150801D8B005460D4973F034FE00B10B4D12AC2946ED
S3150801D8C02046FDF75DF994E80300049B83E803000D
S3150801D8D02046FDF759F915B0BDE8F08F0000C8419B
S3150801D8E0FFFF7F7F00007A440000C8422DE9F04F10
S3150801D8F093B01D46436D53B304460E461746836DD2
S3150801D9002BB3036D1BB30DF1200CD1E900018CE893
S3150801D910030060680368D3F80C802B466146C0474C
S3150801D9203046FDF732F920F00048B749404673F012
S3150801D93001FE20B9B449404673F0F2FD50B108AB77
S3150801D94093E8030086E8030008A8FDF71DF913B05C
S3150801D950BDE8F08FD4F85490D4F858803946484633
S3150801D96001F0F0FB294601F02FFA01F0F1F98246A0
S3150801D97005903946404601F0A9FD294601F011FCFA
S3150801D98001F0FBFB8046206D03685B6939469847C1
S3150801D99083460146404673F007FC0146504673F03C
S3150801D9A0F9FA8046029094F87C30A3B994F8763057
S3150801D9B08BB194F8773073B994F878305BB901462E
S3150801D9C0E06E73F0ADFD002859D14146206F73F022
S3150801D9D089FD002853D1484601F033FA002F65D155
S3150801D9E0B02303FB0700112D62D805EB45035B0045
S3150801D9F02033184402F073F800285BD039464846AC
S3150801DA0001F0A0FB294601F0DFF901F0A3F94FF077
S3150801DA107E5A4FF00408CDF8008004F1200304F182
S3150801DA2010025146FDF75AFD0690E06D73F068FB4A
S3150801DA30CDF8008004F1400304F130025146FDF7A8
S3150801DA404DFD0790D4F864807049A06E73F060FCB0
S3150801DA500146404673F0A8FB8046C4F884000021BD
S3150801DA60584673F053FD00284ED00299206F73F083
S3150801DA7039FD002840F0D0800023039346E008A82A
S3150801DA80FDF783F805463046FDF77FF80146284637
S3150801DA9073F080FAD4F8801073F086FB5C4973F052
S3150801DAA037FC01463046FDF7BFF84DE700209AE7F7
S3150801DAB000209FE7484601F0C4F96FB9B02303FB7C
S3150801DAC00700037813F0100F08D03946484601F0CD
S3150801DAD039FB01F08CF99AE70020F2E7484601F094
S3150801DAE0B0F947B9B02303FB07031B7813F0200FDE
S3150801DAF003D148488BE70023F7E73946484601F042
S3150801DB0021FB01F077F982E70023039300215846A8
S3150801DB1073F0F2FC002840F082800023029394F807
S3150801DB207B303BB9039B002B40F08480029B002B82
S3150801DB3040F09B80D4F88480D4F860A04FF07C51E3
S3150801DB40504673F031FB04900146404673F0CAFC17
S3150801DB50002800F0A580049BC4F88430484601F0EB
S3150801DB6070F9002F40F0AC80B02303FB0703112D99
S3150801DB7000F2A88005EB450568002030184401F03D
S3150801DB80DEFF002840F0A08094F8793023B994F894
S3150801DB907A30002B00F0AB8094F87C303BB9039BBC
S3150801DBA0002B40F0C180029B002B40F0DE80002153
S3150801DBB0584673F0B5FC002840F0E280002158462B
S3150801DBC073F090FC002840F0FA803046FCF7DDFF40
S3150801DBD0002173F087FC002840F013813046FCF7DA
S3150801DBE0D4FF0A4973F09CFC002800F0168110AC9A
S3150801DBF006492046FCF7C4FF94E8030086E80300BB
S3150801DC002046FCF7C1FF08E1FFFF7F7F0000C842FD
S3150801DC100000E1440000C8410123039376E7029915
S3150801DC20E06E73F07DFC10B90023029377E70123B8
S3150801DC30029374E708A8FCF7A8FF82463046FCF76A
S3150801DC40A4FF0146504673F0A5F9764973F060FBC7
S3150801DC50014673F0A1F9616E73F0A6FA01464046D2
S3150801DC6073F098F9C4F8840064E708A8FCF78DFFF7
S3150801DC7082463046FCF789FF0146504673F08AF919
S3150801DC80684973F045FB014673F086F9616E73F0D6
S3150801DC908BFA0146404673F07FF9C4F8840049E7D8
S3150801DCA04FF07F51504673F07FFA8246014640464F
S3150801DCB073F036FC00283FF451AFC4F884A04DE751
S3150801DCC0002354E700205AE7484601F0BAF867B935
S3150801DCD0B02202FB0707F969059873F019FB01469B
S3150801DCE0584673F057F983464EE70027F3E74D493F
S3150801DCF0584673F059FAD4F8801073F055FA054668
S3150801DD004949D4F8840073F04FFA069973F04CFA2E
S3150801DD10079973F049FA0146284673F0F9FA01465C
S3150801DD203046FCF781FF37E708A8FCF72EFF3F4985
S3150801DD3073F0ECFB00283FF436AF08A8FCF725FF83
S3150801DD4005463046FCF721FF0146284673F022F9BD
S3150801DD50D4F8801073F028FA4FF07A5173F024FA48
S3150801DD6001463046FCF760FF2FE708A8FCF70DFFD0
S3150801DD704FF07C5173F0C0FB00283FF418AFDCE785
S3150801DD803046FCF702FF2A4973F0CAFB00283FF424
S3150801DD9015AF3046FCF7F9FE244973F0A3FB0028BA
S3150801DDA03FF40CAF0AAC22492046FCF7E9FE94E899
S3150801DDB0030086E803002046FCF7E6FE05E7304641
S3150801DDC0FCF7E3FE4FF07E5173F08CFB00283FF41D
S3150801DDD0FCAE3046FCF7D9FE4FF07C5173F0A0FB40
S3150801DDE000283FF4F2AE0CAC4FF07E512046FCF70A
S3150801DDF0C7FE94E8030086E803002046FCF7C4FE44
S3150801DE00E3E60EAC00212046FCF7BAFE94E80300CF
S3150801DE1086E803002046FCF7B7FE08A8FCF7B4FE1F
S3150801DE2095E500BF0000C842000061450000C742F1
S3150801DE300000C64210B504460A4B40F8683BFCF799
S3150801DE40A3FE04F16000FCF79FFE04F15800FCF7FD
S3150801DE509BFE04F15000FCF797FE034B2360204616
S3150801DE6010BD00BF243309080833090810B5044654
S3150801DE70FFF7E0FF8821204644F010FA204610BD3E
S3150801DE8090F84C30032B00D0704770B584B0044627
S3150801DE900D4600F168063046FCF777FE014628462E
S3150801DEA0FCF7C2FE3046FCF776FE01462846FCF72B
S3150801DEB0BBFE2846FCF769FE064604F15800FCF746
S3150801DEC064FE0146304673F00DFB20B1583494E8E0
S3150801DED0030085E803002846FCF757FE002173F086
S3150801DEE001FB98B92846FCF750FE0F4973F018FB59
S3150801DEF0C0B102AC0C492046FCF742FE94E8030087
S3150801DF0085E803002046FCF73FFE0BE06C4600213E
S3150801DF102046FCF735FE94E8030085E80300204611
S3150801DF20FCF732FE04B070BD0000C84290F84C30D0
S3150801DF30032B00D07047F0B589B0044600F160059F
S3150801DF402846FCF722FE064604F168073846FCF720
S3150801DF501CFE00F100412846FCF766FE3846FCF730
S3150801DF601AFE00F100412846FCF75EFE2846FCF73A
S3150801DF700CFE0146304673F017F9002173F0BCFA1E
S3150801DF8008B909B0F0BD6D462846FCF7F5FD04F160
S3150801DF90500395E8030083E803002846FCF7F4FDDF
S3150801DFA002AD2846FCF7E8FD04F1580395E803009D
S3150801DFB083E803002846FCF7E7FD04AD2846FCF78D
S3150801DFC0DBFD04F1600395E8030083E803002846B6
S3150801DFD0FCF7DAFD06AD2846FCF7CEFD95E8030009
S3150801DFE0C7E900012846FCF7CFFD022384F84C3027
S3150801DFF0D4E90423C4E91C23C3E7000038B5044661
S3150801E000224B0360224B03608164002580F84C5043
S3150801E0105030FCF7B1FD04F15800FCF7ADFD04F1F1
S3150801E0206000FCF7A9FD04F16800FCF7A5FD0022D4
S3150801E0300023C4E91C230021C4F88010C4E9022383
S3150801E040C4E90423C4E90623C4E90823A5621149DE
S3150801E050E16221630721A186E1860F21A1634FF4BD
S3150801E0607A61E163012184F8401084F8415084F80B
S3150801E070425084F8435084F8445084F8455084F853
S3150801E0804610C4E91E23204638BD00BF08330908D7
S3150801E09024330908CDCC6C4008307047C0E91C23ED
S3150801E0A0704708B56030FCF770FD08BD00F17001D6
S3150801E0B0D1E90001704790F84C00032814BF0020ED
S3150801E0C00120704770B504460D461646D1E902018E
S3150801E0D073F024F80F4973F01BF9034696E8030019
S3150801E0E084E80300AA6B0AB9204670BD1946204682
S3150801E0F0FCF734FEA86BC0EB0010800072F0FCFF41
S3150801E10001464FF07E5073F003F901462046FCF7AD
S3150801E11025FEE9E7002474492DE9F04F97B0054635
S3150801E1200292886C00287AD00C461E46FFF752F9EF
S3150801E130D0F8EC70002F79D0A06CFFF74BF9D0F826
S3150801E140F080B8F1000F75D0A06CFFF743F9D0F84D
S3150801E150F490B9F1000F71D03146384600F0F2FF5C
S3150801E160209900F031FE00F0F3FD82463146404623
S3150801E17001F0ACF9209901F014F800F0FEFF804691
S3150801E180D9F800305B69314648469847414673F0ED
S3150801E1900BF80146504672F0FDFE8046039094F84E
S3150801E1A0453053B90146E06A73F0A6F928B14146EC
S3150801E1B0206B73F0ABF9002844D1384600F041FED4
S3150801E1C0002E43D1B02303FB0600209B112B3FD819
S3150801E1D003EB43035B002033184401F080FC00285D
S3150801E1E038D03146384600F0ADFF209900F0ECFDF5
S3150801E1F000F0B0FD0746A06CFFF7ECF83946406B16
S3150801E20073F08EF9002851D0A06CFFF7E3F8476B3D
S3150801E2102A22002109A869F093FC002655E0284620
S3150801E220FCF7AAFC284617B0BDE8F08F2846FCF78C
S3150801E230A3FCF7E72846FCF79FFCF3E72846FCF71B
S3150801E2409BFCEFE72846FCF797FCEBE70020BCE7C9
S3150801E2500020C2E7384600F0F4FD76B9B02303FB87
S3150801E2600600037813F0100F09D03146384600F03E
S3150801E27069FF00F0BCFD0746BDE70020F1E7384617
S3150801E28000F0DFFD46B9B02303FB06031B7813F044
S3150801E290200F03D1724FAEE70023F7E73146384620
S3150801E2A000F050FF00F0A6FD0746A4E7A06CFFF7B3
S3150801E2B091F83946006C73F015F90028A8D0A06CBE
S3150801E2C0FFF788F8076CA3E70136022E7DDCA06C00
S3150801E2D0FFF780F806F10C0300EB83003946406826
S3150801E2E073F00AF90028EFD0A06CFFF773F806F16E
S3150801E2F0010B06F10D0300EB83003946406873F004
S3150801E30005F90028E0D04FF0000804970595B8F103
S3150801E310140F59DCA06CFFF75DF80BEB4B03C3EB4D
S3150801E320C3034344203300EB43039D88A06CFFF7E6
S3150801E33051F806EB4603C3EBC303434420335F009E
S3150801E34000EB43039888281A72F0DAFE0546A06C9A
S3150801E350FFF740F80BF10C0300EB8300D0F804A09B
S3150801E360A06CFFF737F806F10C034FEA830900EBB7
S3150801E37083004168504672F00DFE0146284672F048
S3150801E380C7FF0546A06CFFF725F88144D9F80410A4
S3150801E390049872F0FFFD294672F006FF0546A06C47
S3150801E3A0FFF718F80744B88872F0A6FE0146284612
S3150801E3B072F0F2FD16AB03EB480573F0F7F825F892
S3150801E3C0340C08F10108A2E7059D2649039872F065
S3150801E3D0EBFE0646A06CFEF7FDFF00F10804304689
S3150801E3E073F0E4F815230093234609AA002180B2A5
S3150801E3F0FFF75EF872F080FE1B4972F089FF064648
S3150801E400194973F08DF800B1174E14AC3146204600
S3150801E410FCF7B6FB94E80300219B83E8030020463A
S3150801E420FCF7B2FB07AC31462046FCF7A9FB029E76
S3150801E4303046FCF7AAFB00F100412046FCF7F4FB45
S3150801E4403046FCF7A8FB00F100412046FCF7ECFB3F
S3150801E45094E8030085E803002046FCF795FBE1E60E
S3150801E4600000C84100007A440000C8422DE9F04F77
S3150801E47091B002900F46154604920CAC2046FCF763
S3150801E4807BFB94E80300C5E900012046FCF77CFB09
S3150801E490B86C88B1FEF79EFFD0F8EC0098B100F091
S3150801E4A0D0FC059098B1BB6A0693A3B14FF0000A58
S3150801E4B0704B03939B468DE00298FCF75DFB02982F
S3150801E4C011B0BDE8F08F0298FCF756FBF7E7029802
S3150801E4D0FCF752FBF3E70298FCF74EFBEFE74FF028
S3150801E4E0000983E0079844F0ABF971E0002533E0B1
S3150801E4F00AA8FCF74AFB834608A8FCF753FBE0B9D0
S3150801E500039B23F000455C49284673F013F880B94C
S3150801E5105949284673F004F858B908A8FCF737FB97
S3150801E520039972F0DFFF40B108A8FCF730FB0390AE
S3150801E53003E008A8FCF72BFB03900AA8FCF724FBC9
S3150801E54008A8FCF721FB0134112C3EDCCED804EBDC
S3150801E55044056D0020354D442146404601F007F833
S3150801E5600646284601F0ABFA0028ECD008AD284645
S3150801E570FCF702FB304600F0DDFF024601950094E8
S3150801E580534639460AA8FFF7C7FD0AA8FCF70AFB4E
S3150801E5900028B1D12BF000453749284672F0CAFF49
S3150801E5A00028A5D13449284672F0BAFF00289FD120
S3150801E5B00AA8FCF7EAFA594672F094FF00289BD09C
S3150801E5C00AA8FCF7E2FA834696E7079844F038F971
S3150801E5D00AF1010ABAF1000F1BDCBAF1000F7FF448
S3150801E5E07EAF4FF0B009059B09FB0A3951460698DB
S3150801E5F001F032FA804609F18C030793184644F074
S3150801E600CFF899F8003013F0040F3FF46BAF0024EC
S3150801E6109AE72BF000441849204672F08BFFB0B9EF
S3150801E6201549204672F07CFF88B9039B23F0004404
S3150801E6301149204672F07EFF20B90F49204672F033
S3150801E6406FFF40B159460298FCF79AFA37E70298E4
S3150801E650FCF792FA33E70EAC03992046FCF790FAD9
S3150801E66094E80300049B83E803002046FCF78CFA30
S3150801E670E8E700BF0000C07FFFFF7F7F70B590B05D
S3150801E680044690F84630002B52D08168C268836FE1
S3150801E690C06F5B1842EB0002A367E267A06C002813
S3150801E6A000F08880FEF796FED0F8F430002B00F0D3
S3150801E6B08D80A06CFEF78EFED0F8F40003689B6887
S3150801E6C098470646824972F06FFD0546D4F88010D0
S3150801E6D0304672F05FFC20F0004025F0004172F0F0
S3150801E6E01FFF28B994F8433043B994F844302BB93D
S3150801E6F0C4F8806000220023C4E91E23A16FE26FDB
S3150801E700E56BE80E6B015B1B60F10000800040EAD7
S3150801E71093709B005B1940F10000C00040EA5370FA
S3150801E720DB00994272EB000352D394F8422042E08F
S3150801E7306D462846FCF720FA04F1500395E80300D4
S3150801E74083E803002846FCF71FFA02AD2846FCF7C2
S3150801E75013FA04F1580395E8030083E803002846F1
S3150801E760FCF712FA04AD2846FCF706FA04F1600331
S3150801E77095E8030083E803002846FCF705FA06AD89
S3150801E7802846FCF7F9F904F1680395E8030083E8DC
S3150801E79003002846FCF7F8F994F8403043B1002302
S3150801E7A084F84C3000220023C4E91E2310B070BD42
S3150801E7B00223F5E7002294F84C30022B3DD0032BB7
S3150801E7C076D03BB1022384F84C30EFE70022F2E71A
S3150801E7D00022F0E794F84030002BE7D123696269FB
S3150801E7E0A169E0695B1A62EB0002A18E394800FB58
S3150801E7F001F18B4272F1000303DA022384F84C30EB
S3150801E800D4E708AD04F1580221462846FFF72EFE43
S3150801E81004F1680295E8030082E8030004F1600345
S3150801E82083E8030004F1500282E803002846FCF756
S3150801E830ABF9032384F84C30B8E723696169206A88
S3150801E840656A1B1A61EB0501E08E224D05FB00F096
S3150801E850834271F10003A9DB1AB994F84130002B00
S3150801E860A4D00AAD04F1580221462846FFF7FEFD59
S3150801E87004F1600395E8030083E8030004F15006F8
S3150801E88086E803002846FCF77FF90CAD3246214697
S3150801E8902846FFF717FC04F1680395E8030083E8A7
S3150801E8A003002846FCF770F9032384F84C307DE70A
S3150801E8B00EAD04F1500221462846FFF703FC6834E1
S3150801E8C095E8030084E803002846FCF75DF96DE73F
S3150801E8D0CDCC4C3D80510100014B0360704700BF10
S3150801E8E04033090810B50446FFF7F6FF24212046F0
S3150801E8F043F0D4FC204610BD38B504460B4872F0E7
S3150801E90049FB0146204672F047FB05464FF07C510C
S3150801E91072F0FCFD38B10549204672F045FC2946DE
S3150801E92072F0F6FC38BD0020FCE700BF0000C842C3
S3150801E93038B50C4601460B4872F02CFB214672F09D
S3150801E9402BFB05464FF07C5172F0E0FD38B10549C5
S3150801E950204672F029FC294672F0DAFC38BD0020FF
S3150801E960FCE700BF0000C8420160426083609DF871
S3150801E9700030037370470000084A026000214161B4
S3150801E98000220276C16180F8202002718260C2608D
S3150801E9900274427464228274704700BF40330908C6
S3150801E9A00430704740697047007E7047C0697047F8
S3150801E9B090F8200070470000F8B50C46037C23B395
S3150801E9C0867C457CAE4220D9284672F095FB0746DF
S3150801E9D0214672F09BFDB8B9304672F08DFB21468F
S3150801E9E072F08AFD98B93946204672F0D3FA094978
S3150801E9F072F0DAFB0446701B72F082FB0146204670
S3150801EA0072F086FC044600E000242046F8BD014C5D
S3150801EA10FBE700BF0000C84210B50446084661611D
S3150801EA204FF07C5172F0B8FA72F09AFDC1B22176B4
S3150801EA30A06810B10368DB68984761692046FFF74B
S3150801EA40BBFFE0614FF07C5172F0A6FA72F088FDC7
S3150801EA50C1B284F82010E06810B10368DB689847F2
S3150801EA6010BD000070B504460D460379022B40D04F
S3150801EA70032B54D0012B02D00B68436101E08B684C
S3150801EA8043612B7B6BB1A5685DB12B68DE684FF0DE
S3150801EA907C51606972F080FA72F062FD014628467F
S3150801EAA0B047A568002D50D02B689E684FF07C5161
S3150801EAB0606972F071FA72F053FD01462846B04753
S3150801EAC0C0B2207661692046FFF776FFE061E56806
S3150801EAD0002D43D02B689E684FF07C5172F05CFA8A
S3150801EAE072F03EFD01462846B047C0B284F82000C0
S3150801EAF070BD49682868FFF7FFFE064660611B4935
S3150801EB0072F004FD10B1194B6361BAE70021304672
S3150801EB1072F0F2FC0028B4D000236361B1E74968BA
S3150801EB202868FFF705FF06466061104972F0EEFC9A
S3150801EB3010B10E4B6361A4E70021304672F0DCFC8C
S3150801EB4000289ED0002363619BE74FF07C516069E2
S3150801EB5072F022FA72F004FDC0B2B2E74FF07C51AE
S3150801EB6072F01AFA72F0FCFCC0B2BFE70000C842A4
S3150801EB70014B0360704700BF5033090810B50446BE
S3150801EB80FFF7F6FF2021204643F088FB204610BDFB
S3150801EB90C0E90023009B8360019BC3609DF8083090
S3150801EBA003749DF80C3043749DF8103083749DF8F6
S3150801EBB01430C3749DF818300375704730B40B4A86
S3150801EBC00260002202750A4941604FF47A71816038
S3150801EBD04FF46161C1600274012141748274C27487
S3150801EBE000240025C0E9064530BC704750330908A2
S3150801EBF00000204104307047007D0238C0B2012868
S3150801EC008CBF002001207047F8B504460B460A7CE4
S3150801EC102AB98A7CA2B94D7C15B9CD7C00E00025BC
S3150801EC20267C86B11F7D6FB9D968986872F0B2F9EA
S3150801EC3020F00041606872F069FC20B93E4602E0A6
S3150801EC400025EDE7002605B935462846F8BD70B515
S3150801EC500446437C8BB1837C8BB90B684D68866906
S3150801EC60C2699E1945EB02058661C561037D032BC1
S3150801EC7064D8DFE803F00712303E037570BD02233E
S3150801EC800375FBE7FFF7C0FF0028F7D001232375BB
S3150801EC9000220023C4E90623F0E7FFF7B5FF10B900
S3150801ECA000232375EAE7A168CA0E4B015B1A62F1D4
S3150801ECB00002920042EA93729B005B1842F100023D
S3150801ECC0D20042EA5372DB009E4275EB0203D5D3AA
S3150801ECD002232375D2E7C37C002BCFD1FFF794FF1C
S3150801ECE00028CBD10323237500220023C4E9062378
S3150801ECF0C4E7FFF789FF10B102232375BEE7E06871
S3150801ED00C20E43011B1A62F10002520242EAD352B1
S3150801ED105B021B1842F100024FEA821C4CEA936C13
S3150801ED209901CB1A6CEB02021B1842F100029E42B2
S3150801ED3075EB0203A2D3002323759FE7002303750E
S3150801ED409CE700220260426070470160426070479A
S3150801ED50006870474068704770B506460546112435
S3150801ED6004E02846FFF7EDFF0835013C002CF8DAE8
S3150801ED700023C6F89030C6F89430C6F89830C6F81D
S3150801ED809C30C6F8A030304670BD2DE9F8430646DA
S3150801ED90894690461F460546112404E02846FFF792
S3150801EDA0D0FF0835013C002CF8DAC6F89090C6F871
S3150801EDB09480C6F89870089BC6F89C30099BC6F8DB
S3150801EDC0A0303046BDE8F883112902D800EBC1000E
S3150801EDD0704700207047C0F890107047D0F890002F
S3150801EDE07047D0F894007047D0F898007047D0F86B
S3150801EDF09C007047D0F8A000704770B50446416082
S3150801EE0000F108060025002D05DB3046FFF7A4FFB3
S3150801EE10A436013DF7E70023C4F8AC30C4F8B03096
S3150801EE20012323800023A370E370204670BD10F1EF
S3150801EE30080205D000F1AC039A4201D0A43BFBE7D6
S3150801EE4070474068704770472DE9F041AEB00746F4
S3150801EE500026002E39DC7B68CEB94FF0B00808FBD6
S3150801EE60063808F18C08404643F09AFC00210191C6
S3150801EE7000910B460A4603A8FFF787FFA42202FB67
S3150801EE80067003A9083068F069FD002416E04FF002
S3150801EE900008E6E700212CAD0A462846FFF755FF8C
S3150801EEA0A42006FB00F0083021463844FFF78CFF02
S3150801EEB0034695E8030083E803000134112CE9DDD4
S3150801EEC0404643F0BDFC0136C3E72EB0BDE8F081EC
S3150801EED02DE9F04FB9B08346099192469946002328
S3150801EEE0029308930693002305930393029A002A33
S3150801EEF000F30181DBF80430002A55D14FF0B00840
S3150801EF0008FB023808F18C030793184643F048FCBE
S3150801EF1098F8003013F0040F49D09BF802203AB153
S3150801EF20BBF8002002998A4245DD069A013206920B
S3150801EF3003F008030493099E33689C68B8F8040033
S3150801EF4072F0DAF801463046A047054633689C68F0
S3150801EF50B8F8060072F0D0F801463046A0470746D1
S3150801EF6033689C68B8F8080072F0C6F8014630465E
S3150801EF70A0470646D9F800309C68B8F80A0072F02E
S3150801EF80BBF801464846A0470A90D9F800309C6864
S3150801EF90B8F80C0072F0B0F801464846A0470B9045
S3150801EFA0049B83B9002557E04FF00008AAE70798A4
S3150801EFB043F046FC9BE00299B1EB420FB8DA089A96
S3150801EFC001320892B4E701900A9B009333463A4608
S3150801EFD029460DA8FFF7D9FEA422029B02FB03B01E
S3150801EFE00DA9083068F0BAFCDCE700243CE098F883
S3150801EFF0003013F0100F5AD00A9F5BE098F80030E2
S3150801F00013F0200F01D00B9F54E0002752E036ACD5
S3150801F0103A4631462046FFF798FEA420029B03FB99
S3150801F02000F0083029465844FFF7CEFE034694E817
S3150801F030030083E8030040E0029AB2EB430F0ADAC1
S3150801F0403146059871F0A8FF059004E0314603980A
S3150801F05071F0A2FF03900135112D3DDCC5D805EBF2
S3150801F0604504640020344444204600F028FD002865
S3150801F070F1D0DAF800309E68204600F086FD72F07D
S3150801F0803BF801465046B0470646D9F800309F6816
S3150801F090204600F07EFD72F02FF801464846B84733
S3150801F0A00746204600F01BFD20B9002D9FD0012DF3
S3150801F0B0A4D00027049B002BA9D19BF80230002B72
S3150801F0C0C4D0BBF80030029A9342B5DD31460398A5
S3150801F0D071F062FF0390BEE7049B2BB198F80030EC
S3150801F0E023F0080388F80030079843F0A9FB029B30
S3150801F0F001330293FAE69BF80230D3B1069B089ACC
S3150801F100934203DD039BCBF8AC3015E0069B089AC6
S3150801F110934203DA059BCBF8AC300DE005990398C9
S3150801F12071F03AFF4FF07C5172F03EF8CBF8AC0023
S3150801F13002E0039BCBF8AC30429BCBF8B03039B038
S3150801F140BDE8F08F0B4629B9A42202FB03F3083365
S3150801F1501844704700207047C37813B1D0F8B0003F
S3150801F1607047D0F8AC0070470022026042608260A6
S3150801F1707047016042608360704700687047406865
S3150801F18070478068704770B506460546112404E045
S3150801F1902846FFF7E9FF0C35013C002CF8DA304622
S3150801F1A070BD112904D801EB410100EB81007047BC
S3150801F1B00020704770B50446054645F8041B00262D
S3150801F1C0002E05DB2846FFF7DEFFD835013EF7E7B7
S3150801F1D00022C4F8DC20C4F8E020FF2384F8E430D8
S3150801F1E084F8E530C4F8E82084F8EC3084F8ED308A
S3150801F1F0002384F8EE30204670BD021D05D000F1CB
S3150801F200DC039A4201D0D83BFBE770470068704798
S3150801F2102DE9F04F89B083460F464FF00008B8F143
S3150801F220000F46DCDBF80030B8F1000F10D14FF0C3
S3150801F230B00A0AFB083A4FF0D80909FB08B909F1DF
S3150801F24004090AF18C0A504643F0AAFA002528E077
S3150801F2504FF0000AEFE729464846FFF7A2FF0446A2
S3150801F260FFF78BFF02902046FFF789FF03902046A0
S3150801F270FFF787FF04903B689E680195CDF80080EB
S3150801F28004AB03AA02A93846B04705AE049B039A04
S3150801F29002993046FFF76DFF96E8070084E80700F4
S3150801F2A00135112DD7DD504643F0CAFA08F1010898
S3150801F2B0B5E709B0BDE8F08F2DE9F04F91B004909C
S3150801F2C088460B689B680846984700274FF0000B4D
S3150801F2D00897079706970597CDF80CB0594B0293EF
S3150801F2E05EE04FF0000A65E0099843F0A9FA56E096
S3150801F2F0002617E00399284672F012F920B17BB26D
S3150801F300079363B2089303952946584671F044FE5C
S3150801F31083460134112C3FDCEAD804EB4406760017
S3150801F3202036564421464846FFF73BFF05463046F8
S3150801F33000F0C5FB0028ECD02846FFF71EFF0A900F
S3150801F3402846FFF71CFF0B902846FFF71AFF0C907B
S3150801F350D8F800301E69019400970CAB0BAA0AA9CC
S3150801F3604046B0470DAE0C9B0B9A0A993046FFF7FB
S3150801F37000FF96E8070085E807002846FFF7FDFE27
S3150801F3800546029972F0AEF80028B3D07BB2059310
S3150801F39063B206930295B7E7099843F051FA013724
S3150801F3A0002F1BDC049B1B68002F9AD14FF0B00A73
S3150801F3B00AFB073A4FF0D809049B09FB073909F1FB
S3150801F3C004090AF18C030993184643F0E9F99AF8F6
S3150801F3D0003013F0040F87D000249BE7D8F80030DB
S3150801F3E0DB684046984718B10123049A82F8EE3043
S3150801F3F0D8F800305B69404698471249029C204676
S3150801F40072F066F840B9049BC3F8E040059A83F8A0
S3150801F410E420069A83F8E5200021039C204672F031
S3150801F42057F840B9049BC3F8E840079A83F8EC20DB
S3150801F430089A83F8ED20049BC3F8DCB011B0BDE847
S3150801F440F08F00BF9AF979442DE9F04F85B08346CC
S3150801F45088464FF00009B9F1000F2FDCDBF80030C0
S3150801F460B9F1000F0ED14FF0B00A0AFB093AD827B5
S3150801F47007FB09B704370AF18C0A504643F090F99D
S3150801F480002613E04FF0000AF1E731463846FFF748
S3150801F49088FE04460C4A01AD134641462846FFF745
S3150801F4A068FE95E8070084E807000136112EECDDB1
S3150801F4B0504643F0C5F909F10109CCE701238BF858
S3150801F4C0EE3005B0BDE8F08F0000C07F21B9D82223
S3150801F4D002FB01000430704700207047D0F8DC00B9
S3150801F4E07047D0F8E000704790F9E5007047D0F80A
S3150801F4F0E800704790F9ED00704790F8EE00704704
S3150801F500002380F8EE30704710B504460249FBF730
S3150801F51037FB204610BD00BF0000C07F10B504466A
S3150801F520FBF72EFB204610BD10B50446FBF72CFB56
S3150801F530204610BD704770B506460546112404E0FD
S3150801F5402846FFF7E1FF0835013C002CF8DA30467A
S3150801F55070BD38B5054640B100F1900403E0083C9A
S3150801F5602046FFF7E1FFA542F9D1284638BD112902
S3150801F57002D800EBC1007047002070470160426065
S3150801F58003729DF800304372704770B5044605460C
S3150801F59045F8041B0026002E05DB2846FFF7CBFF9E
S3150801F5A09035013EF7E70023C4F89430FF2284F82A
S3150801F5B0982084F899204FF6FF71A4F89A10C4F898
S3150801F5C09C3084F8A02084F8A120A4F8A210C4F8DD
S3150801F5D0A430C4F8A830C4F8AC30002384F8B0309D
S3150801F5E084F8B130204670BD70B50446061D08D0B2
S3150801F5F000F19405AE4204D0903D2846FFF7A9FFD5
S3150801F600F8E7204670BD0068704700002DE9F04F05
S3150801F6108FB009908A464FF00009C8460022009229
S3150801F6204FF0FF33069305930293019208930793CC
S3150801F6300493039267E04FFA89F304936BB2079335
S3150801F6400FFA88F3089303942146019871F04AFF4B
S3150801F65010B9029B002B08DA4FFA89F302936BB2B1
S3150801F66005930FFA88F3069301940AAF21463846A3
S3150801F670FFF754FF97E8030086E803003846FFF7CB
S3150801F68053FF08F101080135112D3ADC2946584680
S3150801F690FFF76DFF0646DAF800309B682A464946A9
S3150801F6A050469847044620F000473D49384671F0D0
S3150801F6B041FFC8B93A49384671F032FFA0B9214627
S3150801F6C0009871F069FC00900021204671F01EFF38
S3150801F6D00028B9D02146039871F022FF0028AAD143
S3150801F6E0049B002BB0DAA6E70CAC2E492046FFF79F
S3150801F6F015FF94E8030086E803002046FFF714FF88
S3150801F700C1E709F10109B9F1000F08DC09EBC90BD9
S3150801F710099B03EB0B1B0BF1040B0025B4E7B8F1AE
S3150801F720000F24D0099C039AC4F89420049A84F8FB
S3150801F7309820079A84F89920089AA4F89A20019A99
S3150801F740C4F89C20029A84F8A020059B84F8A1306D
S3150801F750069BA4F8A230404671F0D2FC01460098F7
S3150801F76071F0D6FDC4F8A4000FB0BDE8F08F0022F1
S3150801F7700998C0F89420FF2380F8983080F89930CA
S3150801F7804FF6FF71A0F89A10C0F89C2080F8A030B7
S3150801F79080F8A130A0F8A210C0F8A420E4E700BFC1
S3150801F7A0FFFF7F7F0000C07F2DE9F04F93B00D90DA
S3150801F7B04B7A002B40F028818846086803689B68C5
S3150801F7C09847D8F8040003689B6898474FF0000AE1
S3150801F7D0CDF838A0002203929D4B0193D34602929D
S3150801F7E04FF0FF330C930B93089305920A930993F1
S3150801F7F00793049293E04FF000099DE00F9843F0B8
S3150801F8001FF88AE00F9843F01BF80E9B01330E93FD
S3150801F81083E0002438E000253EE098F80830002B04
S3150801F82031D110AD8B492846FFF778FE95E80300DC
S3150801F83087E803002846FFF777FE24E04FFA8AF3A4
S3150801F840079363B209930FFA8BF30A930495294632
S3150801F850059871F047FE10B9089B002B08DA4FFA94
S3150801F8608AF3089363B20B930FFA8BF30C930595FE
S3150801F870D8F804000368DD68234652463946A84786
S3150801F8800BF1010B01960134112C43DCC3D804EBAF
S3150801F89044056D0020354D4421460698FFF767FE5D
S3150801F8A00746284600F00BF90028B6D0D8F80050CC
S3150801F8B02B68DE683846FFF73DFE07462346524663
S3150801F8C001462846B0473846FBF75FF90546014623
S3150801F8D0029871F061FB0290D8F8000003681B6971
S3150801F8E0984706460146039871F056FB0390314640
S3150801F8F0019871F015FE18B9BBF1000F00D0019EF1
S3150801F9002946049871F00CFE002897D1079B002B15
S3150801F9109DDA93E70F9842F093FF0AF1010ABAF1CB
S3150801F920000F27DC0D9B1B68BAF1000F7FF463AF4C
S3150801F9304FF0B00909FB0A390AEBCA030D9A02EB23
S3150801F94003130433069309F18C030F93184642F007
S3150801F95027FF98F80830002B3FF45BAF99F8003081
S3150801F96013F0010F3FF44AAF13F0040F3FF44AAF07
S3150801F970002489E7D8F8040003681B699847D8F872
S3150801F980000003685B6A9847D8F800000368DB69DA
S3150801F99098470D9C84F8B000D8F8000003681B6AE4
S3150801F9A09847254684F8B1000E9B6BBBBBF1000F47
S3150801F9B02DD0049BC4F89430079B84F89830099B92
S3150801F9C084F899300A9BA4F89A30059BC4F89C30B0
S3150801F9D0089B84F8A0300B9B84F8A1300C9BA4F8F3
S3150801F9E0A230584671F08CFB04460146029871F024
S3150801F9F08FFCC5F8A400019BC5F8A83021460398D9
S3150801FA0071F086FCC5F8AC0013B0BDE8F08F98F824
S3150801FA100830002BF8D100230D98C0F89430FF2246
S3150801FA2080F8982080F899204FF6FF71A0F89A106F
S3150801FA30C0F89C3080F8A02080F8A120A0F8A21078
S3150801FA40C0F8A430C0F8A830C0F8AC30DCE700BF75
S3150801FA509A3F1C460000C07F29B901EBC10300EBA0
S3150801FA6003100430704700207047D0F8940070479F
S3150801FA7090F999007047D0F89C00704790F9A10059
S3150801FA807047D0F8A4007047D0F8AC00704790F8DA
S3150801FA90B000704790F8B10070470022028042809A
S3150801FAA0027170477047037903F0FE0303715BB275
S3150801FAB019B101221343037170470022FAE700794D
S3150801FAC000F001007047037903F0FD0303715BB28F
S3150801FAD019B102221343037170470022FAE700792C
S3150801FAE0C0F340007047037903F0EF0303715BB27B
S3150801FAF019B110221343037170470022FAE70079FE
S3150801FB00C0F300107047037903F0FB0303715BB27E
S3150801FB1019B104221343037170470022FAE70079E9
S3150801FB20C0F380007047037903F0F70303715BB2F2
S3150801FB3019B108221343037170470022FAE70079C5
S3150801FB40C0F3C0007047037903F0DF0303715BB2AA
S3150801FB5019B120221343037170470022FAE700798D
S3150801FB60C0F340107047037903F0BF0303715BB21A
S3150801FB7019B140221343037170470022FAE700794D
S3150801FB80C0F3801070470180704700887047418034
S3150801FB90704740887047007970472DE9F04791F81A
S3150801FBA00C80B8F1000F43D1D1F808A00027002F27
S3150801FBB040DCB7B9B02606FB07A606F18C0948460C
S3150801FBC042F0EEFD337813F0040F0CD013F0100F4A
S3150801FBD002D113F0200F0AD0484642F031FE013710
S3150801FBE0E5E70026E9E7484642F02AFEF7E7002559
S3150801FBF002E0002408E00135112D11DCF9D805EBE6
S3150801FC0045046400203434442046FFF758FF002891
S3150801FC10F1D02046FFF763FF0028ECD0444600E008
S3150801FC200124484642F00CFE002CD8D0A04601E03B
S3150801FC304FF000084046BDE8F0872DE9F04791F8F6
S3150801FC400C80B8F1000F43D1D1F808A00027002F86
S3150801FC5040DC9FB9B02606FB07A606F18C09484683
S3150801FC6042F09EFD337813F0040F09D013F0400FCC
S3150801FC700AD113F0800F07D100250EE00026ECE724
S3150801FC80484642F0DDFD21E0484642F0D9FD4FF0F5
S3150801FC9001081FE0002408E00135112D11DCF9D80F
S3150801FCA005EB45046400203434442046FFF707FF7A
S3150801FCB00028F1D02046FFF722FF04460028EBD0A2
S3150801FCC000E04446484642F0BBFD34B90137BEE779
S3150801FCD04FF000084046BDE8F087A046FAE7C0E9BC
S3150801FCE00023009B83609DF804300373704700006E
S3150801FCF030B4094A02600022027442F2107141606E
S3150801FD000121816001734273827300240025C0E9D1
S3150801FD10064530BC704700BF60330908014B0360D4
S3150801FD20704700BF6033090810B50446024B0360EB
S3150801FD30FFF7F4FF204610BD8833090810B50446BD
S3150801FD40044B0360FFF7EAFF2021204642F0A6FA9A
S3150801FD50204610BD8833090810B50446024B0360D6
S3150801FD60FFF7DCFF204610BD7433090810B50446B9
S3150801FD70044B0360FFF7D2FF2021204642F08EFA9A
S3150801FD80204610BD743309080430704738B5044657
S3150801FD90037B8BB1437B8BB908684A68A3691B1837
S3150801FDA0E06942EB0002A361E261237C032B72D86E
S3150801FDB0DFE803F007143646037438BD02230374DB
S3150801FDC0FBE723689B68204698470028F5D001235E
S3150801FDD0237400220023C4E90623EEE723689B68FF
S3150801FDE02046984710B900232374E6E7A169E2691A
S3150801FDF06568E80E6B015B1B60F10000800040EA54
S3150801FE0093709B005B1940F10000C00040EA5370F3
S3150801FE10DB00994272EB0003CFD302232374CCE7AC
S3150801FE20A37B002BC9D123689B68204698470028E5
S3150801FE30C3D10323237400220023C4E90623BCE7A4
S3150801FE4023689B682046984710B102232374B4E7B8
S3150801FE50A069E169A568EA0E6B015B1B62F1000204
S3150801FE60520242EAD3525B025B1942F100024FEA9F
S3150801FE70821E4EEA936E4FEA831CBCEB03036EEBBC
S3150801FE8002025B1942F10002984271EB020394D314
S3150801FE900023237491E7002323748EE7007C02383C
S3150801FEA0C0B201288CBF002001207047024A0260B7
S3150801FEB0024A0260704700BFE8350908802E090822
S3150801FEC080687047024A0260024A0260704700BFB2
S3150801FED000360908802E090880687047024A0260C0
S3150801FEE0024A0260704700BF18360908802E0908C1
S3150801FEF080687047024A0260024A0260704700BF82
S3150801FF0030360908802E090880687047024A02605F
S3150801FF10024A0260704700BFD0350908802E0908D9
S3150801FF208068704710B50446FFF7C0FF0C212046CC
S3150801FF3042F0B4F9204610BD10B50446FFF7C2FFDA
S3150801FF400C21204642F0AAF9204610BD10B50446F8
S3150801FF50FFF7C4FF0C21204642F0A0F9204610BD48
S3150801FF6010B50446FFF7C6FF0C21204642F096F964
S3150801FF70204610BD10B50446FFF7C8FF0C212046E0
S3150801FF8042F08CF9204610BD044A0260044A026018
S3150801FF90002282604FF07E5242607047802E090827
S3150801FFA0E835090804307047044A0260044A0260C9
S3150801FFB0002282604FF07E5242607047802E090807
S3150801FFC00036090804307047044A0260044A026090
S3150801FFD0002282604FF07E5242607047802E0908E7
S3150801FFE01836090804307047044A0260044A026058
S3150801FFF0002282604FF07E5242607047802E0908C7
S315080200003036090804307047044A0260044A02601E
S31508020010002282604FF07E5242607047802E0908A5
S31508020020D035090804307047F0B5A5B004460D4628
S315080200300C4E44273A46314613A867F08FFC3A46D7
S31508020040F11902A867F08AFC2946606871F0ACF8D3
S31508020050A0601123009302AB13AA0021FBF73EFA14
S3150802006025B0F0BD94330908F0B5A5B004460D468F
S315080200700D4E44273A4606F1880113A867F06EFC2E
S315080200803A46F11902A867F069FC2946606871F0D8
S315080200908BF8A0601123009302AB13AA0021FBF789
S315080200A01DFA25B0F0BD00BF94330908F0B5A7B014
S315080200B004460D460D4E48273A4606F1CC0114A8C9
S315080200C067F04CFC3A4606F58A7102A867F046FCC8
S315080200D02946606871F068F8A0601223009302ABA3
S315080200E014AA0021FBF7FAF927B0F0BD94330908E0
S315080200F0F0B5A7B004460D460D4E48273A4606F512
S31508020100AE7114A867F02AFC3A4606F58A7102A867
S3150802011067F024FC2946606871F046F8A06012234D
S31508020120009302AB14AA0021FBF7D8F927B0F0BD59
S3150802013094330908F0B5A7B004460D460D4E482774
S315080201403A4606F5D27114A867F008FC3A4606F54F
S315080201508A7102A867F002FC2946606871F024F8E1
S31508020160A0601223009302AB14AA0021FBF7B6F98A
S3150802017027B0F0BD94330908014B0360704700BFEE
S315080201804836090810B50446FFF7F6FF2821204627
S3150802019042F084F8204610BDC0E900239DF80030DD
S315080201A003729DF8043043727047000030B40A4A5D
S315080201B002600022027400240025C0E9064580F880
S315080201C020203C2141604FF46161816002734273D1
S315080201D0827330BC704700BF48360908043070473E
S315080201E0007C0238C0B201288CBF0020012070476B
S315080201F090F8200070470B7A0BB9487A70470020AE
S31508020200704738B50446037B4BB10D46437B43B969
S31508020210037C032B53D8DFE803F007142B3B037444
S3150802022038BD02230374FBE7FFF7E5FF84F82000D5
S315080202300028F5D001232374D5E90023C4E906234F
S31508020240EEE7FFF7D8FF84F8200010B900232374DD
S31508020250E6E72B686A68A169E0695B1A62EB000245
S3150802026061688B4272F10003DADB02232374D7E753
S31508020270837B002BD4D1FFF7BEFF84F82000002829
S31508020280CED103232374D5E90023C4E90623C7E79D
S31508020290FFF7B1FF84F8200010B102232374BFE7E9
S315080202A02B686A68A169E0695B1A62EB0002A168B9
S315080202B08B4272F10003B3DB00232374B0E70023F9
S315080202C00374ADE7014B0360704700BF583609084F
S315080202D010B50446FFF7F6FF1821204641F0DEFF67
S315080202E0204610BDC0E900239DF80030037270470E
S315080202F030B4074A026000220273032141600121D9
S315080203000172427200240025C0E9044530BC7047D8
S315080203105836090804307047037A93B130B50A682B
S315080203200469436914194A6842EB03030461436189
S31508020330027B012A11D0022A02D022B100230373BA
S3150802034030BD037370470B7A002BF9D00123037370
S3150802035000220023C0E90423F2E7427A002AEFD1F9
S315080203604568E90E6A01521B61F10001490241EA38
S31508020370D2515202521941F100014FEA811E4EEA48
S31508020380926E4FEA821CBCEB02026EEB0101521915
S3150802039041F1000194428B41D2D302230373CFE782
S315080203A0007B012814BF00200120704710B590F881
S315080203B004C0CCF3810E4FEA5C1CBCF1020F01D0DB
S315080203C0002010BD44795FFA81FC644501D0002003
S315080203D0F7E78479B4EB112F01D00020F1E7C17950
S315080203E0914201D00020ECE7CEF1040E9E4501D0E1
S315080203F00020E6E70120E4E703795B09032B01D035
S315080204000020704790F805C0CBB29C4501D0002069
S3150802041070478379B3EB112F01D000207047C37957
S31508020420934201D0002070470120704710B5044658
S31508020430074B40F85C3B42F024FA04F128003EF0F0
S315080204408FFB04F110003EF08BFB204610BD00BF67
S315080204506836090810B50446FFF7E8FF80212046EA
S3150802046041F01CFF204610BD00B587B0844601F551
S31508020470C0610020049005904FF0400E8DF810E000
S315080204808DF81120120A8DF812208DF813300823E0
S315080204908DF80C308DF80E008DF80D00009101AB29
S315080204A006AA12E9030083E80300694660461CF0BF
S315080204B0D1FB07B05DF804FB10B586B08646BDF8D9
S315080204C020C001F5C0610020049005902B248DF808
S315080204D010408DF81120120A8DF812208DF813306B
S315080204E08DF814C04FEA1C2C8DF815C008238DF818
S315080204F00C308DF80E008DF80D00009101AB06AA9E
S3150802050012E9030083E80300694670461CF0A2FB61
S3150802051006B010BD00B587B0844601F5007100200B
S31508020520049005908DF810208DF8113008238DF867
S315080205300C308DF80E008DF80D00009101AB06AA5D
S3150802054012E9030083E80300694660461CF082FB51
S3150802055007B05DF804FB017042707047F8B50446AF
S3150802056006461D4B46F8103B30463EF0B7FB04F1F3
S31508020570280738463EF0B2FB002323646364A3646B
S31508020580002584F84C5084F84D5084F84E50A4F84F
S315080205905050A4F8525084F8545084F8555084F8B0
S315080205A0565084F8585084F8595004F15C0042F0C9
S315080205B0E9F82571162363710123A3713223238176
S315080205C064236381257330463EF0D5FA38463EF0F9
S315080205D0D2FA2046F8BD00BF683609082DE9F84F59
S315080205E0067B16B304460D464B7B002B40F0CA80A9
S315080205F0437903F5C07103F520702A688A4217D039
S31508020600824202D12A7B082A2ED003F5B06704F16A
S315080206105C08404642F0C4F894F85890404642F0C6
S315080206200FF92B68BB425ED000263046BDE8F88F2C
S31508020630297B0229E4D904F15C07384642F0B0F86E
S315080206402B7984F84C306B7984F84D30AB7984F881
S315080206504E30012384F85630384642F0F1F804F158
S3150802066010003EF004FBE0E795F804A0AB7995F894
S31508020670058048EA03282B7AEF7947EA032795F893
S31508020680099095F80BB0AB7A43EA0B2B04F15C059B
S31508020690284642F085F8BAF1010F0DD0B9F1010FDB
S315080206A019D0012384F85630284642F0C9F804F1D5
S315080206B010003EF0DCFAB8E7404670F021FD3249F8
S315080206C070F072FD2064384670F01AFD2E4970F0FB
S315080206D06BFD6064E2E7584670F00EFD2B4970F038
S315080206E063FDA064DDE72B7B082B01D000269CE77F
S315080206F009F1FF39B9F1030F97D8DFE809F00215B6
S3150802070029360223012244F210012846FFF74EFE3B
S3150802071000288AD06A7A2B7A43EA0223A4F8503050
S31508020720022384F8593080E702231A4644F210015C
S315080207302846FFF73BFE00283FF477AF6A7A2B7A02
S3150802074043EA0223A4F85230022384F859306CE7AC
S31508020750012244F210012846FFF74EFE00283FF414
S3150802076064AF022384F859305FE7022244F210018B
S315080207702846FFF741FE00283FF457AF022384F8C4
S31508020780593052E7002650E700007A44CDCCCC3DDA
S315080207900430704770B50446057BE5B10B78F3B1B2
S315080207A0012384F854304B78DBB1012384F85530A1
S315080207B004F15C06304641F0F3FF94F8563023B153
S315080207C094F85820052A0ED01D46304642F038F8CD
S315080207D084F8575070BD002380F85730FAE7002393
S315080207E0DFE70023E2E794F84C20032A08D094F8BE
S315080207F04E20022A06D094F84D202AB11D46E4E777
S315080208001D46E2E71D46E0E70025DEE738B5044661
S3150802081000F15C05284641F0C3FF94F85640284685
S3150802082042F00EF8204638BD90F85800052814BF45
S3150802083000200120704738B5044600F15C052846B9
S3150802084041F0AEFF246C284641F0FAFF204638BD37
S3150802085038B5044600F15C05284641F0A1FF646CF0
S31508020860284641F0EDFF204638BD38B5044600F16A
S315080208705C05284641F094FF94F84C40284641F01E
S31508020880DFFF204638BD38B5044600F15C05284628
S3150802089041F086FF94F84D40284641F0D1FF2046A4
S315080208A038BD38B5044600F15C05284641F078FFA4
S315080208B094F84E40284641F0C3FF204638BD90F8CA
S315080208C05700704770B504460D4600F15C0630467F
S315080208D041F066FF84F85850304641F0B1FF0023D4
S315080208E084F8593070BD0000F0B583B00446037B26
S315080208F01BB300F1100528463EF0AFF9824B984229
S315080209002BD804F15C06304641F04AFF94F856703B
S3150802091094F85850304641F093FF6B1EDBB2032B16
S3150802092003D894F85930012B26D0042D00F2D08032
S31508020930DFE805F02E4E6E92B00010303EF097F9C1
S3150802094004F15C05284641F02BFF002384F8563053
S31508020950284641F075FF03B0F0BD04F15C06304647
S3150802096041F01EFF002384F85630304641F068FFF6
S3150802097028463EF07CF9C4E704F128003EF06DF9FA
S31508020980614B9842D1D900212046FFF79BFFCCE75D
S3150802099004F1280528463EF060F95C4B984208D8CF
S315080209A0002FD8D0A37973B101212046FFF78AFF19
S315080209B0D1E700231A4661792079FFF7ABFD28466D
S315080209C03EF055F9ECE705212046FFF77BFFC2E723
